:020000040800F2
:1020000000B9002045210008856200080F22000861
:10201000695E0008192D0008F9830008000000001F
:10202000000000000000000000000000697B0008C4
:10203000133F00080000000097210008417E0008BF
:102040005F2100085F2100085F2100085F21000870
:102050005F2100085F2100085F2100085F21000860
:102060005F2100085F2100085F2100085F21000850
:10207000893E0008953E0008A13E0008AD3E0008DC
:10208000B93E0008C53E00085F2100085F21000836
:102090005F2100085F2100085F2100085F21000820
:1020A0005F2100085F2100085F2100085F21000810
:1020B0005F2100085F2100085F2100085F21000800
:1020C0005F2100085F2100085F2100085F210008F0
:1020D0005F210008D5810008ED8100080582000815
:1020E0005F2100085F2100085F2100085F210008D0
:1020F0005F2100085F2100085F2100085F210008C0
:102100005F2100085F2100085F2100085F210008AF
:102110000D7F00085F2100085F2100085F21000893
:102120005F2100085F210008D13E0008DD3E000865
:10213000DFF80CD000F07EFC00480047AF2A000812
:1021400000B900200648804706480047FEE7FEE742
:10215000FEE7FEE7FEE7FEE7FEE7FEE7FEE7FEE757
:10216000097F000831210008EFF3108072B6704734
:1021700080F310887047334A1368012B04D04FF066
:1021800001031360304A1060304A116030484FF04C
:10219000805101607047EFF3108272B629480168E0
:1021A00091B14FF0000101602748016829B1EFF3B8
:1021B000098121E9F00F0068016024490968096874
:1021C000B1E8F00F81F3098882F310884EF0040E15
:1021D00070471E4908601C494FF00000086019490B
:1021E0004FF0010008601B484FF47F01D0F8002039
:1021F00041EA0201016016484FF080510160164823
:102200000068006880F3088861B662B670471EF007
:10221000040F0CBFEFF30880EFF3098020E9F00F03
:1022200040F804ED1EF0040F0CBF80F3088880F323
:10223000098800B50CF036FB5DF804EB4EF0040E97
:10224000704700000805002000050020040500205C
:1022500004ED00E020ED00E008ED00E0202A04DBC2
:10226000203A21FA02F00021704721FA02F3D0400F
:10227000C2F12002914008431946704740EA010329
:102280009B0703D009E008C9121F08C0042AFAD22C
:1022900003E011F8013B00F8013B521EF9D27047F0
:1022A000D2B201E000F8012B491EFBD27047002298
:1022B000F6E710B513460A4604461946FFF7F0FF45
:1022C000204610BD10B5044604E00B7800F8013B31
:1022D00003B1491C521EF8D2204610BD421C10F812
:1022E000011B0029FBD1801A704710B5002200E0C5
:1022F000521C835C8C5CA34201D1002BF8D1D8B274
:10230000E1B2401A10BD30B505460020034600E09A
:102310005B1C934205D2EC5CC85C201A01D1002CF6
:10232000F6D130BDF0B480EA0102D40F4200B2EB26
:10233000410F02D20246084611464A0042D0C30D60
:10234000DDB2C1F3C752AD1A202D35DAC1F3160143
:1023500041F4000204B15242C5F1200602FA06F12E
:102360002A411044B3EBD05F23D0C4B1012DA0EBC0
:10237000C35009DCF0BC4FF0004202EAC352DBB2AA
:1023800000F5000000F0CBBA400000F1807000EBD7
:10239000C350A0F1807040EAD170490009E04908BB
:1023A00041EAC071A0EBC35000F50000400800EB0B
:1023B000C350F0BC00F0AABA6142012202EB410115
:1023C000001BF6E7F0BC704781F00041AAE780F0FF
:1023D0000040A7E780EA010210B502F00043400088
:1023E00022D04A001FD0010E01EB1261C0F356004B
:1023F000C2F3560240F4000042F40002A0FB0220A7
:1024000000047F39140400D0401C50EA124001D46B
:102410004000491EC2B20C0604EBD010401C40081C
:10242000802A02D003E0002010BD20F00100002926
:1024300000DA0020184310BD30B480EA010202F037
:10244000004530F0004221F0004013D090B1C30DA0
:10245000D40DC2F31601C0F31600E41A41F40001D2
:1024600040F400027D34914201D3641C00E0490035
:10247000002C02DA30BC002070474FF4000000232B
:10248000914201D3891A034340084FEA4101F7D131
:1024900051B1914202D14FF0004105E002D24FF01C
:1024A000010101E06FF0010103EBC450284430BC8E
:1024B00000F02CBA2DE9FE4F804681EA0300C00FE0
:1024C0000C46009021F0004123F00045B8EB0200DB
:1024D000A94105D24046214690461C460B4602467D
:1024E00023F00040104347D0270DC7F30A00C3F381
:1024F0000A510290401A019040286BDAC3F313008E
:1025000040F4801B0098924620B10023D2EB030ACE
:1025100063EB0B0B01985946C0F14002504600F0A6
:10252000D4F906460D4650465946019A00F0DCF9AA
:1025300010EB08006141002487EA115284EAE77336
:102540001A4340D0009A62B3019A012A4FEA075217
:1025500015DC001B61EB02014FF0004202EA07525A
:10256000CDE90042001C41F5801132462B4600F0B7
:1025700013FA03B0BDE8F08F40462146F9E7001B8F
:1025800061EB0201001C41F5801300185B4120182B
:10259000A2F5001747EB030140EAD570B6196D416B
:1025A00011E06D084FEA360645EAC0754FEA07525A
:1025B000001B61EB0201001C41F5801149084FEA44
:1025C00030000019514132462B4603B0BDE8F04FB0
:1025D00000F0D3B90098012240000023D0EB0202A2
:1025E00063EBE073009821464FEAE074B8EB00001B
:1025F00061EB0401E9E783F000435BE781F0004110
:1026000058E72DE9FE4F81EA030404F0004421F06D
:10261000004100944FF0000B23F0004350EA010406
:102620005ED052EA03045BD0C3F30A54C1F30A55E7
:102630002C44A4F2F3340194A0FB0254C1F313011F
:1026400041F48011C3F3130343F4801301FB0244EC
:1026500000FB034E840A970A44EA815447EA8357F1
:10266000A4FB076802958D0A05FB07854FEA932CAA
:1026700004FB0C542705029D4FEA065847EA16371B
:10268000B5EB08056EEB070C870E920E47EA811733
:1026900042EA8312A7FB0201B6EB0B0164EB0004D4
:1026A0002B0D43EA0C335E1844EB1C50DA465146BE
:1026B000E7FB0201C5F313044FEA0B3343EA14535B
:1026C0004FEA0432019C43EA0603A4F10C0402948D
:1026D000009CCDE900B400F05FF903B0BDE8F08FD5
:1026E00000200146F9E72DE9F04D81EA030404F0EA
:1026F000004B21F0004514464FF0000A23F0004142
:1027000050EA050220D054EA01021DD0C5F30A5751
:102710000246C5F31303C1F31300C1F30A5640F494
:10272000801543F48013A7EB0608101BD64608F269
:10273000FD3873EB050002D308F1010801E092189F
:102740005B41B8F1000F03DA00200146BDE8F08DCF
:1027500000204FF48011064684460EE0171B73EBF1
:10276000050705D3121B63EB050306434CEA010C76
:1027700049084FEA300092185B4150EA0107EDD159
:1027800052EA030012D082EA040083EA05010843FA
:1027900005D0101BAB4106D20122002306E0002227
:1027A0004FF0004302E06FF0010253101AEB0600F5
:1027B0004CEB085110EB0A0041EB0B01BDE8F04D6A
:1027C00000F0DBB896230022114600F0A8B80EB541
:1027D00040F2334102910021CDE900110A460B4637
:1027E00000F0DAF803B000BD20F00040C10DC0F3E6
:1027F000160040F400007F2901DA00207047962976
:1028000003DCC1F19601C840704796398840704793
:10281000C1F30A5210B5C1F3130140F2FF3341F482
:1028200080119A4201DA002010BD40F233439A42EF
:10283000A2F2334203DC5242FFF710FD10BD90407C
:1028400010BD00F0004230F000400AD0C10D01F58B
:102850006071C0F3160042EA0151C20840071143FB
:1028600070470020014670472DE9F05F05460020C3
:1028700092469B4688460646814640241BE02846F1
:10288000414647462246FFF7E9FC53465A46C01ADE
:10289000914110D311461846224600F016F82D1A21
:1028A00067EB01084F4622460120002100F00DF899
:1028B00017EB00094E41201EA4F10104DFDC48465D
:1028C00031462A464346BDE8F09F202A04DB203AE1
:1028D00000FA02F1002070479140C2F1200320FA73
:1028E00003F3194390407047202A06DBCB17203AA8
:1028F00041FA02F043EAE07306E041FA02F3D04005
:10290000C2F1200291400843194670470029A8BF30
:102910007047401C490008BF20F00100704710B408
:10292000B0FA80FC00FA0CF050EA010404BF10BCBD
:10293000704749B1CCF1200421FA04F411FA0CF1EA
:1029400018BF012121430843A3EB0C01CB1D4FEA23
:1029500000614FEA102042BF002010BC704700EB1E
:10296000C35010440029A4BF10BC7047401C49004C
:1029700008BF20F0010010BC704710B5141E73F1A1
:10298000000408DA401C41F1000192185B411A432F
:1029900001D120F0010010BD2DE9F04D92469B467B
:1029A00011B1B1FA81F202E0B0FA80F22032904621
:1029B000FFF78BFF04460F4640EA0A0041EA0B018D
:1029C00053465A46084313D0114653EA010019D022
:1029D000C8F140025046FFF741FC05460E465046FE
:1029E00059464246FFF771FF084305D0012004E035
:1029F00020463946BDE8F08D0020054346EAE076E2
:102A00002C4337430A986305E40AA0EB0800002230
:102A1000FD0A44EA47540A3002D500200146E9E79E
:102A2000010510196941DDE9084500196941BDE852
:102A3000F04DA2E7064C074D06E0E06840F00103C8
:102A400094E8070098471034AC42F6D3FFF774FBC4
:102A5000C0200108E020010870B58C1810F8015B57
:102A600015F0070301D110F8013B2A1106D110F827
:102A7000012B03E010F8016B01F8016B5B1EF9D12B
:102A80002B0705D40023521E0DD401F8013BFAE7B1
:102A900010F8013BCB1A921C03E013F8015B01F81C
:102AA000015B521EF9D5A142D8D3002070BD10B5EC
:102AB0000CF011FD002010BD30B51649164B0A462A
:102AC0000D7C127D002465B18D7D6D1CEDB28D7580
:102AD000954201D300258D75E9B243F8210000200D
:102AE00011E0002404E000BF43F82400641CE4B2B9
:102AF0009442F9D301220A7430BD00BF53F820106C
:102B0000401C0C44C0B211469042F7D3B4FBF1F024
:102B100030BD000028030020082D00200C4910B50E
:102B20004A7E47F6FF7400236AB14A6E821A00D5C6
:102B30005242A24209D9CA7E4C7DA24205D8521CFB
:102B4000CA76486E10BD01224A76CB76486610BD23
:102B5000280300202DE9F047DFF8949000256C1E33
:102B600001220421484602F0C2F8012001F0D2F906
:102B70004FF47A784FF480761E4F02E06D1C454585
:102B800032D83146384602F0A5F80128F6D045453E
:102B90002AD20024B04625464E4600220421304663
:102BA00002F0A5F8012001F0B5F96400414638466D
:102BB00002F090F8012800D1641C01220421304663
:102BC00002F095F8012001F0A5F96D1CEDB2182D69
:102BD000E3D309484078411E032901D8E40803E003
:102BE000401F012800D8A4082046BDE8F087000057
:102BF00000100140000C0140082C0020104810B5C6
:102C000001681048416410490978C1720F49097878
:102C100001730F49096881640E4909684163002105
:102C2000417306F02FFC04F0D1FE05F0FBFC05F02B
:102C3000E5F809484078BDE8104006F077BB000091
:102C400044000020280300203F0000203E00002018
:102C5000480000204C000020082C002010B51A4C21
:102C60001A490422606C08601949E07A0870194911
:102C7000207B08701849A06C08601849606B0860D8
:102C8000124917A00EF066F80122114917A00EF0A4
:102C900061F801220F4918A00EF05CF804220E49D9
:102CA00018A00EF057F804220C4919A00EF052F8A3
:102CB00005F0A4FB207808B1012803D1BDE810403D
:102CC00005F0BABC10BD000028030020440000201D
:102CD0003F0000203E000020480000204C00002063
:102CE00061645F4D617876616C00000061645F49EA
:102CF0006E746576616C000061645F506F696E741C
:102D00000000000061645F5370616E7A0000000093
:102D100061645F5A65726F00FEE700001CB5052113
:102D20000320CDE900014FF480630022064907A08B
:102D30000CF03DF907490028C86003D0BDE81C40ED
:102D40000CF046BA1CBD0000D12D00084275747409
:102D50006F6E00004C02002030B503460020024692
:102D6000064C08E09D5C4540EDB2521C34F815500D
:102D700092B285EA10208A42F4D330BD1C160108B5
:102D80000F4910B57E200870452048700D48007826
:102D900030308870032020220A54401C1228FBDBAC
:102DA000094C4FF0FF3120680CF04FF80C22044919
:102DB000064802F05FFE2068BDE810400CF02AB81B
:102DC000B02400208C010020A4010020280700204E
:102DD0004FF0010B0025DFF8F893FE4EC821C9F82B
:102DE00018103078022801D0072817D1FA4902209C
:102DF0008D740B5C8A7C401C1A448A741228F8DBA0
:102E0000F64C4FF0FF3120680CF01FF81322F24906
:102E1000F34802F02FFE20680BF0FCFFEC4C1C3452
:102E2000207808B1401C2070607808B1401C6070A8
:102E3000A07808B1401CA070E07808B1401CE07098
:102E400020780F2800D3257060780F2800D3657094
:102E5000A078052800D3A570E078052800D3E57098
:102E6000E04F4FF40041384601F034FF00287CD099
:102E70002078002879D199F802000128FAD1307819
:102E800002283FD007283DD0D748C178FE2926D058
:102E9000D6490988002922D181780A0620D5D44A4A
:102EA0001278EAB9804688071AD406F023FCD14884
:102EB000D149012200880880D04998F803000870A1
:102EC000CFA00DF047FF0422D149D2A00DF042FF60
:102ED0000222C949D2A00DF03DFF09F04DFBA2E04E
:102EE00070200DF06BFC00280BD0D0480078002833
:102EF00007D1CF4800680BF08DFF0021F2200CF0C5
:102F0000F7FC90E006F0F6FBFFF73AFFC94807210F
:102F100001707E21417005218170C749097841B156
:102F2000C649097801F00F02C549097862F31F11FB
:102F300003E0C349097801F00F01C170C14991F85C
:102F40000080B8F1010F31D0B8F1030F2ED0142159
:102F50000171BD4980F805B00A788271521C0A706F
:102F6000C57101210278835C00E061E010F801C0C6
:102F7000491C6344835402788A42F3DCD1B2B8F12D
:102F8000000F425CC2F1FF0242542CD00121C12249
:102F900008460CF041FFA749AC480DF04BFFAC4B85
:102FA0000146AC4A186001209A4607E0A221CFE70B
:102FB0000B5C02EB000C401C0CF8013C0B788342CC
:102FC000F6DADFF894824FF0FF31D8F800000BF00A
:102FD0003CFFDAF800009F490278A04802F04AFD61
:102FE000D8F800001DE0804601219D4B007806E0E6
:102FF00018F8012003EB010C491C0CF8012C884245
:10300000F6DADFF860A24FF0FF31DAF800000BF0DB
:103010001CFF98F800209249934802F02BFDDAF843
:1030200000000BF0F7FE84F800B06570A570E57045
:103030004FF48041384601F04DFE00287ED0607884
:1030400000287BD199F80200012877D13078022836
:103050000ED007280CD065480088002807D16B20C7
:103060000DF0ACFB002802D1F4200CF0CBFC94E076
:1030700006F040FBFFF784FE6E48072101707E21B9
:103080004170052181706C49097841B16B4909781B
:1030900001F00F026A49097862F31F1103E06849E1
:1030A000097801F00F01C170664991F80080B8F10C
:1030B000010F31D0B8F1030F2ED014210171624AF3
:1030C0000221417111788171491C1170C571012172
:1030D000027810F801C0491C835C63448354027871
:1030E0008A42F5DC824601460078B8F1000F0A5C9E
:1030F000C2F1FF020AF800202FD00121C1220846A8
:103100000CF08AFE4B4951480DF094FE504B01469D
:10311000504A1860012007E0A221CFE70B5C02EBC8
:10312000000C401C0CF8013C0B788342F6DADFF807
:1031300028814FF0FF31D8F8000000E032E00BF0BA
:1031400084FE4348434900680278444802F092FCF8
:10315000D8F800000BF05EFE0DE00120404B0A782D
:1031600007E000BF11F800C003EB0008401C08F89E
:1031700001CC8242F6DADFF8EC804FF0FF31D8F86C
:1031800000000BF062FE9AF800203549364802F044
:1031900071FCD8F800000BF03DFE257084F801B0FA
:1031A000A570E5704FF40051B846384601F092FD25
:1031B00068B1A07858B9307802287DD007287BD034
:1031C0002A4800780E2876D006F094FA50E067E09E
:1031D0004C0200203B000020B0240020A40100206D
:1031E00028070020000C0140EC020020C40200204F
:1031F000BC0200209202002042000020BB020020FE
:10320000636F6D706C6574656F7264657200000049
:10321000D8020020626567696E74696D6500000000
:10322000626567696E77656967687400C00200202F
:10323000D4020020EC0100203400002035000020E2
:103240008C01002037000020BD020020842B0020CC
:10325000D8010020702300209C010020E8070020F6
:1032600070240020A0010020280800203800002041
:103270004FF47A700BF060FF4FF40051404601F0BC
:1032800029FD10B1307801284CD05D480178012922
:1032900076D080F800B02570657084F802B0E570D3
:1032A0004FF48051404601F015FD0028E07868D0C9
:1032B000B8B3A1E000E014E052480178012908D039
:1032C000491E0170FFF75CFD4F480078032803D0CA
:1032D00004E04E490978F4E70CF012FC06F00AFA13
:1032E000D9E7E07828B1D9E905121144C9F81410DA
:1032F00001E0C9F814B04FF48051404601F0EAFCF7
:103300000028C8D0D9F8140040F2DC514F4688425A
:10331000C1D906F0EFF97D610CF080FF0CF080FF61
:10332000B9E73CE0DFF8E8A04FF0FF31DAF8000041
:103330000BF08BFD3749384F00200A5C3A54401C93
:103340002828FADBDAF800000BF064FD02E0C82060
:103350000BF0F2FE4FF40051404601F0BBFC002898
:10336000F5D1411EDAF800000BF06FFD2822202174
:1033700029480BF0F3FB294A002150780B3805E06F
:103380000BE036E053181B797B54491C8842F9DA6C
:10339000DAF800000BF03EFD7DE705707BE7307842
:1033A000022812D0072810D0062805D11C48017821
:1033B00041B1057006F09EF925706570A57084F81E
:1033C00003B019E080F800B0F4E70E480F4A017826
:1033D0001278914202D180F800B001E0491C0170DE
:1033E000FFF7CEFC084800780328E3D10CF088FBF7
:1033F000E0E708B9C9F81450C8200BF09DFEEAE4D4
:10340000290200208C010020370000203A00002013
:103410002C020020F702002004290020B4280020FC
:1034200048020020DFF8E493DFF8E4A3DFF8E4B318
:1034300000254FF00108F84C207808B1401C20709E
:10344000607808B1401C6070A07808B1401CA07082
:10345000E07808B1401CE070207908B1401C207170
:103460002078052800D325706078052800D3657082
:10347000A078052800D3A570E078052800D3E57072
:103480002079052800D32571E44E3078052875D2BF
:10349000E34F4FF40041384601F01CFC08B120789E
:1034A00008B34FF48041384601F014FC38B130784D
:1034B000042804D0062802D06078002870D04FF489
:1034C0000051384601F006FC10B1A078002868D001
:1034D0004FF48041384601F0FDFB002802D03078DF
:1034E000042870D073E206F005F9CE480078B0B138
:1034F000012827D0022831D0032842D0042851D0F7
:1035000005285BD0062867D0072872D0082871D01C
:10351000092870D00A286FD00B286ED0F2E099F8F5
:1035200000004E46012801D9401E00E00A203070FC
:103530000122B649BCA00DF00DFC307830308AF87D
:103540000600DFE0B9480178012901D9491E00E0F1
:103550000E2101700122B549B5A0D1E0B54801782E
:1035600009B1491E03E03178042908D00D2101700A
:103570000CF0C2FB0122AF49AFA0C1E065E202211D
:10358000F5E73078042833D0062831D0012801D956
:10359000401E00E0032030700122A049A7A0AFE048
:1035A000B4E0F3E1A6490878012801D9401E00E003
:1035B0000A2008700122A249A2A0A1E0A24908782D
:1035C00010B1401E01E000E2032008700CF0F8FA90
:1035D00001229D499DA093E08F481C38017869B174
:1035E00001290FD0022913D0032916D004291BD09A
:1035F00088E020E04FE059E064E077E0816831B393
:10360000491E03E081680A297CD90A39816079E082
:103610008168642976D96439F8E78168B1F57A7FE1
:1036200070D9A1F57A71F1E7816842F21072914286
:1036300068D9891AEAE778481C38407840B10128EF
:103640000BD002280FD0032814D004281AD059E038
:103650007F49086878B3401E1BE07D4801680A294D
:1036600050D90A3904E07A48016864294AD9643992
:10367000016047E076480168B1F57A7F42D9A1F54B
:103680007A71F5E7724942F210720868904239D9AE
:10369000801A086036E06F48017809B1491E00E0E1
:1036A0000821017001226B496BA029E06C49087860
:1036B00010B1401E01E025E0032008700122684996
:1036C00068A01DE09BF80010012909D0022901D053
:1036D000052907D08BF8008001224E4964A00FE035
:1036E000052100E002218BF80010F5E76349087816
:1036F00008B1401E00E00320087001225F4960A06D
:103700000DF028FB84F8008065703CE105F0F2FFC5
:1037100044480078B0B1012822D002282DD00328D7
:1037200043D004284AD005285BD0062867D0072854
:1037300066D0082865D0092864D00A2863D00B28F1
:1037400062D01DE199F800100A2903D2491C89F8BA
:10375000001001E089F8008001222C4932A00DE11F
:10376000324801780E2902D2491C017001E080F82C
:10377000008001222D492EA000E12E4908780D2855
:1037800004D23278042A01D0062A0BD1022802D2B0
:103790003278042A06D00D700CF0AEFA01222549C9
:1037A00025A0EBE0401C0870F6E73078032801D232
:1037B000401C30700122194920A0DFE0204E3078F3
:1037C0000A2802D2401C307001E086F800800122F5
:1037D0001B491CA00DF0BEFA307830308AF8060084
:1037E000CEE019480178032902D2491C017000E09B
:1037F00005700CF0E5F90122134914A0BEE041E088
:103800005FE082E08EE09AE0ACE00000350000204E
:10381000400200203F000020680200203B00002002
:10382000000C01402802002043480000380000201E
:103830005451000036000020574C0000504D00004D
:103840003A00002043430000370000204150490067
:103850006C0300203D00002061645F4653000000BF
:103860003E00002061645F506F696E7400000000CC
:1038700061645F496E746576616C000039000020F8
:10388000424C45008248017841B1012909D0022902
:103890000BD003290CD004290ED071E08168491C9B
:1038A00001E081680A3181606AE081686431FAE789
:1038B000816801F57A71F6E7826842F2107111446D
:1038C000F1E77348407840B101280AD002280DD0B2
:1038D00003280FD0042812D052E06E480168491C1A
:1038E00002E06C4801680A31016049E069480168FA
:1038F0006431F9E76748016801F57A71F4E76548D2
:1039000042F2107102681144EEE763480178082919
:1039100002D2491C017000E005705F490122AFF23C
:10392000C8002BE05D490878032802D2401C0870CB
:1039300000E00D7059490122AFF2D8001EE09BF85B
:103940000010012908D0022908D08BF800805449C2
:103950000122AFF2E40011E0022100E005218BF822
:103960000010F4E74F490878032802D2401C087081
:1039700000E00D704B490122AFF2FC000DF0EAF9B6
:10398000257084F80180A570E5706AE046480078EB
:10399000062802D0072809D010E03D4908780428FD
:1039A00002D0401C087007E00D7005E038494878E7
:1039B000042808D0401C487005F09CFE25706570F6
:1039C00084F80280E0E74D70F6E7E07868B14FF4E4
:1039D0008051384601F07EF9B8B33078042841D0E0
:1039E00006283FD0E07818B33CE0304800780E2835
:1039F0002D48017802D205290BD001E00A2908D010
:103A0000491C01702848007806283FD0072802D0BA
:103A100009E005701EE01E4845708068D0B100BF07
:103A20000CF04EF916E0082814D1FFF717F911E051
:103A30001E4800780E2819D21B490878052805D0A1
:103A40000B2806D0401C087016E00BE00B20087015
:103A500000E00D7005F04EFE25706570A57084F8CD
:103A600003802571C8200BF067FBE4E40E48017861
:103A70000B29CED0491C01700B480078062805D0D0
:103A80000728D0D1024845708068C9E70048C0E7E0
:103A90004C0200206C0300203D0000203E0000206E
:103AA0003F000020390000202802002038000020BC
:103AB0001CB505210420CDE900014FF4407300221C
:103AC000064907A00BF073FA08490028486303D0A1
:103AD000BDE81C400BF07CBB1CBD0000F13A0008A7
:103AE000436865636B5765696768740070020020FE
:103AF000DFF82492894EDFF828B2DFF828A28A4C3A
:103B00000025B17811F0780F30D0BAF80000574690
:103B100060B3B9F80020C1F3C300521C92B2C0EBED
:103B20000010A9F80020B2EB800F21D9DFF8FC814A
:103B30004FF0FF31D8F800000BF087F97C49608C1A
:103B4000022208807BA00DF005F97D490120087054
:103B5000D8F800000BF05EF97A4800680BF05AF9CB
:103B6000B07820F07800B0703D8001E0A9F80050F6
:103B7000607A002873D04FF0FF31206B0BF065F9AD
:103B8000E078022809D9B4F91220E16A891AB4F957
:103B90001020891A801EE162E070E178E06A90FBF3
:103BA000F1F06084206B0BF035F9E0790F2824D315
:103BB00065495D483C300A78C2704A7802718A785B
:103BC0004271C9788171618CA0F801106279017825
:103BD00062F346115D4A127862F3041121F00F017D
:103BE0000170014607225A480CF0B0FD608BA0839B
:103BF000208B6083608C2083E57196F80080607B69
:103C0000C8F38102824201D91E2800D36573617B0B
:103C1000277A01EB410358460BF803700344677A97
:103C2000DFF830C15F70B4F92270BCF900C067459D
:103C300006DD18F00C0F03D0474F3F78012F0FD04F
:103C40009D70E562E5704FF4004323825B1E638242
:103C5000491C6173A5722573E572002116E052E0DC
:103C600001279F70EDE700BF01EB410394F80AC004
:103C7000C75C03446744A7725F7894F80CC0491C82
:103C8000674427739B78E77A3B44E3728A42EBDC14
:103C9000217B09B964212173A17A64235943237BD1
:103CA000B1FBF3F1C9B2E173642900D9E573E17B9B
:103CB000A37B994206D8E17AB1EB520F1ED9B178B5
:103CC00049071BD55FF0000101EB4102491C8554F7
:103CD00002441E2955709570F6DB2049BAF80000A1
:103CE0000978084307D11E4800680BF093F80021BB
:103CF000F1200BF0FDFD1B49012008702572657253
:103D0000A5722573E572E079401CE0714FF47A707A
:103D10000BF012FAF5E60000CE020020EC020020C3
:103D20005A280020C4020020700200202C0200202B
:103D300042000020626567696E7765696768740094
:103D4000B8020020D0020020D8020020B9020020D2
:103D50003C0C0020CC020020BC020020C00200204D
:103D6000D40200206802002001B50848009A816B47
:103D70008A4201D9511A00E0891A0091182901D20A
:103D8000012100E000218170C17008BD28030020DE
:103D9000064A116A936A01F10A000A398B4201D37B
:103DA000834201D900209071704700002803002051
:103DB0000C4810B505218173C26B846A1146531FEC
:103DC0000022491D9C420BD98C4209D20179052958
:103DD00003D302710121817110BD491C017110BD15
:103DE000027110BD2803002010B50B490024CA6BD6
:103DF0008B6A02F13200323A93420BD9834209D2E4
:103E00000879142803D30C710120887110BD401C5F
:103E1000087110BD0C7110BD2803002010B5074CAF
:103E2000E07C08B900F00CF8A06AFFF79DFF00F0F5
:103E300049F9BDE8104000F075B8000028030020E3
:103E400010B5104C0020A071FEF784FE2063FEF731
:103E500033FE206300F04AF9206305F0EBFAA0621C
:103E6000FFF7C2FFA06AE063A0790028ECD004F05D
:103E7000D9FB206CA0622062E062E063A0630120B5
:103E8000E07410BD28030020014800F0DBBB0000F7
:103E9000440A0020014800F0D5BB0000000A0020C1
:103EA000014800F0CFBB000034090020014800F0B9
:103EB000C9BB0000F0080020014800F0C3BB0000AF
:103EC00078090020014800F0BDBB0000BC090020BB
:103ED000014800F0B7BB000068080020014800F06E
:103EE000B1BB0000AC08002030B590F84050012470
:103EF000AC40C56B6C60046863604368102B03685A
:103F000003D099600068C26030BD9A600068C160EB
:103F100030BD704701B5009801E0401E00900028B8
:103F2000FBD108BD30B505F065FA174C606AE06456
:103F3000A26B216A914201D3891A00E0511AE37AF7
:103F4000626C0025B2FBF3F202EB82025A2303EB10
:103F500042028A4201D3E57101E00121E1710A21A7
:103F600003F0F2FDE17A4843606200D1257201EB73
:103F70004102824200D3657201EB8101B0EB810FF7
:103F800000D8657030BD000028030020054D42F2C6
:103F90001074287808B905F0ADFF20460BF0CCF876
:103FA000F7E70000B90200201CB53D4C3D4E3E4DE8
:103FB00008F096F93078032804D3062802D00428A4
:103FC0002ED068E07E2020704520607037490020A8
:103FD00023180A5C401C9A700828F9DB3449072032
:103FE000C0F1070223188A5C9A72401EF8D500209F
:103FF000A0740220A17C225C401C1144A1741228F0
:10400000F8DB2C4F4FF0FF3138680AF01EFF132207
:104010002349294801F02EFD38680AF0FBFE3AE0FA
:1040200001A8009021480A2306224CF60261283894
:104030000AF001FB58BB0198800704D528780128B5
:1040400001D105F07BFC0198000504D528780128F2
:1040500001D105F023FF0198800505D528780128B6
:1040600002D1002006F018F90198400507D52878FC
:10407000012804D11148B0F9000005F0D5FE0198DF
:10408000400404D52878012801D106F009F80C482D
:10409000006806F05DF84FF4C8700BF04DF887E744
:1040A000B02400203B000020880100203827002099
:1040B00040020020A401002028070020C6020020A2
:1040C0009802002010B5084CA07920B1FFF760FEDF
:1040D00004F0C2FA01E0FFF76BFEA06A2062FFF76E
:1040E00043FEA06AE06310BD280300202DE9F14FD4
:1040F000AA4CAB4F86B007F11805E67B05F1180A0C
:104100000698FEF75FFB002E7ED0616DFEF70AF980
:1041100006466065607C401CC1B26174A07C81422F
:1041200073D33A46B968D160884611464F688F60AC
:10413000096851608946FEF745FB01463046FEF7A7
:104140007BF906469648214606600020487448657B
:10415000A868E86001906868A860029028686860B4
:10416000039090494046FEF735F983468E4938461C
:10417000FEF730F980468D494846FEF72BF9074691
:104180008B493046FEF726F93946FEF7CBF8414613
:10419000FEF7C8F85946FEF7C5F82860814607467D
:1041A000DAF80800CAF80C000090DAF80400CAF83F
:1041B00008008346DAF800005546CAF80400824633
:1041C00078490198FEF706F9019077490298FEF7C1
:1041D00001F9029075490398FEF7FCF8804674498E
:1041E0003846FEF7F7F84146FEF79CF80299FEF7CD
:1041F00099F80199FEF796F82860694D8046483590
:104200000746A868E86001E08CE081E004906868F7
:10421000A860039028686860029062490098FEF7E1
:10422000D9F8009060495846FEF7D4F883465F49B4
:104230005046FEF7CFF882465D493846FEF7CAF889
:104240005146FEF76FF85946FEF76CF80099FEF7F5
:1042500069F8286018350746A868E86083466868EA
:10426000A86001902868686000904E490498FEF7A5
:10427000B1F804904C490398FEF7ACF803904B4911
:104280000298FEF7A7F8824649493846FEF7A2F899
:104290005146FEF747F80399FEF744F80499FEF7F4
:1042A00041F8286018358246A868E8606868A86008
:1042B000286868603B495846FEF78CF802903A49F6
:1042C0000198FEF787F8019038490098FEF782F8C8
:1042D000834637495046FEF77DF85946FEF722F8E7
:1042E0000199FEF71FF80299FEF71CF82860A5F166
:1042F00088004078E8B3012848D0022846D0032837
:1043000044D0042842D0052842D0062843D027654F
:104310004FF07C51206DFEF705F807B0BDE8F04F77
:10432000FEF762BADFF87890002109F1600909F11F
:10433000180202F1180302F1300B02F1480E564642
:10434000A2F1300C47F8210045F8210046F8210081
:104350004CF8210049F8210042F8210043F82100DF
:10436000DFF83C804BF821004EF8210008F1D80816
:1043700000E00BE048F82100491CC9B20429E1D350
:104380000120E073069807B0BDE8F08F2665BFE70F
:10439000C4F85090BCE7C4F85080B9E72803002067
:1043A000182C0020CDCCCC3E9A99993ECDCC4C3ED9
:1043B000CDCCCC3D7047000006490020C8610648BE
:1043C000016941F004010161016941F040010161AD
:1043D00070470000880A002000200240064A0021A1
:1043E000D16106490A6942F002020A61486108691E
:1043F00040F0400008617047880A00200020024019
:10440000044B0022DA61044A136943F0010313618B
:1044100001807047880A00200020024014480022D2
:10442000C168CB06134904D5CA6942F00202CA61C9
:104430001022C3685B0705D5CB6943F00103CB614C
:1044400042F00402C369DB0707D0CB6943F00403E1
:10445000CB61C16921F00101C161A2F5807101390F
:1044600001D0C2607047C16921F00101C16170478C
:1044700000200240880A002070B5054600F03CFC90
:104480000646114C09E0681C07D025B100F034FC49
:10449000801BA84201D9032070BDE068C007F2D19B
:1044A000E068800601D52020E060E068C00605D401
:1044B000E069C00702D1E068400703D5FFF7AEFF0F
:1044C000012070BD002070BD0020024010B590F8A2
:1044D00021100022022905D00421816380F82020C8
:1044E000012010BD01680B6823F00E030B6001680A
:1044F0000B6823F001030B6090F84030C46B01217E
:1045000001FA03F3636080F8211080F82020104640
:1045100010BD00002DE9F05F90F821100024022961
:1045200003D004218163012485E001680A6822F038
:104530000E020A6001680A6822F001020A603F4E1A
:104540003E4FB215DFF8F4C0DFF8F090DFF8ECA0D2
:10455000DFF8E8B0DFF8E4E00168783F1301150206
:10456000ACF1640CA9F15009AAF13C0AABF1280B9B
:10457000AEF1140E4FF48018B14227D9B9420ED0D3
:10458000614512D049451DD0514518D0594518D024
:10459000714501D1424615E0294EB14201D10122B7
:1045A00010E0274E1436B14201D110220AE0244E09
:1045B0002836B14206D0224A3C32914201D11A46F5
:1045C00000E02A461E49091F0A602BE0B94213D0B9
:1045D000614517D0494522D051451DD059451DD0C0
:1045E000714501D142461AE0B14202D14FF08072CA
:1045F00015E0134EB14201D1012210E0104E1436E5
:10460000B14201D110220AE00D4E2836B14206D047
:104610000B4A3C32914201D11A4600E02A46074932
:1046200080394A60012180F82110002180F8201093
:10463000416B01B188472046BDE8F09F80000240F1
:10464000080402402DE9F05FC16B0A6801680B683D
:10465000046C4FF0040808FA04F8844D844E854F2A
:10466000DFF814C2DFF81492DFF814A2DFF814B2F6
:10467000DFF814E218EA020F65D05FEA437862D5EA
:104680000A68920603D40A6822F004020A60DFF87E
:10469000F0814FF48062016808F1140813011402DC
:1046A000414524D9A9420DD0B1420FD0B9421AD008
:1046B000614515D0494515D0514501D1120312E08D
:1046C000594501D104220EE0714501D140220AE092
:1046D0006D4D1435A94206D06B4A2832914201D162
:1046E0001A4600E022466749091F0A6029E0A942EC
:1046F00013D0B14215D0B94220D061451BD04945F5
:104700001BD0514502D14FF4800217E0414502D140
:104710004FF0806212E0594501D104220EE071454C
:1047200001D140220AE0584D1435A94206D0564A1C
:104730002832914201D11A4600E022464B490839FD
:104740004A60C16A71E04FF0020808FA04F818EAFA
:10475000020F70D05FEA83786DD50A68920606D49E
:104760000A6822F00A020A60012180F82110DFF8AD
:1047700010814FF40072016808F11408130114024B
:10478000414524D9A9420DD0B1420FD0B9421AD027
:10479000614515D0494515D0514501D1120312E0AC
:1047A000594501D102220EE0714501D120220AE0D3
:1047B000354D1435A94206D0334A2832914201D1F1
:1047C0001A4600E022462F49091F0A6029E0A94243
:1047D00013D0B14215D0B94220D061451BD0494514
:1047E0001BD0514502D14FF4001217E0414502D1D0
:1047F0004FF0007212E0594501D102220EE07145DE
:1048000001D120220AE0204D1435A94206D01E4ACB
:104810002832914201D11A4600E022461349083954
:104820004A60002180F82010816A00291CD0BDE870
:10483000F05F0847FFE70825A540154214D01A0786
:1048400012D50A6822F00E020A6090F84020C36B6D
:10485000012101FA02F25A60816380F821100021DF
:1048600080F82010016BE0E7BDE8F09F08000240EF
:104870001C00024030000240440002405800024048
:104880006C000240080402401C04024030B560B1D4
:104890001A4B026814219A4209D2194B1344B3FBF4
:1048A000F1F18900016417490AE0012030BD134B82
:1048B0005B421344B3FBF1F1890001640F490839ED
:1048C000C163022180F82110136843F6F0718B4315
:1048D000F0E901142143D0E902452C432143046946
:1048E0002143446921438469214319431160002114
:1048F0004163012242770177084630BD0804024037
:10490000F8FFFDBF0000024070B5044690F820009B
:10491000002501280CD0012084F8200094F82160A3
:104920000020012E06D084F820000225284670BD04
:10493000022070BD022684F82160A063206806680A
:1049400026F0010606602046FFF7CEFAE06A00284E
:104950002068016802D041F00E0106E021F0040158
:1049600001602068016841F00A0101602068016867
:1049700041F001010160D9E72DE9F04705462648DD
:104980000F460126017E01290FD0012181460176C3
:104990002868DFF888804CF25034022808D0A246FC
:1049A0002046FFF769FDA8B131E00220BDE8F0879D
:1049B0002046FFF761FD08BB0120FFF7FDFC204604
:1049C000FFF75AFDD8F81010064621F00401C8F888
:1049D00010101CE04FF0FF303860AC6811E020464A
:1049E000FFF7FCFC5046FFF747FDD8F81010060013
:1049F00021F00201C8F8101001D03C6007E004F576
:104A00000064D5E9020100EBC120A042E7D80021F3
:104A100089F818103046C9E7880A002000200240B3
:104A20000348016941F080010161002070470000E6
:104A3000002002402DE9F05F07461C48884600240C
:104A4000017E15461E46012909D0012181460176C5
:104A50004CF2503A5046FFF70FFD18B122E0022009
:104A6000BDE8F09F012F02D0022F00D00427D346CB
:104A7000DFF83CA0220128463146FDF7EFFB81B26A
:104A800008EB4400FFF7BCFC5846FFF7F5FCDAF8EA
:104A9000102022F00102CAF8102018B9641CE4B2F8
:104AA000BC42E7D3002289F81820D9E7880A002001
:104AB00000200240064900200A69120607D5054A6F
:104AC0004A60054A4A600969090600D50120704715
:104AD0000020024023016745AB89EFCD2DE9F84F57
:104AE000DFF8C891002409F1040A0AF1040B2346F7
:104AF0000F270BF1040ED1E00125A54006EA0502BF
:104B0000AA4276D1DFF8A8C14E68A6EB0C0866452C
:104B10002BD00DDC032E34D005DC36B3012E19D09A
:104B2000022E2FD11BE0112E16D0122E2AD119E001
:104B3000B8F5881F19D006DCB8F5803F15D0B8F558
:104B4000801F1FD111E0B8F5001F0ED0B8F5041F6B
:104B500018D10AE0CB6815E0CB681B1D12E0CB68CA
:104B600008330FE0CB680C330CE08B682BB1012BC2
:104B70004FF0080303D0456104E0042302E005611F
:104B800000E00023FF2A01D8064601E000F10406F8
:104B90004FEA840501D9A5F12005D6F8008007FA6F
:104BA00005FC28EA0C0803FA05F548EA0508C6F8EA
:104BB00000804D68ED0070D53E4DAE6946F00106AF
:104BC000AE61AD6924F0030605F0010500953A4D8C
:104BD00006EB050CDCF80850A607360F07FA06F8B6
:104BE00025EA0805DFF8D480404503D14FF00008DE
:104BF00025E052E0DFF8C880404502D14FF00108BF
:104C00001DE0DFF8C080404502D14FF0020816E0F9
:104C1000DFF8B480404502D14FF003080FE0DFF821
:104C2000AC80404502D14FF0040808E0DFF8A080D6
:104C3000404502D14FF0050801E04FF0060808FAA0
:104C400006F848EA0508CCF808804D68D9F80060F5
:104C5000ED034D4601D5164300E096432E604D68A6
:104C6000DAF80060AD03554601D5164300E09643DF
:104C70002E604D68DBF80060ED025D4601D51643FD
:104C800000E096432E604D68DEF80060AD02754688
:104C900001D5164300E096432E60641C0A68164650
:104CA000E2407FF429AFBDE8F88F00000004014026
:104CB00000001110001002400000014000080140F7
:104CC000000C014000100140001401400018014098
:104CD000001C01408068084000D001207047C26875
:104CE00021EA02030A4043EA0241016170470AB126
:104CF000016170470904FBE70148806870470000C4
:104D000008000020074810B5016841F0100101605B
:104D1000032000F075F8002000F006F800F024F8F9
:104D2000002010BD0020024070B50D4D04464FF428
:104D30007A712878B1FBF0F00A490968B1FBF0F00C
:104D400000F0ECFA48B9102C07D200222146501E80
:104D500000F036F800206C6070BD012070BD0000CE
:104D600008000020040000200C4808B5816941F0CB
:104D700001018161816901F001010091C16941F086
:104D80008051C161C06900F08050009004484168C2
:104D900021F0E06141F00071416008BD0010024067
:104DA00000000140002809DB00F01F0201219140B2
:104DB0004009800000F1E020C0F8001170470000B9
:104DC000F0B40E4B1B680C46C3F30223C3F1070576
:104DD000042D00D90425191D072901D2002300E064
:104DE000DB1E012606FA05F1491E214099409E402E
:104DF000761E16403143F0BC03F076BC0CED00E0AB
:104E0000064900F0070208684FF6FF03184040EA21
:104E10000220034A10430860704700000CED00E0D8
:104E20000000FA052DE9F0470F46050061D0434E1A
:104E3000306800F00700B84209D2306820F007005F
:104E400038433060306800F00700B84251D128681C
:104E50003B4C810712D5400703D5606840F4E06001
:104E600060602878000703D5606840F46050606097
:104E70006068A96820F0F000084360602878C007E7
:104E800028D06868012810D02168022810D089072E
:104E900000292EDA616821F0030101436160FFF708
:104EA0002BFF804641F288390DE021688903EFE746
:104EB0008901EDE7FFF720FFA0EB0801494502D982
:104EC0000320BDE8F0876068696800F00C00B0EB73
:104ED000810FEFD1306800F00700B8420BD930687D
:104EE00020F0070038433060306800F00700B84217
:104EF00001D00120E5E72878400705D56068E9681A
:104F000020F4E060084360602878000706D56068F8
:104F1000296920F4605040EAC100606000F038F870
:104F20006168084AC1F30311515CC8400649086032
:104F300006480068FFF7F8FE0020C2E700200240A4
:104F400000100240000F0108040000200C000020A7
:104F50000448054900684968044AC1F30221515CCC
:104F6000C84070470400002000100240100F0108E4
:104F70000448054900684968044AC1F3C221515CEC
:104F8000C84070470400002000100240100F0108C4
:104F900012A185B00FC98DE80F0014A0144A006853
:104FA00004905168134801F00C03042B10D0082B17
:104FB0000ED1C1F38343C9031DF803000AD551681C
:104FC00004AAC1F34041515C0A4A5043B0FBF1F0DE
:104FD00005B0704708494843FAE70000020304059A
:104FE000060708090A0B0C0D0E0F10100102000035
:104FF0000010024000127A0000093D002DE9F84F30
:10500000040070D02078C04DC00749D06868C0F354
:105010008100012807D06868C0F38100022809D107
:105020006868C00306D52868800339D56068002801
:10503000E7D035E06068B0F5803F0BD010B1B0F537
:10504000A02F11D0286820F480302860286820F430
:10505000802002E0286840F480302860606890B1C9
:10506000FFF74AFE06460AE0286840F480202860E0
:10507000F0E700BFFFF740FE801B642873D8286864
:105080008003F7D50CE0FFF737FE064605E000BFCA
:10509000FFF732FE801B6428F0D828688003F7D41D
:1050A00020789A4E80074FF001094FF0000839D55B
:1050B000686810F00C0F07D06868C0F38100022800
:1050C00009D16868C00306D42868800714D5206910
:1050D000012808D110E02069B0B1C6F80090FFF7B0
:1050E0000BFE074605E00AE1FFF706FEC01B02289B
:1050F000C4D828688007F7D52868616920F0F800CF
:1051000040EAC10028600DE0C6F80080FFF7F4FD1A
:10511000074604E0FFF7F0FDC01B022823D82868EB
:105120008007F7D4207800072CD57948A169D9B138
:10513000C0F80090FFF7E0FD074604E0FFF7DCFD54
:10514000C01B02280FD8686A8007F7D571484FF452
:10515000FA510068B0FBF1F0009000BF0098411ECA
:105160000091FAD20EE080E0C0F80080FFF7C4FDA5
:10517000074604E0FFF7C0FDC01B022875D8686A27
:105180008007F7D42078400760D5E8690027C00081
:1051900008D4E86940F08050E861E869012700F030
:1051A000805000905C480168C90513D401688346AB
:1051B00041F480710160FFF79FFD824606E000BF69
:1051C000FFF79AFDA0EB0A0064284ED8DBF8000038
:1051D000C005F5D5E06801280AD008B1052813D02C
:1051E000286A20F001002862286A20F0040002E00A
:1051F000286A40F001002862E06841F2883B98B1DB
:10520000FFF77AFD82460BE0286A40F0040028622E
:10521000EEE700BFFFF770FDA0EB0A0159455AD831
:10522000286A8007F6D50CE0FFF766FD824605E0A8
:10523000FFF762FDA0EB0A0159454CD8286A8007A8
:10524000F6D41FB1E86920F08050E861E06988B3C6
:105250006968C1F38101022944D00228C6F8608040
:1052600004D0FFF749FD044638E034E0FFF744FD81
:10527000074604E0FFF740FDC01B02282BD8286832
:105280008001F7D4206AB0F5803F05D16868A16835
:1052900020F4003008436860D4E9080108436968D5
:1052A00021F4741108436860C6F86090FFF724FD8C
:1052B000044606E025E000BFFFF71EFD001B0228A4
:1052C00009D828688001F7D51BE000BFFFF714FD5F
:1052D000001B022802D90320BDE8F88F286880014E
:1052E000F4D40EE00128F7D06868226A00F4803117
:1052F000914204D1616A00F47010884201D001200B
:10530000EAE70020E8E70000001002400000424207
:1053100080044242040000200070004010B5401E8E
:10532000B0F1807F01D3012010BD4FF0E024606117
:105330000F21601703F0D8F90020A0610720206139
:10534000002010BD10B504460068416994F839206A
:10535000C1F3C011212A0BD151B1416921F0800163
:105360004161206B08B1FFF7B1F8204602F054FE0E
:105370002068416994F83A20C1F38011222A0BD1A8
:1053800051B1416921F040014161606B08B1FFF703
:105390009DF8204602F032FE002010BD704700004C
:1053A00070B5026804461068D168536910F00F0F99
:1053B00052D003F0010501F490762E435FD0C2076E
:1053C00005D0CA0503D5E26B42F00102E263420751
:1053D00005D5DA0703D0E26B42F00202E2638207EE
:1053E00005D5DA0703D0E26B42F00402E26302075C
:1053F00007D501F020022A4303D0E26B42F00802F5
:10540000E263E26B002A33D0800604D5880602D519
:10541000204602F00AFE20684069E16BC0F380106C
:10542000090700D428B3204602F0E8FD206841694E
:1054300049061AD5416921F040014161606BA0B174
:105440002D494163606BFFF765F8002810D0606B51
:10545000416BBDE870400847830610D58B060ED51A
:105460002046BDE8704002F0E0BD2046FFF796FF01
:1054700070BD2046FFF792FF0020E06370BD030679
:105480002BD50B0629D594F839002128F6D1A06830
:10549000B0F5805F01D12069B0B1206A411C216262
:1054A000216800784860E08C401E0004000CE08415
:1054B000E4D12068C16821F08001C1602068C16822
:1054C00041F04001C16070BD206A0088C0F308004F
:1054D0005060206A801C2062E5E74006F3D548064C
:1054E000F1D5D168204621F04001D160202184F817
:1054F000391000F0FFFA70BD257F000870B5040078
:1055000004D094F83900002510B106E0012070BDE8
:1055100084F83850204600F023F8242084F839001D
:105520002068C16821F40051C160204602F0C4FD2A
:105530002068016921F4904101612068416921F0EE
:105540002A0141612068C16841F40051C160E563EE
:10555000202084F8390084F83A00002070BD000053
:105560002DE9F04F85B00025009501950295039532
:105570000446DFF878830368DD4802210322DFF860
:1055800074C3102780264FF480694FF4006B4345A5
:1055900057D1C36943F40023C361C36903F40023F3
:1055A0000493836943F0100383618069CDE900911E
:1055B00000F01000CDE903206946E1466046FFF7A0
:1055C0008DFACDE900B5A846694648460295FFF731
:1055D00085FADFF82893C8494846C0E90015C0E9B4
:1055E0000256C9F81050C9F81450C9F81850C9F833
:1055F0001C50FFF74BF908B1FEF7DCFEBF4DBE486B
:10560000C4F8349044352830C9F82440C5E900076F
:10561000C5E90286C5F81080C5F81480C5F8188061
:105620002846C5F81C80FFF731F908B1FEF7C2FE25
:1056300025630022012134206C62FFF7C1FB342076
:10564000F0E0DFF8BC824FF0040A43452AD1C36979
:1056500043F48013C361C36903F480130493836923
:1056600043F010038361836903F01003049383699B
:1056700043F0200383618069039200F020000490CE
:105680004FF48050CDE9000169466046FFF726FAE5
:10569000CDE900A569469B480295FFF71FFA05B0C2
:1056A000BDE8F08FDFF86082DFF860C243455CD16F
:1056B000836943F480438361836903F480430493E3
:1056C000836943F0040383618069039200F004005E
:1056D00004904FF40070CDE900016946E046604651
:1056E000FFF7FCF9CDE90095694640460295FFF7C2
:1056F000F5F9DFF80892864909F188094846B0466D
:10570000C0E90015C0E90256C9F81050C9F8145094
:10571000C9F81850C9F81C50FFF7B8F808B1FEF7DF
:1057200049FE764E7A48C4F83490CC361438C9F81D
:1057300024403060C6E90175C6E903857561B5612D
:105740003046F561FFF7A2F808B1FEF733FE266395
:105750000022012125207462FFF732FB2520FFF78C
:1057600021FB20460BF098FA99E7DFF8A881434522
:105770005BD1C36943F40033C361C36903F40033ED
:105780000493836943F0040383618069CDE900A138
:1057900000F00400CDE903206946E0466046FFF7CB
:1057A0009DF90820CDE90005A946694640460295C5
:1057B000FFF794F9DFF86081554940461431C0E99C
:1057C0000015C0E90256C8F81050C8F81450C8F8BF
:1057D0001850C8F81C50FFF759F808B1FEF7EAFD59
:1057E0004D4D4B48C4F8348044352830C8F8244027
:1057F000C5E90007C5E90296C5F81090C5F81490F0
:10580000C5F818902846C5F81C90FFF73FF808B176
:10581000FEF7D0FD25630022012126206C62FFF7F0
:10582000CFFA2620FFF7BEFA39E7DFF8F0C063456C
:105830009AD1C36943F48023C361C36903F480230D
:105840000493836943F0080383618069CDE9009183
:1058500000F00800CDE90320DFF8C490694648460F
:10586000FFF73CF9CDE900B5A846694648460295E0
:10587000FFF734F9DFF8A090254909F18809484677
:105880002839C0E90015C0E90256C9F81050C9F816
:105890001450C9F81850C9F81C50FEF7F7FF08B1AA
:1058A000FEF788FD1C4D1A48C4F83490CC353C38BE
:1058B000C9F82440C5E90007C5E90286C5F810808B
:1058C000C5F81480C5F818802846C5F81C80FEF776
:1058D000DDFF08B1FEF76EFD2563002201212720C0
:1058E0006C62FFF76DFA27209CE70000004C004037
:1058F00000100240001001403004024068080020FF
:1059000000500040001401400038014000080140F0
:105910005800024000440040780900200048004040
:10592000000C0140F8B5044690F83A0020283CD11C
:10593000C1B3BAB394F83800012836D0012084F8F6
:105940003800A162A2850025E563222084F83A0090
:10595000636B17489862636B1648D862636B16488E
:105960001863606B134645630846666B2168024600
:105970003046091DFEF7C8FF2068016841680091A4
:1059800084F83850C16841F48071C1602068416971
:1059900041F0010141612068416941F040014161EC
:1059A0000020F8BDFFE70120FBE70220F9E7000037
:1059B0007F7F0008BB7F0008357F00087047704775
:1059C0002DE9F843044690F839001F4616460D4667
:1059D00020284CD1C5B1BEB194F83800012846D07A
:1059E000012084F838004FF00008C4F83C802120E2
:1059F00084F83900FFF780F9A6848146E684A06820
:105A0000B0F5805F03D004E00120BDE8F883206991
:105A100028B12E465FF0000584F838800EE000269D
:105A2000FAE78021204602F0A3FBA0B9AEB116F838
:105A3000010B21684860E08C401EE084E08C4B46FE
:105A40004FF0000200970028EBD14FF040012046B4
:105A500002F08EFB30B10320D7E735F8020BC0F31C
:105A60000800E6E7202084F839000020CDE7022076
:105A7000CBE7000070B5044690F83900202830D1FB
:105A800069B362B394F8380001282AD0012084F861
:105A900038002162A284E2840025E563212084F895
:105AA0003900236B10489862236B1048D862236B2F
:105AB0000F481863206B134645632668206B321D20
:105AC000FEF722FF21686FF04000086084F838502C
:105AD0002068416941F080014161002070BD0120D2
:105AE00070BD022070BD0000C57F0008F37F000874
:105AF000357F0008704770472DE9FF5F374EDDE9BD
:105B00000E811D46894601230827F07DDFF8D0A0CD
:105B10001446002148B900204FEA0A0242F820103A
:105B2000401CC0B2B842F9D3F375307E401CC0B2FD
:105B30003076B84200D33176DDE90001FCF768FE2B
:105B4000327E4AF82200002001E0401CC0B2B84278
:105B5000FBD3002001E0401CC0B2B842FBD3314669
:105B6000D6E91C27B3461646886F22462B46DBF83B
:105B70007C10FCF79FFC0D46044642464B46FCF762
:105B800099FC02460B4620462946FCF7ACFD8146AF
:105B90008A46DDE9000132463B46FCF72CFD4A46C9
:105BA0005346FCF72EFD32463B46FCF783FC064687
:105BB0000F464A46534600200A49FCF71CFD224680
:105BC0002B46FCF71EFDCBE91C67CBE91E0104B098
:105BD00030463946BDE8F05FFCF71ABE28030020C6
:105BE000082F00200000F03F294808B5416941F026
:105BF00001014161416901F001010091416941F0F8
:105C0000020141614069002200F002000090012180
:105C10000C20FFF7D5F80C20FFF7C4F80022012173
:105C20000D20FFF7CDF80D20FFF7BCF80022012171
:105C30000E20FFF7C5F80E20FFF7B4F8002201216F
:105C40000F20FFF7BDF80F20FFF7ACF8002201216D
:105C50001020FFF7B5F81020FFF7A4F8002201216B
:105C60001120FFF7ADF81120FFF79CF80022012169
:105C70003A20FFF7A5F83A20FFF794F80022012117
:105C80003B20FFF79DF8BDE808403B20FFF78AB8AE
:105C9000001002402DE9F04385B00024294800940B
:105CA000019402940394816941F01001816181693A
:105CB00001F010010491816941F020018161816945
:105CC00001F020010491816941F004018161816941
:105CD00001F004010491816941F00801816180694A
:105CE000DFF8648000F0080042F2CF150490002233
:105CF00029464046FEF7FBFFDFF850904FF400774F
:105D0000002239464846FEF7F2FF0126CDE900564B
:105D1000022569464046CDE90245FEF7DFFE4FF415
:105D200071408DE8310069464846FEF7D7FECDE95F
:105D3000007669464846CDE90245FEF7CFFE05B03C
:105D4000BDE8F0830010024000100140000C01404B
:105D50000C4810B50A4901604FF4614141600021CF
:105D600081600C22C160C0E904128161C161FFF74A
:105D7000C5FB002803D0BDE81040FEF71BBB10BDDB
:105D8000004C0040280700200C4810B50A4901606B
:105D90004FF4E1314160002181600C22C160C0E913
:105DA00004128161C161FFF7A9FB002803D0BDE89F
:105DB0001040FEF7FFBA10BD0050004068070020F9
:105DC0000C4810B50A4901604FF41651416000219A
:105DD00081600C22C160C0E904128161C161FFF7DA
:105DE0008DFB002803D0BDE81040FEF7E3BA10BDDC
:105DF00000380140A80700200C4810B50A4901608E
:105E00004FF416514160002181600C22C160C0E94D
:105E100004128161C161FFF771FB002803D0BDE866
:105E20001040FEF7C7BA10BD00440040E80700204C
:105E30000C4810B50A4901604FF416514160002129
:105E400081600C22C160C0E904128161C161FFF769
:105E500055FB002803D0BDE81040FEF7ABBA10BDDB
:105E60000048004028080020FEE700001CB505217E
:105E70000320CDE900014FF480630022064907A00A
:105E800009F095F807490028C86003D0BDE81C4018
:105E900009F09EB91CBD0000253400084368656305
:105EA0006B4D42004C020020E44CDFF88093DFF899
:105EB00080B3DFF88083E04E4FF00A0AA4F11805A2
:105EC00028780B2805D2002120226254491C082979
:105ED000FBDBB0B1012821D002282DD0032847D008
:105EE000042853D0052858D0062858D0072870D049
:105EF00008286FD009286ED00A286DD00B286CD0E6
:105F00001EE199F8001043E05246B1FBF2F3B3FBF7
:105F1000F2F70AFB17333033A37122E0C94AC84BAA
:105F20000021127803EBC202C1F10703D35C635472
:105F3000491C0829F8DB03E19BF80010632904D908
:105F40006422B1FBF2F23032E271092908D95246DB
:105F5000B1FBF2F3B3FBFAF70AFB17323032A2714E
:105F60005246B1FBF2F30AFB131130316171E7E0E5
:105F7000B34A00213378783202EBC302C1F1070340
:105F8000D35C6354491C0829F8DBD9E0AE49097891
:105F90000929B9D83031A171D2E0AC49F0E0E978F3
:105FA000491CCAB2AA49EA700B78042B03D1D10765
:105FB00001D0202114E0A74942F20F770968B942C5
:105FC0000CD97F1CB1FBF7F7B7FBFAFC0AFB1C717D
:105FD00005E04DE0CDE0CEE0CFE0D0E00021303173
:105FE0002171032B03D1D10701D020210EE0994963
:105FF0004FF47A770968B94206D3B1FBF7F7B7FBDC
:10600000FAFC0AFB1C7100E000213031E170022B28
:1060100003D1D10701D020210DE08E490968632901
:1060200007D96427B1FBF7F7B7FBFAFC0AFB1C7131
:1060300000E000213031A170012B03D1D10701D044
:1060400020210DE083490968092907D95746B1FB8A
:10605000F7F1B1FBFAFC0AFB1C1100E00021303122
:1060600061701BB9D10701D0202168E0794960E057
:10607000E978491CCAB27849EA700B78042B03D13D
:10608000D10701D020210FE0744942F20F7709684F
:10609000B94207D97F1CB1FBF7F7B7FBFAFC0AFB43
:1060A0001C7100E0002130312171032B03D1D10795
:1060B00001D020210EE069494FF47A770968B9428E
:1060C00006D3B1FBF7F7B7FBFAFC0AFB1C7100E043
:1060D00000213031E170022B03D1D10701D0202102
:1060E0000DE05E490968632907D96427B1FBF7F71A
:1060F000B7FBFAFC0AFB1C7100E000213031A170F3
:10610000012B03D1D10701D020210DE053490968AB
:10611000092907D95746B1FBF7F1B1FBFAFC0AFB95
:106120001C1100E00021303161700BB9D1079BD107
:106130004A490A68B2FBFAF30AFB13213031217095
:10614000317803291ED306291CD003294ED00729F4
:106150004CD03B4A0021603A02EBC000404A435C0D
:106160005354491C0829FADB3E480078012857D1CE
:1061700050E03D4904E03D4902E03D4900E03D4931
:10618000097807E77E2188F80010452188F801107A
:106190002B4B0021603B424603EBC0005718435C89
:1061A000491CBB700829F9DB5FF00700C0F107014B
:1061B0001318615C9972401EF8D50020907402207B
:1061C000917C135C401C194491741228F8DB2A4F0F
:1061D0004FF0FF31386808F038FE13221549274880
:1061E000FFF748FC386808F015FE19E0144A002152
:1061F000603A02EBC0001A4A435C5354491C082918
:10620000FADB0720C0F107011318615C1972401E08
:10621000F8D505E003F042FE1948006803F098FF46
:106220004FF4C87008F088FF4AE6000035000020EF
:1062300036000020B02400203B0000204002002057
:106240003B150108380000203A00002037000020EC
:106250004C020020540200204D0200206C0300205C
:1062600004290020880100203D0000203E0000207D
:106270003F00002039000020A40100202807002052
:1062800098020020704700002DE9F041324D0026B1
:106290006878212800D96E703048006807F07EFCCD
:1062A0002F4F6978C928785408D02A78F02A01D06D
:1062B000AA784AB1491C6970BDE8F081C9203870DC
:1062C0006E702E70AE700AE0222943D2092906D3DF
:1062D000394411F8091CC92901D1D92803D068789B
:1062E000401C6870E8E7AE626E71AE712E710024DA
:1062F0004FF0010868782044384410F8080CA0F1E9
:106300003001092913D8C4F10500C1B20A2006F0F2
:10631000F1FF6978AA6A2144394411F8081C303920
:1063200001FB0020A862A879401CA87103E0C428E2
:1063300001D185F80480641C062CDBDB287910B1C0
:10634000A86A4042A8626E7109F0BEFEF020287073
:1063500085F802806E70AFE770020020AC0100206B
:10636000602700202DE9F047894D00266878322803
:1063700000D96E7087482978874F0068F02901D0CE
:10638000A97859B107F00AFC69780A2878544CD0EA
:1063900009284AD0A878401CA870C1E007F0FEFB8D
:1063A00069784FF0F0094FF0010A78540A2802D0BA
:1063B00009287DD0B4E00D2902D138783D2805D0D8
:1063C000781810F8062C202A31D034E0AE622E71F5
:1063D0006E71AE710024B84608EB0407B878303807
:1063E00009280ED8C4F10500C1B20A2006F082FFC8
:1063F000B978AA6A303901FB0020A862A879401C4C
:10640000A871641C062CE7DB98F801002D2802D146
:1064100085F804A002E02879012802D1A86A404248
:10642000A86209F051FE85F80090AE704BE010F8BC
:10643000050C6B2802D02B2942D044E0AE622E71AD
:106440006E71AE710024A84698F8010020443844CB
:1064500010F80C0CA0F13001092918D8C4F105007E
:10646000C1B20A2006F046FF98F80110D8F828209B
:106470002144394411F80C1C303901FB0020C8F8C4
:10648000280098F80600401C88F8060003E02D2834
:1064900001D188F804A0641C062CD5DB98F8040010
:1064A000012804D1D8F828004042C8F8280000E0AC
:1064B00031E009F009FE88F8009088F8026002E0F7
:1064C0003878312802D06E70BDE8F087AE622E7148
:1064D0006E71AE710024B84608EB0407787AA0F11B
:1064E000300109290FD8C4F10500C1B20A2006F015
:1064F00001FF797AAA6A303901FB0020A862A879E5
:10650000401CA87103E02D2801D185F804A0641C6B
:10651000062CE1DB7FE7781810F80A0C2D2802D052
:10652000491C6970D0E76E71AE71AE622E710024A5
:1065300068782044384410F8090CA0F1300109298A
:1065400013D8C4F10400C1B20A2006F0D3FE697862
:10655000AA6A2144394411F8091C303901FB002092
:10656000A862A879401CA87103E02D2801D185F804
:1065700004A0641C052CDBDB2879012802D1A86A61
:106580004042A86209F0A0FD85F80090AE709BE73C
:1065900070020020AC010020602700202DE9F047A8
:1065A000364E002470780A2800D974703448317847
:1065B000344F00684FF00109F02901D0B17881B162
:1065C00007F0ECFA717800F07F000D2878544BD07A
:1065D00002284CD0B078401CB070491C7170BDE8E6
:1065E000F08707F0DBFA00F07F0170780229395458
:1065F00005D0072835D33978022902D031E0397027
:1066000036E0B97920292CD0B4627471B4710025B8
:10661000A0467C19A078303809280ED8C5F10400AE
:10662000C1B20A2006F066FEA178B26A303901FBD9
:106630000020B062B079401CB0716D1C86F80580F6
:10664000052DE6DB78782D2802D1B06A4042B06291
:1066500009F03AFDF020307086F8029086F801804B
:10666000BDE7401C7070BAE7B4707470B7E738705B
:1066700086F801903470B470B1E700007002002019
:10668000AC0100206027002070B5274C0025607801
:106690008C2800D965702548006807F07FFA244AE5
:1066A000617850542378F02B3AD00123B3EB101FBC
:1066B00036D1501810F8012C022A31D110F8022CD2
:1066C00072BB10F8032C012A2AD110F8042C3ABB13
:1066D00010F8052C102A23D1164A10F8063C12781F
:1066E00093421DD110F8131C914217D16571A57109
:1066F00010F80B1C10F80A2C090441EA022110F8CA
:10670000092C1143A16210F80C0C000701D5484276
:10671000A06209F0D9FCF0202070A570657070BDF2
:10672000491C617070BD000070020020AC010020A7
:1067300060270020350000202DE9F0412E4C002775
:106740006078212800D967702C48006807F026FA85
:106750002B4E61780228705408D02278F02A01D09C
:10676000A2784AB1491C6170BDE8F0810220307006
:1067700067702770A7700AE022293BD2102906D340
:10678000314411F8101C022901D10D2803D0607882
:10679000401C6070E8E7A7626771A7710025607808
:1067A0002844304410F80C0C3038092812D8C5F1B0
:1067B0000500C1B20A2006F09DFD6178A26A294455
:1067C000314411F80C1C303901FB0020A062A07983
:1067D000401CA0716D1C062DE1DBB078622802D14F
:1067E000A06A4042A062677109F06EFCF020207040
:1067F0000120A0706770B7E770020020AC01002094
:10680000602700202DE9F0412D4D00246878401CC0
:10681000C0B268703C2800D96C702A48006807F044
:10682000BDF9294E69784F2870542DD02878F0286A
:106830002FD0A87800282CD115292AD130784F28BC
:1068400027D17078542824D1B078412821D1AC6266
:106850002C716C71AC7100244FF001083719387C31
:10686000A0F13001092916D8C4F10500C1B20A20EF
:1068700006F040FD397CAA6A303901FB0020A8628D
:10688000A879401CA8710AE04F2030706C702C7001
:10689000AC70BDE8F0812D2801D185F80480641C1E
:1068A000072CDBDB2879012802D1A86A4042A862C4
:1068B00009F00AFCF020287085F80280E9E7000062
:1068C00070020020AC010020602700202DE9F0417B
:1068D0002D4D00246878401CC0B26870442800D94F
:1068E0006C702A48006807F059F9294E6978022827
:1068F00070542DD02878F0282FD0A87800282CD1DB
:1069000030292AD13078022827D196F83000032880
:1069100023D1AC622C716C71AC7100244FF0010872
:10692000371997F82300A0F13001092917D8C4F1CD
:106930000500C1B20A2006F0DDFC97F82310AA6A10
:10694000303901FB0020A862A879401CA8710AE038
:10695000022030706C702C70AC70BDE8F0812D2876
:1069600001D185F80480641C062CD9DB2879012824
:1069700002D1A86A4042A86209F0A6FBF020287064
:1069800085F80280E9E7000070020020AC010020D9
:10699000602700202DE9F047314C0025607827283A
:1069A00000D965702F4821782F4F00684FF00109FA
:1069B000F02901D0A17859B107F0F0F861780328E7
:1069C000785444D0022844D0A078401CA07005E040
:1069D00007F0E4F861780328785403D0491C61700B
:1069E000BDE8F087092930D1387802282DD1A56279
:1069F0006571A5715FF0000607EB060898F80200C4
:106A0000303809280FD8C6F10600C1B20A2006F0B6
:106A100071FC98F80210A26A303901FB0020A062D4
:106A2000A079401CA071387A761C30386071072E2E
:106A3000E2DB78782B2802D0A06A4042A06209F0FD
:106A400043FBF020207084F802906570C8E7A570C1
:106A5000FBE7A570387084F801902570C0E700004E
:106A600070020020AC010020602700202DE9F041D9
:106A7000344D00246878401CC0B26870352800D9B5
:106A80006C703148006807F089F8304E6A7801214F
:106A9000B05432B1032804D1B01810F8010C2328E7
:106AA00032D02878F0284AD0A878002847D16878D2
:106AB000325C042A01D0002A41D11A283FD1307813
:106AC00023283CD17078032839D1B07A0A2836D1EE
:106AD000AC622C716C71AC710024884637197879DE
:106AE000A0F13001092917D8C4F10400C1B20A206D
:106AF00006F000FC7979AA6A303901FB0020A8620F
:106B0000A879401CA8710BE023203070032070701E
:106B100069702C70AC70CAE72D2801D185F804800B
:106B2000641C052CDADB2879012802D1A86A4042CE
:106B3000A86209F0C9FAF020287085F80280BDE843
:106B4000F081000070020020AC01002060270020CE
:106B50002DE9F047644D00266878112800D96E7041
:106B60006248297801270068DFF88481F02901D084
:106B7000A97891B107F012F869780D2808F801009A
:106B80007ED020287DD030287BD03D2879D02D287C
:106B900077D0A878401CA87006E006F0FFFF69785F
:106BA0000D2808F8010003D0491C6970BDE8F08782
:106BB0004FF0F00A0A2909D908EB010010F8012C5E
:106BC000292A03D110F8040C28282CD004297DD9B7
:106BD00008EB010010F8010C20287BD0AE622E716A
:106BE0006E71AE715FF000046978C4F10509A1EB24
:106BF000090118F80100A0F1300109294BD8C4F1AE
:106C00000400C1B20A2006F075FB6A78A2EB090203
:106C100018F80210AA6A303901FB0020A862A8798E
:106C2000401CA8713AE0AE622E716E71AE71002404
:106C30006978C4F10909A1EB090118F8010030389D
:106C4000092812D8C4F10400C1B20A2006F052FB90
:106C50006A78A2EB090218F80210AA6A303901FB1F
:106C60000020A862A879401CA871641C052CDFDBF9
:106C700069782C4608EB010010F80B0C2D2801E078
:106C80002AE02BE01FD1284629791AE0816A49427F
:106C900081622F7117E02D2800D12F71641C052C03
:106CA000A2DB29792C46012902D1A06A4042A062C8
:106CB0006078062807D9404410F8070C2D2802D127
:106CC00028460029E2D009F0FFF900E002E084F84C
:106CD00000A0A7706E7069E7AE70FBE7AE7088F831
:106CE00000006F702E7061E770020020AC01002080
:106CF000602700202DE9F041344D002768782128D5
:106D000000D96F703248006806F048FF314E69784C
:106D100000F07F00705409B1022808D02A78F02AC8
:106D200001D0AA784AB1491C6970BDE8F0810220FF
:106D300030706F702F70AF7010E0222944D210298C
:106D40000CD3314411F8102C022A07D111F80E1C73
:106D5000302901D0322901D10D2803D06878401C98
:106D60006870E2E7AF626F71AF7100246878204409
:106D7000304410F80C0C3038092812D8C4F1050042
:106D8000C1B20A2006F0B6FA6978AA6A21443144F1
:106D900011F80C1C303901FB0020A862A879401CB6
:106DA000A871641C062CE1DB6878304410F80E0CE6
:106DB000322802D1A86A4042A8626F7109F084F9B2
:106DC000F02028700120A8706F70AEE770020020DC
:106DD000AC010020602700202DE9F047384D002449
:106DE0006878272800D96C7036482978364E0068B4
:106DF0004FF00109F02901D0A97859B106F0CEFE73
:106E000069780328705451D0022852D0A878401CC9
:106E1000A87005E006F0C2FE69780328705403D01C
:106E2000491C6970BDE8F087A8460B293BD1307832
:106E3000022838D1AC626C71AC7100257719B87832
:106E40003038092812D8C5F10500C1B20A2006F071
:106E500051FABA78D8F82830303A02FB0030C8F836
:106E6000280098F80600401C88F806006D1C062DC6
:106E7000E4DB307A45463038C0B288F80500012896
:106E800005D16C71A86A0A2190FBF1F0A8627078B4
:106E90002B2802D0A86A4042A86209F015F9F02018
:106EA000287085F8029088F80140BBE7AC706C70E0
:106EB000B8E7AC70307085F801902C70B2E7000034
:106EC00070020020AC010020602700202DE9F04175
:106ED0002F4C00256078262800D965702D48006861
:106EE00006F05CFE2C4E617800F07F0003297054A0
:106EF00001D3022808D02078F02801D0A07848B12A
:106F0000491C6170BDE8F081022030706570257009
:106F1000A5700CE0262939D2112908D3701810F871
:106F2000111C022903D110F8010C0D2803D0607840
:106F3000401C6070E6E7A5626571A846A571002552
:106F400077193879303809280ED8C5F10500C1B253
:106F50000A2006F0CFF93979A26A303901FB002006
:106F6000A062A079401CA0716D1C062DE8DBB078F2
:106F7000800702D5A06A4042A062454684F8058099
:106F800009F0A2F8F02020700120A0706570B9E728
:106F900070020020AC0100206027002070B52E4C4C
:106FA0002C484FF4807600F13C023146206206F016
:106FB000C3FD2848B5000C3000F598722946606280
:106FC00006F0BAFD23483146183000F22452A06280
:106FD00006F0B2FD1F483146243000F5C362E0627E
:106FE00006F0AAFD1B483146303000F20C722063D7
:106FF00006F0A2FD1948314600F10C02606306F06C
:107000009BFD1748294600F13002A06306F094FD6D
:1070100013486E100C3000F224423146E06306F053
:107020008BFD0F482946183000F5C362206406F036
:1070300083FD0C48802100F10C02A06406F07CFD69
:107040000748314624306064BDE8704000F60C22E9
:1070500006F072BD6C0D00208C010020A8150020E8
:10706000B4160020E42200202DE9F05FFA4C4FF026
:107070000008E06B06F048FD002813D0E06B06F036
:1070800081FD2179F54D012741B101290CD06854CA
:10709000E278002691427CD3002011E07E2801D1C5
:1070A00028702771BDE8F09F687002212171401C93
:1070B000E070F7E7295C401C414401F0FF0880B212
:1070C0009042F7D3A95CC8F1FF0088422BD104227B
:1070D000E249E34807F0F1FEE149E24A8B78107893
:1070E000834201D0FF2BF1D1C978DFF87C831029CE
:1070F0001AD0112925D0122930D015292ED0DFF829
:107100006CC314297ED0A1297DD0A4297CD0162956
:107110007BD017297AD0192979D01A2978D01B2940
:1071200077D0182976D094E1E078E179284410F8F6
:10713000010C8842F7D188F80070772008F010FA27
:1071400087E1E078E179284410F8010C8842EAD11F
:107150006B2008F005FA88F800707AE1C44ADFF87D
:1071600014B3BA461770122902D0152912D070E153
:10717000702007F0D1F908F021FF6878B749801C2A
:10718000C2B2BD4809F0E2FADBF8000007F042FEA7
:107190005FE158E1DFF8E492B04F99F800007F1EFC
:1071A000FD2806D16878C05DFD2802D9702007F05F
:1071B000B3F9687899F80010C25D8A4205D0801C46
:1071C000C2B2A649AC4809F0C1FA6B2008F0C8F970
:1071D00099F80000FD2807D16878C05DFD2803D923
:1071E000DBF8000007F016FE6978C85DFF2816D0AE
:1071F000FE2814D089F800009848C01E085CA049F9
:10720000C00908E00EE0B6E006E1DBE0E5E0EAE018
:10721000F1E0F6E003E10870F52008F0F3FB88F8F0
:1072200000A016E1DFF85C929749DFF830B289F8E8
:1072300000600978DFF820820BF1640B08F1600828
:10724000002902D04FF0010106E029796A79114442
:1072500000F593721144C9B24FF0070288F800207C
:107260004FF07E0388F801304FF0050388F80230B4
:1072700003D09BF8023040EA031088F803004FF077
:10728000A40088F804002B7988F80530687988F81C
:107290000600C1F1FF0088F807009CF80000AA462C
:1072A00020B34FF001014FF0C102084608F0B4FDD1
:1072B00069497648603109F0BDFD0121744AE064F6
:1072C00004E0435C5518491C05F8013C03788B42E7
:1072D000F7DA4FF0FF31206907F0B7FDE06C6C4939
:1072E00002786C48FEF7C6FB206915E06A49012068
:1072F0000D1818F80030401C05F8013C8242F7DAFE
:107300004FF0FF31606907F0A0FD98F80020624956
:107310006248FEF7AFFB606907F07CFD89F80070FA
:107320009AF804005E4D012802D002281DD090E09A
:107330002878002818D15B480078002814D15A48D2
:107340000088002810D15948006807F063FD9BF8B9
:1073500002000109F32008F0CBFA554806705548A1
:107360000670554806702F7073E0687848BBF420AB
:1073700008F048FB6DE0A846474D042740354FF024
:10738000FF3900BFE91918F8070001F8040CAE74C2
:107390000220A97C2A5C401C1144A9741228F8DB45
:1073A0004946A06907F051FD3B491322403143484B
:1073B000FEF760FBA06907F02DFD7F1CBFB2162F02
:1073C000E0D346E028798CF80000012227493CA050
:1073D00009F0C0FC08F0F4FB1EE03A4928790122CC
:1073E000087039A004E02879107001221D4937A0E7
:1073F00009F0B0FC10E0364928790122087035A068
:10740000F6E702F077F9344928790122087033A0B1
:1074100009F0A0FC08F070FC02F06CF919E03048AB
:10742000E9790170A9794170697981702979C17010
:107430002C4888F8007007706B2008F091F804223F
:10744000274929A0D4E7491CC8B220715A287FF6E1
:1074500030AE2671E67025E68C010020142600204F
:10746000B302002035000020BE02002037000020BB
:107470001F030020D0020020DC0B0020C1020020EE
:10748000C20200202A02002034000020842B0020A9
:1074900070230020E8070020702400202808002026
:1074A00068020020C0020020C4020020D402002094
:1074B0007D020020780200207902002028070020A9
:1074C000415049003B000020504D0000434800005F
:1074D000380000205451000036000020574C0000B6
:1074E000D80200204E02002054696D65436F6E7310
:1074F000740000002DE9F0415B4D0026286C06F079
:1075000003FB002821D0286C06F03CFB6A78574C1E
:107510000121C2B10027012A19D0022A25D07E28D4
:1075200035D07D2836D0A97811B1AF7080F0200019
:10753000A054521C6A70A17868780A46C91C81421E
:1075400003D203202DE07E281CD0BDE8F0817E28E8
:1075500009D07D2819D0A97811B1AF7080F0200032
:10756000607002200CE02070EFE77E280AD07D28B2
:107570000BD0A97811B1AF7080F02000A07003206B
:107580006870E2E720706970DFE7A970DDE72070BE
:107590006970D0E7A970CEE7235C401C3344DEB2AB
:1075A00080B28142F8D83148C6F1FF01C01C105C9E
:1075B000814257D1E078902854D1A07C0A21B1EBC8
:1075C000101F05D0142809D0294AB22813D016E07C
:1075D000A12803D127480078022843D10F2605E0CF
:1075E000A15D686C06F0AFFA761CB6B2A078C01C3C
:1075F000B042F5D829E0E07C2146032806D0617C22
:107600001278914215D0FF2913D01EE0164B0020AE
:1076100058330E1836791E54401C80B20828F8D30F
:10762000607C1178884201D1012000E0002028729E
:107630000BE00F2605E0A15DE86B06F084FA761CEE
:10764000B6B2A078C01CB042F5D8A07C182809D1E9
:10765000054900205031221812790A54401C80B28A
:107660000828F8D36F7070E78C010020B025002047
:10767000350000203B0000202DE9F05FB84E0027C8
:10768000706C06F041FA002815D0706C06F07AFA9A
:10769000B179B44C4FF0010A41B101290DD06054C9
:1076A0007279002591427BD3002011E07E2802D11F
:1076B000207086F806A0BDE8F09F60700221B171CD
:1076C000401C7071F7E7215C401C3944CFB280B296
:1076D0009042F8D3A15CC7F1FF00B04688422ED19A
:1076E000A67898F8003006F00F019F4A9F48474659
:1076F000994207D190F800C0BCF1020F12D0BCF142
:10770000070F0FD092F800C0614507D190F800C074
:10771000BCF1020F02D0BCF1070F03D1002BDED168
:107720000A2EDCD1E6784FF0FF3BA12E08D0F12ED7
:1077300006D0A42E3DD0A22E43D0142E41D002E17B
:107740000078022801D00728F9D1A07BC82802D1EF
:10775000E17BB72925D0E17B2174E0733033844984
:10776000A37304200B18225C401C80B203F8042C85
:107770001628F7D38D7402208A7C0B5C401C1A44B7
:107780008A741228F8DB5946B86907F05EFB1322A9
:1077900077497848FEF76EF9B86907F03BFBD2E00D
:1077A000D6E0202060752075E074A07460742074A9
:1077B000D3E70078022801D0072801D101F09AFF11
:1077C000C1E0007802287DD007287BD060780528AA
:1077D00078D1DFF8A491624E0720603689F8005016
:1077E00030707E2070700520B070644800780028EA
:1077F000107801D040EA0110F070A420307159488F
:107800006438017971714079B071F5710120317876
:10781000335C401C725C1A44725431788142F6DC4D
:10782000C8B2315CC1F1FF0131545548007808B34A
:107830000121C122084608F0EFFA49495148603158
:1078400009F0F8FA0121504AF86404E0435C561844
:10785000491C06F8013C03788B42F7DA594638692F
:1078600007F0F3FAF86C484902784848FEF702F945
:10787000386917E03E4A0120403A317805E0335C30
:1078800002EB000C401C0CF8013C8142F7DA59462F
:10789000786907F0DAFA3649327840393C48FEF721
:1078A000E9F8786907F0B6FA89F800A05746207918
:1078B000DFF8E090DFF8E0A0DFF8E0B0384E012814
:1078C00004D000E032E0022831D03CE0307868BBE0
:1078D00034488178090602D53349097831B1C07836
:1078E000FE2830D03148007868B12CE001F002FF6A
:1078F0002F4830490222008808802FA009F02AFA78
:1079000004F03AFE1FE02F48008878B92E4800683E
:1079100007F080FAA0780109F32007F0E9FF89F861
:1079200000508AF800508BF8005037700BE07078E8
:1079300048B9F42008F066F889F800508AF8005039
:107940008BF80050777088F8065088F80550B2E63A
:10795000491CC8B2B0715A28F9D9B5717571AAE637
:107960008C01002078260020350000203B000020FC
:10797000B0240020280700202A0200203400002024
:1079800037000020842B002070230020E80700200F
:10799000280800207D0200207802002079020020C3
:1079A00068020020EC020020BC020020C00200207F
:1079B0009202002042000020626567696E77656967
:1079C00067687400C4020020D40200200248034902
:1079D00000784870704700003D000020082C00200F
:1079E00070B52F4D4FF0FF31286807F02EFA2D4863
:1079F0000078E8B101281ED002281FD0032820D02B
:107A0000042821D0052822D0062823D0072824D0F6
:107A1000082825D0092826D00A2827D00B2828D0C6
:107A20000C2829D00D282AD01F4C0E282DD031E04B
:107A3000FFF760F92EE0FEF7E5FE2BE0FEF792FC83
:107A400028E000F02BFD25E0FFF710F822E0FFF71B
:107A50007FF81FE0FEF7A2FD1CE0FEF715FC19E021
:107A6000FEF734FF16E0FEF70FFE13E0FFF72EFAE5
:107A700010E0FFF7B1F90DE0FEF78CFF0AE0FEF72A
:107A80005BFE07E0206806F089F8206806F048F8F9
:107A90000028F7D12868BDE8704007F0BBB90000A6
:107AA0002C02002038000020AC0100201CB50B483F
:107AB00000780E2811D104200521CDE900014302F0
:107AC0000022074907A007F072FA094900288863D5
:107AD00003D0BDE81C4007F07BBB1CBD3800002074
:107AE000F57A00085265616457656967687400003B
:107AF00070020020104E114D114F124C4FF0FF3804
:107B00004146286807F0A1F904F0D8FE80B2E0846D
:107B1000317801B14042A06238786071286807F07E
:107B200079F908F0D1FAE08B322801D8401CE083C3
:107B30007D2007F001FBE3E7310300202C02002049
:107B40003E0000207002002003B5DDE90001B0FB1B
:107B5000F1F0DDE90012B1FBF2F302FB1311B2EB1D
:107B6000410F00D8401C0CBD704700008F4CDFF85F
:107B70002C92DFF82CB28B4FDFF82CA28C4D4FF0FB
:107B80000008661EE879142801D9A87918B1A879E7
:107B900001284ED0FAE020790F21B1EB101F13D14C
:107BA000103820712178012004F8018004E0625C23
:107BB000235C401C1A44625421788142F7DCC8B22D
:107BC000205CC0F1FF00605499F800004FF0FF31D5
:107BD0000028DAF800001FD007F037F92079F828DC
:107BE0000ED0E8280CD00020C022002108F014F9A3
:107BF0006E49704809F01EF90121CBF8000006E03B
:107C00000120F1E7425C7B18491C03F8012C027843
:107C10008A42F7DAD2B2A6E007F017F901202278FB
:107C200004E0215C3B18401C03F8011C8242F8DA96
:107C300099E06B2008F0C2FDF0B303F0DDFF401CBB
:107C40004CD099F8000018B32079F8280CD0002007
:107C5000C022002108F0E0F85449564809F0EAF83B
:107C60000121CBF8000006E00120F1E7425C7B181F
:107C7000491C03F8012C02788A42F7DA4FF0FF31F1
:107C8000DAF8000007F0E1F8DBF80000027810E015
:107C90000120217804E0225C3B18401C03F8012CF1
:107CA0008142F8DA4FF0FF31DAF8000007F0CDF842
:107CB00022783C49404800E011E0FDF7DBFE32202D
:107CC00007F03AFADAF8000007F0A4F885F8068021
:107CD00085F8078020783949805D087056E0A879DA
:107CE000012853D1772008F069FD04284ED903F00C
:107CF000ABFF04284AD199F8000018B32079F8287E
:107D00000CD00020C022002108F086F8274929481D
:107D100009F090F80121CBF8000006E00120F1E71E
:107D2000425C7B18491C03F8012C02788A42F7DA7E
:107D30004FF0FF31DAF8000007F087F8DBF80000B9
:107D4000027810E00120217804E0225C3B18401CFE
:107D500003F8012C8142F8DA4FF0FF31DAF8000025
:107D600007F073F822780F491348FDF783FE32209D
:107D700007F0E2F9DAF8000007F04CF885F8068021
:107D800085F807802078815D0C480170E879401CF7
:107D9000E871642007F0D0F9F4E600003700002015
:107DA000D8010020702300209C010020DC26002048
:107DB000B8020020842B0020E80700209301002057
:107DC0001CB50520009001904FF440730022064935
:107DD00006A007F0ECF808490028C86203D0BDE807
:107DE0001C4007F0F5B91CBD6D7B000853656E643F
:107DF0005769666900000000B802002070B50E489F
:107E0000062204244578182300210C48082D0ED2A0
:107E1000DFE805F00409090909090909C1730174BA
:107E20000475847470BD01740375827470BD01742F
:107E300020210175F5E70000082C00202803002010
:107E400010B506F05FFD07F05BFABDE8104006F0E4
:107E500067BD30B58FB028216846FAF728FA14219B
:107E60000AA8FAF724FA01210804CDE90010002439
:107E7000029402250491CDE907504FF4E0100990D7
:107E80006846FDF7BBF80F20CDE90A056802CDE989
:107E90000C400E9002210AA8FCF7C4FF0FB030BDC1
:107EA000144910B54868144A10F00C03134803D065
:107EB000042B01D0082B09D002604968104AC1F395
:107EC0000311515C0268CA40026010BD4A684B68E9
:107ED00002F470124FF0020413F4803F04EB92425C
:107EE00002D04B689B0301D5064B00E0024B5A437E
:107EF000E2E700000010024000127A0004000020B7
:107F0000000F010800093D007047000010B504484B
:107F1000FDF746FABDE81040014800F07FB90000C7
:107F20002807002010B5406A0021C185C184FDF7F3
:107F300035FA10BD70B5446A2068406994F839106C
:107F4000C0F3C0100025212904D118B1E5842046D2
:107F500000F062F82068406994F83A10C0F380108D
:107F6000222904D118B1E585204600F047F8E06BDE
:107F700040F01000E0632046FDF710FA70BD10B528
:107F80000146406A09680968890613D40021C18541
:107F90000168CA6822F48072CA6001684A6922F0E6
:107FA00001024A6101684A6922F040024A612021C7
:107FB00080F83A10FDF702FD10BD10B5406AFDF7DC
:107FC000FEFC10BD10B50146406A096809688906C3
:107FD0000CD40021C18401684A6922F080024A6100
:107FE0000068C16841F04001C16010BDFDF782FD2D
:107FF00010BD10B5406AFDF77EFD10BD0168CA686E
:1080000022F49072CA6001684A6922F001024A6152
:10801000202180F83A1070470168CA6822F0C00237
:10802000CA60202180F83910704710B590F83A10D6
:10803000222901D0022010BD82684FF480539A4259
:1080400001D1016921B1816A9A421BD04AB10AE08B
:108050000268816A5268C2F308020A80816A891C38
:1080600008E0026972B10268526802F07F020A7089
:10807000816A491C8162C18D491E0904090CC185B0
:1080800003D016E002685268F1E70168CA6822F07E
:108090002002CA600168CA6822F48072CA6001685E
:1080A0004A6922F001024A61202180F83A10FDF766
:1080B00085FC002010BD000070B504460068016911
:1080C000E26821F44051114301612169A06808432D
:1080D000616908432168CA6841F20C639A4302430C
:1080E000CA6020684169A26921F44071114341616D
:1080F0001E492068884202D1FCF73AFF01E0FCF7F4
:1081000027FF00EBC00101EB0012606864218000D2
:10811000B2FBF0F3B3FBF1F36FF018067343B2FB5D
:10812000F0F5B2FBF0F605EB8305322303EB051502
:10813000B5FBF1F5B6FBF1F605F0F00505EB06151C
:10814000B2FBF0F6B2FBF0F0B0FBF1F06FF018020A
:10815000504306EB800003EB0010B0FBF1F0216808
:1081600000F00F002844886070BD00000038014016
:108170002DE9F041984617460E460446069D1DE03F
:10818000681C1BD02DB1FCF7B7FDA0EB0800A8427E
:1081900014D92068C16821F4D071C1602068416998
:1081A00021F001014161202084F8390084F83A006F
:1081B000002084F838000320BDE8F08120680068C2
:1081C00036EA000004D00020B842D9D00020F3E7FE
:1081D0000120F9E710B50448FDF7E2F8BDE81040CA
:1081E000014800F01BB80000A807002010B50448A3
:1081F000FDF7D6F8BDE81040014800F00FB80000C8
:10820000E807002010B50448FDF7CAF8BDE81040A3
:10821000014800F003B8000028080020F8B5074620
:1082200000680168C1F3001100296FD001680025C2
:10823000406800903846FDF785F8514C257051494B
:108240003868884217D1504800684068C0F164001F
:1082500020704E4E04E0715D012000F0B3F86D1CFB
:1082600020788542F7DB64220021484806F076FC3E
:108270006422464976E0464A4649904229D146481A
:1082800000684068C0F1640020700878434E0128FF
:1082900001D0002512E030784F2812D170784B2899
:1082A0000FD1B0780D280CD13D48006806F0B2FD22
:1082B00007E0715D022000F085F86D1C2078854292
:1082C000F7DB64220021354806F048FC642233497C
:1082D00048E0344A90422AD1334800684068C0F1EF
:1082E000640020700878314E012801D0002513E089
:1082F00030784F2813D170784B2810D1B0780D28E2
:108300000DD12B48006806F085FD08E036E0715D70
:10831000032000F057F86D1C20788542F7DB6422BB
:108320000021224806F01AFC642220491AE0214963
:1083300088421AD1204800684068C0F1640020706B
:1083400000251E4E04E0715D042000F03BF86D1C1A
:1083500020788542F7DB64220021184806F0FEFBF6
:10836000164964223846FDF7DDFA2078002805D04A
:1083700013480068BDE8F84006F04CBDF8BD0000A9
:108380000100002000380140F0080020980500207E
:10839000004400400000002078090020FC05002077
:1083A0009C01002000480040000A002060060020D8
:1083B000A0010020004C004068080020C4060020F6
:1083C000980100200B4A01280AD002280AD003286D
:1083D0000AD004280AD005280AD1106B05F0B3BBD7
:1083E000106AFBE7506AF9E7906AF7E7D06AF5E7A9
:1083F000704700008C010020FEE70000034804499C
:1084000001224078087003A008F0A4BC082C0020CA
:108410003D00002061645F46530000002DE9F041FB
:108420001D4F88460446012204213846FCF75FFCB4
:108430000120FBF76FFD25E008EB0400002510F894
:10844000016C002204213846FCF751FC300601D5AE
:10845000012200E0002201213846FCF748FC0120FF
:10846000FBF758FD012204213846FCF740FC0120AF
:10847000FBF750FD70066D1C060EEDB2082DE0D323
:10848000641EE4B2002CD7D13846BDE8F04100228A
:108490000121FCF72CBC0000001001402DE9F04741
:1084A000524C00256078252800D965705048006836
:1084B00005F074FB4F4E61784FF00109721870544B
:1084C00012F8012C772A03D16E280AD0772808D019
:1084D0002378F02B01D0A37863B1491C6170BDE80B
:1084E000F087772030706E20707084F801902570CE
:1084F000A57007E00F2977D20C2903D30D2A01D1EB
:108500000A2803D06078401C6070E8E7A5626571B6
:10851000A846A5714FF00A0A0D2902D00C2924D0D3
:108520004CE000257719F878A0F1300109290FD81F
:10853000C5F10600C1B20A2004F0DCFEF978A26A97
:10854000303901FB0020A062A079401CA07108E036
:108550002E2806D1C5F106006071A16A91FBFAF0E0
:10856000A0626D1C072DDDDB28E000257719F87867
:10857000303809280FD8C5F10400C1B20A2004F030
:10858000B9FEF978A26A303901FB0020A062A07917
:10859000401CA07109E0B8782E2806D1C5F106006C
:1085A0006071A16A91FBFAF0A0626D1C052DDDDB04
:1085B000607918B9A16A91FBFAF0A062B0782D2811
:1085C0000CD084F8048000BF07F07EFDF0202070FE
:1085D00084F8029084F8018081E705E084F8049033
:1085E000A06A4042A062EFE7657078E77002002061
:1085F000AC010020602700200948017800290ED135
:10860000817900290BD0817A002908D1826B016A17
:10861000036C8A1A1A440264816300F00DB8704733
:1086200028030020024803490068086470470000DE
:108630005000002028030020034804490422006C55
:10864000086003A008F086BB28030020500000202B
:1086500061645F546172650030B51A49C87A4B6C29
:1086600000EB80008400B3FBF4F0B3FBF4F3CA6AC0
:108670000024101A13448A6A82421DD39A421BD8DE
:10868000886B431E451C9A4201D3AA4214D9451F48
:10869000431DAA4210D99A420ED24B79052B0DD315
:1086A000084B82421B6C03D3401C5B1C886302E0B6
:1086B000401E5B1E88630B644C7130BD5B1C4B71AC
:1086C00030BD0000280300200FB4054B10B503A9EE
:1086D000044A029800F0A6FB10BC5DF814FB0000F1
:1086E00025C100088C0500200907090E002804DBBD
:1086F00000F1E02080F80014704700F00F0000F156
:10870000E02080F8141D7047002806D00E4910F0B4
:10871000FF0F03D0C0B2085C401C704710F47F4FBD
:1087200004D0C0F30720085C0930704710F47F0FB5
:1087300004D0C0F30740085C1130704701EB1060B3
:108740000078193070470000CA18010802E008C814
:10875000121F08C1002AFAD170477047002001E0BB
:1087600001C1121F002AFBD170472DE9F04F89B0DB
:10877000154683460C4600268846EA461BE004F16F
:108780002009A94501D2202700E02F1B3B466A465D
:108790002146584600F026F80020514608E0FF2EFA
:1087A00004D00A5CFF2A01D104EB00080E5C401CD7
:1087B000B842F4D34C46AC42E1D3FF2E03D0284656
:1087C00009B0BDE8F08F08F1030020F00300F7E7DF
:1087D00010B50024806801F0A3FF002800DA01240E
:1087E000204610BD10B50024806802F003F9204631
:1087F00010BD10B50024806802F0B4F9002800DA3A
:108800000324204610BD002210B5491E0B4605E08A
:108810004C0100EBD404247814B1521C491EF7D249
:10882000981A10BD70B504000498154606D0B1B171
:10883000002D25D0227C002A69D132E035A0FFF737
:1088400043FF37A0FFF740FF172236A13BA0FFF7F9
:108850003BFF3D4A3DA13EA0FFF736FFFEE72DA0BE
:10886000FFF732FF2EA0FFF72FFF18222DA133A014
:10887000FFF72AFF344A3EA135A0FFF725FFFEE7A8
:1088800024A0FFF721FF26A0FFF71EFF192225A134
:108890002AA0FFF719FF2C4A37A12DA0FFF714FFDC
:1088A000FEE721602371E06101F0BCFE284601F083
:1088B000E3FFA06000281DD01C3001F0EDFDE16851
:1088C000006A002922D0B1FBF0F200FB1210002850
:1088D0001DD010A0FFF7F8FE11A0FFF7F5FE2F2224
:1088E00010A116A0FFF7F0FE174A26A118A0FFF767
:1088F000EBFEFEE707A0FFF7E7FE09A0FFF7E4FEA7
:10890000294628A0FFF7E0FE042070BDE0600020AB
:1089100070BD00005B466C61736844425D000000FE
:10892000200000002E2E5C666C61736864625C73CC
:1089300072635C6664622E63000000002825733A4F
:1089400025642920000000001B100108646200005B
:108950002825732920686173206173736572742000
:108960006661696C65642061742025732E0A0000BD
:108970006E616D6500000000706172745F6E616D04
:108980006500000064622D3E7365635F73697A65FC
:10899000202520626C6F636B5F73697A65203D3DB3
:1089A000203000004572726F723A20506172746913
:1089B00074696F6E2028257329206E6F7420666F8E
:1089C000756E642E0A00000070B50D00044610D0CC
:1089D00012A0FFF779FE14A0FFF776FE2079226837
:1089E000002818D011A12B46BDE8704011A0FFF758
:1089F0006BBE1B4C01250574207800280AD107A006
:108A0000FFF762FE08A0FFF75FFE16A117A0FFF7B1
:108A10005BFE257070BD1EA1E5E700005B466C6142
:108A2000736844425D00000020000000545344423B
:108A3000000000004572726F723A202573202825CD
:108A4000732920697320696E697469616C697A653C
:108A5000206661696C20282564292E0A0000000028
:108A600030000020312E302E30000000466C617343
:108A70006844422056257320697320696E697469C1
:108A8000616C697A6520737563636573732E0A0080
:108A90004B56444200000000F0B599B00026044651
:108AA0000120179684F8290022483546CDE9004078
:108AB00017AB324611A90296204606F08BFDA0683E
:108AC000E168806BB0FBF1F0179988420CD11AA0D5
:108AD000FFF7FAFD1CA02168FFF7F6FD1CA0FFF7C9
:108AE000F3FD204602F0E4FA616909B120468847A7
:108AF00024482346CDE90050002211A918460295CA
:108B000006F068FD204F2246002303A91046009777
:108B100003F0F2FF94F8280018B1204603F070FB30
:108B2000F1E784F82950A16909B12046884719B0B6
:108B30003046F0BD259800085B466C61736844427E
:108B40005D5B6B765D0000005B25735D20000000BF
:108B5000416C6C20736563746F7220686561646535
:108B60007220697320696E636F72726563742E2060
:108B700053657420697420746F2064656661756C38
:108B8000742E0A00019700082197000870B51C4652
:108B900015000DD06FF0180202EB4412D3082A46DC
:108BA000FFF720FE21462846BDE87040FFF72BBEA8
:108BB00008A0FFF789FD0CA0FFF786FDA4220BA1FA
:108BC00011A0FFF781FD134A13A117A0FFF77CFD49
:108BD000FEE700005B466C61736844425D5B757440
:108BE000696C735D00000000200000002E2E5C66A2
:108BF0006C61736864625C7372635C6664625F7507
:108C000074696C732E6300002825733A256429204B
:108C100000000000CA1401087374617475735F74F6
:108C200061626C650000000028257329206861736B
:108C300020617373657274206661696C656420617C
:108C4000742025732E0A000070B506466FF01800D8
:108C500000EB41101546C1084FF0FF34FF223046AB
:108C6000F9F71EFB1DB1AC000020241F3055204633
:108C700070BD000070B51446049A0D4606469A422F
:108C800010D319A0FFF720FD1CA0FFF71DFD8D22BA
:108C90001BA122A0FFF718FD234A24A12AA0FFF759
:108CA00013FDFEE76CB119462046FFF7CDFF411CCE
:108CB00018D0221829183046BDE870400423FFF769
:108CC00098BD09A0FFF700FD0CA0FFF7FDFC8E2268
:108CD0000BA112A0FFF7F8FC134A23A11AA0FFF77B
:108CE000F3FCFEE7002070BD5B466C617368444294
:108CF0005D5B7574696C735D00000000200000000E
:108D00002E2E5C666C61736864625C7372635C6671
:108D100064625F7574696C732E6300002825733A72
:108D20002564292000000000B814010873746174E0
:108D300075735F696E646578203C20737461747527
:108D4000735F6E756D0000002825732920686173BC
:108D500020617373657274206661696C656420615B
:108D6000742025732E0A00007374617475735F7428
:108D700061626C650000000003480168814201D017
:108D80000120704700207047780500202DE9F04F42
:108D900089B092468B460646002400E0641C305D94
:108DA000202803D0092801D05C45F7D34FF0FF38C5
:108DB0007CB3194804F10609184F056811E0062232
:108DC00017492868F9F79FFA50B9286822463146B2
:108DD000801DF9F798FA18B9296811F8090020B12F
:108DE000083538688542EAD314E06C688CB12021DC
:108DF0006846F9F75CFA6A465946304604F030FA9C
:108E000038B16946A047CAF80000002009B0BDE8A3
:108E1000F08FFFE74046F9E7E4040020E804002073
:108E200054D200082DE9FF4F8DB00F4605460026AD
:108E300006E025280BD0DDE90F1290476D1C761C4B
:108E400028780028F5D111B03046BDE8F08F002415
:108E5000A246A1460122EC4900E0044315F8013F77
:108E6000203B02FA03F00842F7D128782A2810D0D4
:108E70006FF02F022878A0F13001092914D80AEBED
:108E80008A0102EB410144F0020400EB010A6D1C6F
:108E9000F0E701CF5FEA000A03D544F40054CAF1B9
:108EA000000A44F002046D1C28782E2817D115F80A
:108EB000010F44F004042A280ED06FF02F02287806
:108EC000A0F1300109290AD809EB890102EB41011F
:108ED00000EB01096D1CF2E757F8049B6D1C287824
:108EE0006C280FD006DC4C2817D068280DD06A28D3
:108EF00014D104E0742810D07A280FD10DE044F486
:108F000000140AE044F4801401E044F44014697849
:108F1000814202D104F580146D1C6D1C2A786E2AE2
:108F20001FD00CDC632A31D004DC002A8BD0582AF5
:108F300011D1A3E0642A68D0692A0CD165E0732AB4
:108F40002ED004DC6F2A73D0702A04D19BE0752ADE
:108F50006FD0782A6ED01046DDE90F129047761C4C
:108F600050E1C4F30250022806D0032809D0042897
:108F700001CF09D0066045E101CFF117C0E90061DA
:108F800040E101CF06803DE106703BE117F8040B9C
:108F90008DF8000000208DF80100EB46012003E071
:108FA00057F804BB4FF0FF3061074FF0000102D4C7
:108FB0000DE008F10101884649450FDA8045F8DBEC
:108FC0001BF808100029F4D108E008F101018846D7
:108FD0008142FADB1BF808100029F6D1DDE90F23E6
:108FE000AAEB08008146214600F036F9304400EB38
:108FF000080604E0DDE90F121BF8010B9047B8F1F9
:109000000108F7D221464846F7E00A21C4F302538B
:109010004FF0000B0891022B04D001CFC117032B96
:1090200009D00AE0FF1D27F00707F7E8020108E072
:1090300032E01FE020E000B2C117042B01D140B2A2
:10904000C117031E71F1000307DA4FF0000CD0EBDB
:109050000C006CEB01012D2302E0230504D52B232A
:109060008DF82430012303E0E30701D02023F7E744
:10907000984658E00A2110E010210EE010204FF031
:10908000000B08900CE010214FF0000B44F004049A
:109090004FF00809089103E008214FF0000B0891F8
:1090A000C4F30253022B04D001CF0021032B06D0BE
:1090B00006E0FF1D27F00707F7E8020103E080B292
:1090C000042B00D1C0B24FF0000823072BD5702A23
:1090D00007D0DDF820C08CF0100C5CEA0B0C05D03A
:1090E0000EE040238DF82430012308E050EA01030C
:1090F00006D030238DF824308DF8252002239846A1
:10910000DDF820C08CF0080C5CEA0B0C0BD150EAA7
:10911000010301D1630706D530238DF824304FF0C9
:109120000108A9F10109582A04D038A20B9208AA13
:109130000A920BE03AA2F9E75B46089AF9F794FB2A
:109140000B9B9B5C0A9A521E0A92137050EA010212
:10915000F2D10A98ADEB000000F1200B600702D5B8
:1091600024F4803401E04FF00109D94502DDA9EB78
:109170000B0000E0002000EB0B0141440890AAEB3B
:10918000010AE00306D4DDE90F232146504600F032
:1091900063F806444FF0000908E009A911F8090036
:1091A000DDE90F12904709F10109761CC145F4DB96
:1091B000E0030CD5DDE90F232146504600F04CF8C2
:1091C000064404E0DDE90F1230209047761C089930
:1091D000481E08900029F5DC08E00A980A990078F2
:1091E000491C0A91DDE90F129047761CBBF1000182
:1091F000ABF1010BF1DC21465046DDE90F2300F015
:1092000019F806446D1C1BE6092801003031323381
:1092100034353637383961626364656600000000B2
:10922000303132333435363738394142434445469C
:10923000000000002DE9F041044600251E461746B7
:10924000880404D405E039462020B0476D1C641E14
:10925000F9D52846BDE8F0812DE9F0410446002506
:109260001E469046C80301D5302700E02027880419
:1092700004D505E041463846B0476D1C641EF9D55B
:109280002846BDE8F08100002DE9FC411F46044658
:10929000DDE90831DDE90A651C3040600060C4E9A1
:1092A0000A27C4E90C310A4623211846243405F064
:1092B00055FCD4E903014218D4E901010D4B121FFA
:1092C00005F004FB2060A67666760020A562E061CA
:1092D000E562606120766066A066243C00902346CB
:1092E0000190054A194604F1540006F07BF800206D
:1092F000BDE8FC81F9EF00083FF2000810B5029CC0
:1093000024F001044474C0E909120021C0E90B31C2
:109310001C304060006010BDF0E907124A60D0E9DF
:1093200000121160406000607047000070B5064692
:109330006420FAF7EFFD002202212B48FBF7D7FC4F
:10934000012251022948FBF7D2FC6420FAF7E2FD22
:10935000274CFF252146A570657025700320FFF777
:109360005DF86570257021460220FFF757F8C82088
:10937000FAF7D0FD0820207021460120FFF74EF8B3
:109380000020A0700420607066B378202070184917
:109390000320FFF743F81020207015490120FFF744
:1093A0003DF88020A07002206070172020701049C6
:1093B0000320FFF733F8282020700D490120FFF724
:1093C0002DF8402020700A490120FFF727F85C2083
:1093D000207007490120FFF721F8BDE87040052003
:1093E000FAF798BD5020D1E700100140000C014071
:1093F000840300200E4810B5046A016C002301228A
:109400008C4203D303724372641A02E00272427206
:109410000C1B4462846BA14205D3091B04E08372D8
:1094200010BD827210BD611A0529FAD2F7E700005B
:1094300028030020F1B5104D1048A96C0E46F8F72E
:10944000FBFF0446686BF9F7BDF92146F8F7BCFF4E
:1094500004460098F9F7B6F92146F8F7B5FF31460A
:10946000F8F7B8FFF9F7EDF90022054BF9F722F804
:10947000BDE8F840F9F7CCB9280300200024F448EF
:109480000000E03F70B56420FAF744FD002202219D
:109490002948FBF72CFC012251022848FBF727FC46
:1094A0006420FAF737FD264CFF252146A57065702C
:1094B00025700320FEF7B2FF65702570214602205B
:1094C000FEF7ACFFC820FAF725FD082020702146E2
:1094D0000120FEF7A3FF0025A57004206070502036
:1094E000207021460320FEF799FF102020702146AE
:1094F0000120FEF793FFA5700220607017202070F6
:1095000021460320FEF78AFF2820207021460120F3
:10951000FEF784FF4020207021460120FEF77EFFE9
:109520005C20207021460120FEF778FFBDE87040E6
:109530000520FAF7EFBC000000100140000C0140CC
:109540008403002000224FF480710148FBF7CFBB59
:1095500000100140012211020148FBF7C8BB0000C6
:10956000001001402DE9F84317468846814604263D
:109570001D46FF2231466846F8F792FE25F00304A7
:1095800023463A4641464846FFF733F92A1B00284E
:109590000CD1002A0AD0E1196846F8F76FFE04EBF7
:1095A000080133466A464846FFF723F9BDE8F883C9
:1095B0002DE9F0418AB0002504464FF0FF300795B1
:1095C0000895CDE9030403A8CDE905208846214884
:1095D00008A9CDE9001007AB2A460295414620466E
:1095E00005F0F8FF1C4F0898012640B1CDE900575F
:1095F00004AB022241462046029605F0EBFF079895
:10960000002823D00399491C20D1012802D894F8BE
:10961000280048B1CDE9005704AB0122414620465D
:10962000029605F0D7FF11E00CA0FFF74DF80FA050
:109630002168FFF749F840F243320EA114A0FFF76A
:1096400043F816A0FFF740F884F8286003980AB0A2
:10965000BDE8F08195F60008C99600085B466C618C
:10966000736844425D5B6B765D0000005B25735D53
:10967000200000002E2E5C666C61736864625C736F
:1096800072635C6664625F6B7664622E63000000E6
:109690002825733A25642920000000005472696768
:1096A000676572206120474320636865636B2061B2
:1096B0006674657220616C6C6F63204B5620666126
:1096C000696C65642E0A0000027862B102694B6819
:1096D0009A4208D98278012A07D0022A03D10A685F
:1096E00092F828200AB10020704789684069086014
:1096F000012070470148406805F08CBB4C020020F7
:1097000010B502460846117839B19178032904D181
:10971000012180F8281002F073FD002010BD000028
:1097200030B50D4604464178007887B009B103286A
:1097300002D0012837D033E020A0FEF7C5FF23A0D8
:109740002968FEF7C1FFA17804F110022148FEF755
:10975000BBFF2146284603F021FC002817A010D0AB
:10976000FEF7B2FF19A02968FEF7AEFF40F2BA5229
:1097700019A120A0FEF7A8FF2148A168FEF7A4FFC9
:1097800019E0FEF7A1FF11A02968FEF79DFF4FF435
:10979000B76211A117A0FEF797FF1AA0FEF794FF7A
:1097A000002007B030BD05200090062301AA2846FE
:1097B000216BFFF75FFA0120F3E700005B466C6165
:1097C000736844425D5B6B765D0000005B25735DF2
:1097D00020000000CC1B01082E2E5C666C617368B3
:1097E00064625C7372635C6664625F6B7664622E53
:1097F000630000002825733A25642920000000003A
:10980000641C01085265636F76657279207468651F
:10981000204B56207375636365737366756C2E0AEF
:109820000000000070B504460078A8B90D46164641
:109830000AA0FEF749FF0DA03168FEF745FF0D486D
:109840006168FEF741FF28684FF0FF32401C286036
:109850003046616802F062FB002070BD5B466C61BF
:10986000736844425D5B6B765D0000005B25735D51
:1098700020000000881B01082DE9F0410646007811
:109880000D680C46012728B1707802280ED00128F7
:109890001DD02DE017A0FEF717FF1AA02968FEF7CC
:1098A00013FF1AA07168FEF70FFF0CE0686A401CF6
:1098B00018D010A0FEF708FF12A02968FEF704FFD9
:1098C0001D48FEF701FF27710120BDE8F081A06867
:1098D000401CA0607068E0608868012808D1686A50
:1098E000401C05D12822314605F12000F8F7C6FCBE
:1098F0000020EAE75B466C61736844425D5B747309
:109900006C5D00005B25735D20000000536563748F
:109910006F72202830782530387529206865616499
:10992000657220696E666F20697320696E636F725D
:10993000726563742E0A0000981D010870B51B4DF6
:109940000720FF21287300206873E974287515210A
:109950002846F9F701FA6875000AA875002014492D
:10996000A5220A54401C80B20828FAD300240A1900
:10997000285D641CA4B21072172CF8D321445A201D
:109980000C4D08724FF0FF31286805F05EFA09347B
:10999000A2B207490848FCF76DF8286805F03AFAC2
:1099A000BDE87040322005F0C7BB0000C1030020B5
:1099B000B0240020A40100202807002010B503F0E7
:1099C00061F9002010BD10B503F092F9002010BD20
:1099D0002DE9F04F8DB0054600208DF82C009B46F8
:1099E00092460F46169E10464C69F8F777FC2028E1
:1099F0000ED979A0FEF768FE7BA02968FEF764FE09
:109A000020217BA0FEF760FE05200DB0BDE8F08FA1
:109A1000FF22282101A8F8F743FC80480690504611
:109A2000F8F75CFCC0B28DF82400C01C20F00301E4
:109A3000F01C20F00300084428300A960790E968DB
:109A4000243988420BD964A0FEF73EFE66A029683F
:109A5000FEF73AFE72A0FEF737FE0720D5E7601C3E
:109A600007D139462846079A03F050FC0446401CAB
:109A70007ED00BAB39462846079A06F0E7FF5FEA2F
:109A8000000876D1FF208DF83000082209A90020B7
:109A900001F056FA08909DF82420514601F050FA42
:109AA00008909DF82400C11C21F003010E1A05E066
:109AB00001220CA9089801F043FA0890761EF7D20B
:109AC00059460A9A089801F03BFA08900A980A99B0
:109AD000C01C20F00300461A05E001220CA90898DA
:109AE00001F02EFA0890761EF7D201AE4FF0010970
:109AF0000623324621462846CDF80090FFF7BAF8F3
:109B00005FEA000808D1142306F1140204F11401DD
:109B10002846FEF76EFE8046B8F1000F5AD19DF838
:109B20002430524604F128012846FFF71BFD8046E9
:109B30009DF82C0078B99DF82400C01C20F003008B
:109B400001190A98C01C20F003000A182846283280
:109B5000796807F068F89DF8242023465146284686
:109B600006F026FFB8F1000F34D19DF8240001E083
:109B70002EE02FE0C01C20F0030001195A462846B1
:109B800028310A9BFFF7EEFC5FEA000822D1022091
:109B90000090062301AA21462846FFF76BF85FEAEA
:109BA000000817D19DF82C00A0B10BA0FEF78CFD8A
:109BB0000DA02968FEF788FD40F27A4220A127A077
:109BC000FEF782FD28A0FEF77FFD85F8289001E0D2
:109BD0004FF00708404618E75B466C6173684442E3
:109BE0005D5B6B765D0000005B25735D200000000F
:109BF0004572726F723A20546865204B56206E6130
:109C00006D65206C656E677468206973206D6F7276
:109C100065207468616E2025640A00004B56303060
:109C20004572726F723A20546865204B56207369F2
:109C30007A6520697320746F6F206269670A00007B
:109C40002E2E5C666C61736864625C7372635C6622
:109C500064625F6B7664622E630000002825733AAD
:109C6000256429200000000054726967676572202E
:109C70006120474320636865636B20616674657289
:109C80002063726561746564204B562E0A000000E3
:109C90002DE9F04395B01D4614008946074604D1CE
:109CA00006AA01F00BFF80B106AC2F4E002D21D08B
:109CB00004200090062301AA3846216BFEF7DAFF44
:109CC00031780546294320D032E028A0FEF7FCFC7D
:109CD0002AA03968FEF7F8FC40F25E3229A130A0D4
:109CE000FEF7F2FC494631A0FEF7EEFC052015B068
:109CF000BDE8F08303200090062301AA3846216BBB
:109D0000FEF7B8FF0546012013E0B9F100004FF05F
:109D1000FF3805D0F8F7E2FA02464346494604E028
:109D200034B1A278434604F11001384606F040FEF3
:109D300000203070F868246B401E84430C3485B9D1
:109D4000042301AA21463846FEF720FF012808D146
:109D500002200090042301AA21463846FEF78AFF1C
:109D600005462846C3E70000310000205B466C61D1
:109D7000736844425D5B6B765D0000005B25735D3C
:109D8000200000002E2E5C666C61736864625C7358
:109D900072635C6664625F6B7664622E63000000CF
:109DA0002825733A25642920000000004E6F742096
:109DB000666F756E64202725732720696E204B56C9
:109DC0002E0A000000256F1E064C012640F6B8380A
:109DD0003946E06905F039F82672404605F0ACF9DD
:109DE0002572F5E7B80200201CB505210620CDE953
:109DF00000014FF480730022064907A005F0D7F850
:109E000008490028486203D0BDE81C4005F0E0B9CD
:109E10001CBD0000C59D000864656C61795F6B65C1
:109E200079000000B8020020F0B500221949202373
:109E30008B54521CD2B21E2AFAD35C2543240D70D7
:109E4000154B4C7031228A701A7A42B100228F1859
:109E50009E5C521CD2B2FE700C2AF8D306E09E5CC7
:109E60008F18521CD2B2FE70082AF8D3CD740C752C
:109E700033224A751C220A23521ED2B2002808DD62
:109E800090FBF3F403FB140490FBF3F030348C5498
:109E9000F2E7F0BDA70400200429002070B50021DE
:109EA000124820224254491CC9B21E29FAD35C240C
:109EB000432304700E4A437031218170117A41B1FD
:109EC00000214618555C491CC9B2F5700C29F8D31D
:109ED00006E0555C4618491CC9B2F5700829F8D34C
:109EE000C47403753321417570BD0000A7040020C0
:109EF0000429002000B591B024220DA108A8F8F78C
:109F0000BDF902200021CDE904100690079022231C
:109F100096221E211A208DE80F0001230022242101
:109F200008A800F017F8322005F006F911B000BDBE
:109F30002020BFC6C5C8CCDA544D5257617463683F
:109F40002020C8ABBBECBACFC8D5C1B8BCE0BFD8E5
:109F5000CFB5CDB32DE9F05F0D460AA94C4C91E881
:109F6000C05F05F124012173090A6173E27423754E
:109F700005F11B016175090AA175267680236376B8
:109F80000022A776E27684F81C80637784F81E901E
:109F9000E27784F820A084F821B084F828C084F8FF
:109FA00029E0290A84F82E5084F82F1084F83020F4
:109FB00084F831203226114605E0425CA255761C19
:109FC000491CB6B289B2A942F7D331463048F8F7F6
:109FD000C3FEA055761CB1B2000A6054491C32354C
:109FE000A8B2A62602235B278AB201252AE0215CBB
:109FF000A52905D0A62903D05A2901D05B291FD154
:10A00000114607E004EB010C1CF801CC04F801C078
:10A01000491E89B28142F5D8215CA52906D0A6291E
:10A020000AD05A2904D05B2906D007E0265400E064
:10A03000275421184B7001E021184D70521C92B228
:10A04000401E80B20028D2D11249A5230B54401CD7
:10A0500080B20828FAD3002504E0605D4B196D1C1E
:10A060001872ADB29542F8D329445A200A4C0872AE
:10A070004FF0FF31206804F0E8FE0935AAB2054927
:10A080000648FBF7F7FC2068BDE8F05F04F0C2BEAD
:10A09000C1030020B0240020A401002028070020D4
:10A0A00010B50020264920220A54401CC0B21E28A8
:10A0B000FAD35C20087043204870224A322088700E
:10A0C00013780320D62B0DD0202B08D01E4B1C1844
:10A0D00014F8034C0C54401CC0B20928F7D3137A6F
:10A0E00083B918E05378B42BF0D19378D02BEDD10D
:10A0F000D378D02BEAD110BD131813F8093C0B54B8
:10A10000401CC0B21528F7D307E0131813F8093C18
:10A110000B54401CC0B21128F7D30C4819220A2353
:10A12000B0F900000028E6DD90FBF3F403FB140413
:10A1300090FBF3F0521ED2B230348C54F2E70000A0
:10A14000C5040020DC280020E615010820030020BB
:10A150002DE9F043B1B008AC9C21201DF8F7A7F819
:10A1600047480021006808904648425C6254491CF8
:10A17000C9B21929F9D3434919201E310A1812F816
:10A18000192C2254401CC0B23528F7D33D49672012
:10A190003C310A1812F8672C2254401CC0B28028A7
:10A1A000F7D34FF0430C8DF864C031208DF8650073
:10A1B0005C26354B35488DF863601B78077846215F
:10A1C000DFF8CC90072243EA07054FF020081DB1C5
:10A1D00019F80200605401E004F80180491CC9B27A
:10A1E000521EF4D56654491CC8B2332104F800C08D
:10A1F000401CC0B2224A2154401CC1B20020121D92
:10A2000001EB000C155C401CC0B204F80C50062891
:10A21000F6D3204867250268110000D5494279B17C
:10A220000A2000290FDD91FBF0FC00FB1C1C91FBB8
:10A23000F0F16D1EEDB20CF1300C04F805C0F0E742
:10A2400030208DF88600002A02DA2D208DF880005B
:10A250000BB9012F11D102200021CDE90410069085
:10A2600008220790B021CDE90020CDE90216012394
:10A270000022802108A8FFF76DFE31B0BDE8F08311
:10A28000DC15010889040020B9020020000000202C
:10A29000400200209802002010B500210B4A202324
:10A2A0005354491CC9B21E29FAD35C2111704321B1
:10A2B000517033219170002807D1054914180B5CA7
:10A2C000401CC0B2E3700E28F8D310BD89040020F2
:10A2D000F7020020F0B50446007893B00D46002840
:10A2E00057D0A078022801D0032852D10320009033
:10A2F000616804230FAA28460C31FEF7BBFC606896
:10A3000040F2F937243005AE0D9001A9284603F03C
:10A31000D1FD9DF8050000281DD09DF804000228FD
:10A3200001D0032817D101A9284602F037FE0028E2
:10A3300011D019A0FEF7C8F91BA02968FEF7C4F9CF
:10A340003A461BA121A0FEF7BFF99DF80610324640
:10A3500021A0FEF7B9F901AA2146284602F032FAF7
:10A360000D90401CD1D1421E2846616801F0D6FDF7
:10A3700009A0FEF7A9F90CA02968FEF7A5F940F29B
:10A38000FE320BA111A0FEF79FF91EA06168FEF737
:10A390009BF913B00020F0BD5B466C6173684442CA
:10A3A0005D5B6B765D0000005B25735D2000000047
:10A3B0002E2E5C666C61736864625C7372635C66AB
:10A3C00064625F6B7664622E630000002825733A36
:10A3D00025642920000000004572726F723A204DFA
:10A3E0006F76656420746865204B562028252E2AD8
:10A3F000732920666F72204743206661696C65642B
:10A400002E0A0000436F6C6C6563742061207365D5
:10A4100063746F7220403078253038580A0000008D
:10A4200070B50D46144600212B226254491CC9B256
:10A430000329FAD34FF0FF3104F007FD21462846E7
:10A44000BDE870400322FBF715BBF0B500F10067D3
:10A4500085B000200E46CD0A0490490500D06D1C41
:10A46000009001200390FAF725FB00240EE007EB93
:10A47000C420029004A96846FAF77EFA28B1FAF7D8
:10A48000CFFA4FF0FF3005B0F0BD641CAC42EED304
:10A49000FAF7C6FA3046F6E710B50E49097841B129
:10A4A00070B10D4C18222168F7F72DFF78B100200C
:10A4B00010BD094A09A113320AA0FEF705F9FEE70B
:10A4C000054A10A1133207A0FEF7FEF8FEE7206848
:10A4D00010BD0000210000205C0F0108696E697446
:10A4E0005F6F6B0028257329206861732061737387
:10A4F000657274206661696C6564206174202573DF
:10A500002E0A00006E616D65000000003EB51F4D13
:10A51000287808B100203EBD1D480468A16AF9B141
:10A52000E16A002923D0216B002927D0606A00B19D
:10A53000804717493F22091D16A0FEF7C5F804F110
:10A540001800234607C88DE8070018221146164850
:10A55000FEF7BAF815A0FEF7B7F801202870D9E782
:10A560000B4A13A1121D19A0FEF7AEF8FEE7084A28
:10A570001EA1121D15A0FEF7A7F8FEE7044A22A1AE
:10A58000121D12A0FEF7A0F8FEE700002100002037
:10A590005C0F01085B442F46414C5D202825733A2F
:10A5A0002564292000000000F81901080A000000B5
:10A5B0006465766963655F7461626C655B695D2D76
:10A5C0003E6F70732E726561640000002825732948
:10A5D0002068617320617373657274206661696CB1
:10A5E00065642061742025732E0A00006465766915
:10A5F00063655F7461626C655B695D2D3E6F70734E
:10A600002E777269746500006465766963655F74AE
:10A6100061626C655B695D2D3E6F70732E65726162
:10A620007365000070B5FFF771FF114D04000ED483
:10A6300000F05AF9041E0ADD2878002815D10120FF
:10A6400028700CA0FEF740F80FA111A008E0002030
:10A6500028703E221B491CA0FEF736F80AA121A053
:10A66000FEF732F82CA0FEF72FF8204670BD000050
:10A67000200000201B5B33323B32326D5B492F469A
:10A68000414C5D2000000000302E352E30000000CF
:10A69000466C617368204162737472616374696FA0
:10A6A0006E204C6179657220285625732920696EC9
:10A6B000697469616C697A65207375636365737326
:10A6C0002E000000500F01081B5B33313B32326D0E
:10A6D0005B452F46414C5D202825733A256429208F
:10A6E00000000000466C61736820416273747261FF
:10A6F0006374696F6E204C617965722028562573EA
:10A700002920696E697469616C697A65206661697E
:10A710006C65642E000000001B5B306D0A000000B9
:10A720002DE9F04116460D4604000FD0A16BA81983
:10A730004FF0FF3788420FD94FF4E7721D491EA032
:10A74000FDF7C2FF23A0FDF7BFFF2EE0194A2FA19E
:10A7500030A0FDF7B9FFFEE704F11C008046FFF7CB
:10A760009BFEB8B1616B026B4B193146184690479E
:10A7700004000CD54FF4EE720E490FA0FDF7A4FFB4
:10A7800041462CA0FDF7A0FF38A0FDF79DFF204615
:10A79000BDE8F08140F2D512064907A0FDF794FF0D
:10A7A000221D41463348FDF78FFF30A0FDF78CFF97
:10A7B0003846EDE7071001081B5B33313B32326D41
:10A7C0005B452F46414C5D202825733A256429209E
:10A7D00000000000506172746974696F6E206572C8
:10A7E000617365206572726F7221205061727469A5
:10A7F00074696F6E2061646472657373206F757421
:10A80000206F6620626F756E642E00007061727436
:10A81000000000002825732920686173206173738C
:10A82000657274206661696C6564206174202573AB
:10A830002E0A0000506172746974696F6E2065722F
:10A84000617365206572726F722120466C61736856
:10A8500020646576696365282573292065726173B4
:10A8600065206572726F7221000000001B5B306D05
:10A870000A0000003C1B010870B50F4D0646287801
:10A8800008B100240EE00D4A0DA10FA0FDF71CFF3A
:10A89000FEE7686800EB84113046091DF7F725FDD7
:10A8A00028B1641CA8688442F3D3002070BD686896
:10A8B00000EB841070BD000024000020980F0108F8
:10A8C000696E69745F6F6B00282573292068617356
:10A8D00020617373657274206661696C65642061C0
:10A8E000742025732E0A00002DE9F041244C2078B5
:10A8F00010B1A068BDE8F081224860600620002504
:10A900004FF48876A060606800EB85101C30FFF77C
:10A91000C3FD07001BD06068F96900EB8510406B30
:10A92000884223DB4FF48B72174918A0FDF7CCFE49
:10A930006068FB6900EB85111B484A6B091DFDF738
:10A94000C3FE1AA0FDF7C0FE0020A06014E032464E
:10A950000D4918A0FDF7B8FE606800EB85111AA03C
:10A960001C31FDF7B1FE12A0FDF7AEFEA0686D1C14
:10A970008542C8D30120207000F0AEF9B9E700008D
:10A9800024000020401F0108850F01081B5B3331A4
:10A990003B32326D5B452F46414C5D202825733A92
:10A9A0002564292000000000541A01081B5B306D4B
:10A9B0000A0000005B442F46414C5D202825733A75
:10A9C00025642920000000005761726E696E673AA5
:10A9D00020446F204E4F5420666F756E642074685B
:10A9E0006520666C617368206465766963652825F7
:10A9F00073292E002DE9F0471E4690460D460400AF
:10AA000012D0B8F1000F15D0A16BA8194FF0FF3785
:10AA1000884215D94FF4BF72214922A0FDF754FE98
:10AA200027A0FDF751FE35E01D4A33A134A0FDF704
:10AA30004BFEFEE71A4A3AA131A0FDF745FEFEE7BC
:10AA400004F11C008146FFF727FDC0B1616B846AE9
:10AA50004B19324641461846A04704000CD54FF426
:10AA6000C6720F490FA0FDF72FFE49462DA0FDF736
:10AA70002BFE39A0FDF728FE2046BDE8F08740F206
:10AA80008512074907A0FDF71FFE221D49463448DD
:10AA9000FDF71AFE30A0FDF717FE3846EDE700007F
:10AAA000E00F01081B5B33313B32326D5B452F46B3
:10AAB000414C5D202825733A2564292000000000C0
:10AAC000506172746974696F6E207265616420658B
:10AAD00072726F722120506172746974696F6E2096
:10AAE00061646472657373206F7574206F66206291
:10AAF0006F756E642E0000007061727400000000BB
:10AB0000282573292068617320617373657274202E
:10AB10006661696C65642061742025732E0A0000EB
:10AB200062756600506172746974696F6E20726537
:10AB30006164206572726F722120466C61736820B7
:10AB400064657669636528257329207265616420D0
:10AB50006572726F722100001B5B306D0A0000008D
:10AB6000F01A01082DE9F0471E4690460D460400F4
:10AB700012D0B8F1000F15D0A16BA8194FF0FF3714
:10AB8000884215D940F2A712214922A0FDF79CFD69
:10AB900027A0FDF799FD35E01D4A33A134A0FDF74C
:10ABA00093FDFEE71A4A3AA131A0FDF78DFDFEE7BD
:10ABB00004F11C008146FFF76FFCC0B1616BC46AF1
:10ABC0004B19324641461846A04704000CD540F2C6
:10ABD000B5120F490FA0FDF777FD49462DA0FDF7EF
:10ABE00073FD3AA0FDF770FD2046BDE8F0874FF4F5
:10ABF000D772074907A0FDF767FD221D4946354872
:10AC0000FDF762FD31A0FDF75FFD3846EDE700007E
:10AC1000F30F01081B5B33313B32326D5B452F462E
:10AC2000414C5D202825733A25642920000000004E
:10AC3000506172746974696F6E20777269746520EF
:10AC40006572726F722120506172746974696F6EDF
:10AC50002061646472657373206F7574206F662061
:10AC6000626F756E642E00007061727400000000E7
:10AC700028257329206861732061737365727420BD
:10AC80006661696C65642061742025732E0A00007A
:10AC900062756600506172746974696F6E207772B4
:10ACA000697465206572726F722120466C617368E9
:10ACB0002064657669636528257329207772697435
:10ACC00065206572726F7221000000001B5B306DA1
:10ACD0000A000000A41A01082DE9F04786B00FF21F
:10ACE000F00A0FF2F4085046F7F7F8FA81464046AA
:10ACF000F7F7F4FA3B4C0546A068E0B1002617E0F0
:10AD0000606800EB8617381DF7F7E8FA484503D965
:10AD1000381DF7F7E3FA814607F11C000746F7F7FD
:10AD2000DDFAA84203D93846F7F7D8FA0546761C6B
:10AD3000A0688642E4D32CA0FDF7C6FC2FA0FDF747
:10AD4000C3FC3EA0FDF7C0FC27A0FDF7BDFC182604
:10AD50008DE860015346324649463AA0FDF7B4FCFF
:10AD600036A0FDF7B1FC20A0FDF7AEFC41A0FDF739
:10AD7000ABFC32A0FDF7A8FC0027B04618E06068E5
:10AD800000EB871618A0FDF79FFCD6E90D0106F130
:10AD90001C02CDE90220CDE900580491331D182290
:10ADA000494644A0FDF790FC24A0FDF78DFC7F1CD4
:10ADB000A0688742E3D30CA0FDF786FC47A0FDF70F
:10ADC00083FC06B01DA0BDE8F047FDF77DBC000088
:10ADD0006E616D6500000000666C6173685F64659C
:10ADE00076000000240000201B5B33323B32326DC2
:10ADF0005B492F46414C5D20000000003D3D3D3D3C
:10AE00003D3D3D3D3D3D3D3D3D3D3D3D3D3D3D3D72
:10AE10002046414C20706172746974696F6E2074B1
:10AE200061626C65203D3D3D3D3D3D3D3D3D3D3DCF
:10AE30003D3D3D3D3D3D3D3D3D0000001B5B306DDA
:10AE40000A0000007C20252D2A2E2A73207C202534
:10AE50002D2A2E2A73207C2020206F66667365744D
:10AE60002020207C202020206C656E6774682020C4
:10AE70007C0000002D2D2D2D2D2D2D2D2D2D2D2D3A
:10AE80002D2D2D2D2D2D2D2D2D2D2D2D2D2D2D2DF2
:10AE90002D2D2D2D2D2D2D2D2D2D2D2D2D2D2D2DE2
:10AEA0002D2D2D2D2D2D2D2D2D2D2D2D2D2D2D2DD2
:10AEB0002D0000007C20252D2A2E2A73207C2025A1
:10AEC0002D2A2E2A73207C2030782530386C78206B
:10AED0007C20307825303878207C00003D3D3D3D99
:10AEE0003D3D3D3D3D3D3D3D3D3D3D3D3D3D3D3D92
:10AEF0003D3D3D3D3D3D3D3D3D3D3D3D3D3D3D3D82
:10AF00003D3D3D3D3D3D3D3D3D3D3D3D3D3D3D3D71
:10AF10003D3D3D3D3D3D3D3D3D000000C0E9001251
:10AF2000704770B505464C680869A04200D20446D7
:10AF30000A68C96823462846FDF754FC204670BDC0
:10AF400010B5C043064B07E011F8014B4440E4B292
:10AF500053F8244084EA1020521EF5D2C04310BD9D
:10AF6000B81001082DE9F0410546007C8EB014466A
:10AF70008846B0B1696909B128468847414654F806
:10AF8000048B002654F80C7B6A46284600F096FD98
:10AF900008B30CB1039820600398B84210D206465B
:10AFA0000FE011A0FDF790FB13A02968FDF78CFBC3
:10AFB00013A02968FDF788FB00200EB0BDE8F081E2
:10AFC0003E46B8F1000009D00246334628460D99A6
:10AFD000FDF708FC02E00CB100202060A96909B16E
:10AFE000284688473046E8E75B466C617368444210
:10AFF0005D5B6B765D0000005B25735D20000000EB
:10B000004572726F723A204B5620282573292069A9
:10B01000736E277420696E697469616C697A652042
:10B020004F4B2E0A0000000070B50446007C154608
:10B030000E4680B162690AB120469047D5E90023E7
:10B040003146204605F0FEF8A169054609B12046C3
:10B050008847284670BD06A0FDF736FB08A021688A
:10B06000FDF732FB08A02168FDF72EFB082070BD1C
:10B070005B466C61736844425D5B6B765D0000000B
:10B080005B25735D200000004572726F723A204BA1
:10B090005620282573292069736E277420696E69EC
:10B0A0007469616C697A65204F4B2E0A00000000BC
:10B0B0002DE9F047416988B00446002601B1884770
:10B0C00000254FF0FF3908E04A462946204600F0A7
:10B0D00025FF060029D1E0680544A068806BA842DE
:10B0E000F2D800254FF0080A4FF004081AE000BF1C
:10B0F00005EB4507216A0AEB8700085820B908EBE1
:10B1000087000858F7F7EAF8CDF818900090206A01
:10B1100008EB8701435850F8272001A92046FEF785
:10B1200057FC6D1C606AA842E2D8A16909B12046AB
:10B13000884708B03046BDE8F087000010B504002D
:10B1400009D000291AD0012931D0022932D003298F
:10B1500000D1826110BD18A0FDF7B6FA1AA02168CF
:10B16000FDF7B2FA40F2FB5219A120A0FDF7ACFAAC
:10B17000214A22A122A0FDF7A7FAFEE7207C0028A1
:10B1800012D00DA0FDF7A0FA0FA02168FDF79CFAE0
:10B190004FF4C0620EA115A0FDF796FA164A20A141
:10B1A00017A0FDF791FAFEE71068E06010BDC068D7
:10B1B000106010BD426110BD5B466C617368444213
:10B1C0005D5B6B765D0000005B25735D2000000019
:10B1D0002E2E5C666C61736864625C7372635C667D
:10B1E00064625F6B7664622E630000002825733A08
:10B1F00025642920000000004F100108646200004F
:10B200002825732920686173206173736572742027
:10B210006661696C65642061742025732E0A0000E4
:10B2200064622D3E706172656E742E696E69745F22
:10B230006F6B203D3D2066616C736500F8B5044678
:10B2400006981E0007D0009000232046FDF7EAFA7A
:10B2500005007DD112E04BA0FDF736FA4DA0216824
:10B26000FDF732FA40F223624CA153A0FDF72CFA0D
:10B27000544A55A157A0FDF727FAFEE7002084F8AD
:10B28000280084F82900D6E90001C4E90801A06873
:10B29000816BE068B1FBF0F2012A12D839A0FDF70A
:10B2A00013FA3CA02168FDF70FFA4FF4C6623BA1E8
:10B2B00041A0FDF709FA434A4E4946A0FDF704FABA
:10B2C000FEE7B1FBF0F200FB1212002A12D02DA013
:10B2D000FDF7FAF92FA02168FDF7F6F940F2326286
:10B2E0002EA135A0FDF7F0F9364A43A139A0FDF7AC
:10B2F000EBF9FEE7B1FBF0F0022812D221A0FDF736
:10B30000E3F924A02168FDF7DFF940F2346223A1BC
:10B3100029A0FDF7D9F92B4A41A12EA0FDF7D4F9B8
:10B32000FEE70020B0F1010104EBC002401CC2F8AE
:10B33000AC100428F8D3002004EBC002401C1163B9
:10B340001028F9D30FA0FDF7BFF912A0216800E083
:10B3500011E0FDF7B9F940F23F6210A116A0FDF728
:10B36000B3F9A16838A08A6B091DFDF7ADF9204635
:10B37000FDF792FB054601462046FDF725FB2846D2
:10B38000F8BD00005B466C61736844425D5B6B76A0
:10B390005D0000005B25735D200000002E2E5C66C2
:10B3A0006C61736864625C7372635C6664625F6B39
:10B3B0007664622E630000002825733A25642920F4
:10B3C000000000006010010864656661756C745FC0
:10B3D0006B760000282573292068617320617373E0
:10B3E000657274206661696C6564206174202573E0
:10B3F0002E0A0000B41C010864625F706172745F01
:10B4000073697A652864622920252064625F736508
:10B41000635F73697A6528646229203D3D203000AE
:10B4200064625F706172745F73697A65286462290F
:10B43000202F2064625F7365635F73697A65286497
:10B440006229203E3D2032004B56444220696E2046
:10B45000706172746974696F6E2025732C20736932
:10B460007A652069732025752062797465732E0AC8
:10B470000000000010B5040007D0072930D2DFE833
:10B4800001F017303234363A3E001EA0FDF71CF9A9
:10B4900020A02168FDF718F940F29E221FA126A0E6
:10B4A000FDF712F9274A28A128A0FDF70DF9FEE7BC
:10B4B000207C002812D013A0FDF706F915A0216802
:10B4C000FDF702F940F2A32214A11BA0FDF7FCF83E
:10B4D0001C4A26A11DA0FDF7F7F8FEE71068E06002
:10B4E00010BDE0680CE0626110BDA26110BD107873
:10B4F00084F8580010BD94F85800107010BDA06C6E
:10B50000106010BD5B466C61736844425D5B747390
:10B510006C5D00005B25735D200000002E2E5C66D4
:10B520006C61736864625C7372635C6664625F74AE
:10B530007364622E630000002825733A2564292075
:10B54000000000009810010864620000282573299B
:10B550002068617320617373657274206661696C21
:10B5600065642061742025732E0A000064622D3EFC
:10B57000706172656E742E696E69745F6F6B203DC9
:10B580003D2066616C7365002DE9F0419CB01D00A3
:10B59000DDE922734FF000080446CDF81080CDF8A5
:10B5A0001480CDF81880039007D000930123204623
:10B5B000FDF738F9060078D112E061A0FDF784F8B4
:10B5C00063A02168FDF780F840F2CD2262A169A056
:10B5D000FDF77AF86A4A6BA16DA0FDF775F8FEE7F2
:10B5E000C4E91357012184F85810881E6065606211
:10B5F000A068826BE068B2FBF0F300FB1323002B22
:10B6000012D04FA0FDF760F851A02168FDF75CF85B
:10B6100040F2DB2250A157A0FDF756F8584A64A12A
:10B620005BA0FDF751F8FEE7B2FBF0F2022A12D25E
:10B6300043A0FDF749F846A02168FDF745F840F220
:10B64000DD2245A14BA0FDF73FF84D4A62A150A075
:10B65000FDF73AF8FEE7B84212D839A0FDF734F802
:10B660003BA02168FDF730F840F2DF223AA141A06B
:10B67000FDF72AF8424A62A145A0FDF725F8FEE74A
:10B680006648CDF82080CDF80080CDE9010145461F
:10B6900003AB002207A9204603F0C9FF9DF8100064
:10B6A00020B1204605F03EF90EE040E0059808B1D3
:10B6B000069800E0606AE1680844A168896B8842E6
:10B6C00001D3656500E060651DA0FCF7FDFF20A0CB
:10B6D0002168FCF7F9FF40F2F6221FA125A0FCF734
:10B6E000F3FF4F48636A626D2168FCF7EDFF0123A9
:10B6F00004F120022046616A02F0E6FD94F8210080
:10B70000022802D0012802D011E0206B0EE0616D0A
:10B71000606A81420BD008B9A068806BE1680023A1
:10B72000411A12AA204602F0CFFD1698A0643146B5
:10B730002046FDF749F91CB03046BDE8F081000015
:10B740005B466C61736844425D5B74736C5D0000C2
:10B750005B25735D200000002E2E5C666C617368B3
:10B7600064625C7372635C6664625F747364622EAD
:10B77000630000002825733A25642920000000009A
:10B78000A91001086765745F74696D6500000000A9
:10B790002825732920686173206173736572742092
:10B7A0006661696C65642061742025732E0A00004F
:10B7B00064625F706172745F73697A65286462297C
:10B7C00020252064625F7365635F73697A6528640E
:10B7D0006229203D3D20300064625F706172745FB9
:10B7E00073697A6528646229202F2064625F73651B
:10B7F000635F73697A6528646229203E3D203200C8
:10B800006D61785F6C656E203C2064625F73656378
:10B810005F73697A652864622900000079980008DE
:10B82000501D010870B50446007C0D4670B1626978
:10B830000AB1204690472946204604F0D7FFA16967
:10B84000054609B120468847284670BD06A0FCF78A
:10B850003BFF09A02168FCF737FF09A02168FCF72E
:10B8600033FF082070BD00005B466C617368444282
:10B870005D5B74736C5D00005B25735D20000000F0
:10B880004572726F723A2054534C20282573292038
:10B8900069736E277420696E697469616C697A6571
:10B8A000204F4B2E0A00000010B54169044601B13B
:10B8B0008847204605F036F8A169002903D02046C4
:10B8C000BDE81040084710BD2DE9FF4F0546D0F8F0
:10B8D00054904FF0000A007C8FB09B460E46D04635
:10B8E00050B93AA0FCF7F0FE3CA02968FCF7ECFE4A
:10B8F0003CA02968FCF7E8FEBBF1000F19D04C46CC
:10B90000002305AA2146284602F0DEFC48B99DF82E
:10B910001500022810D0032814D0012809D0E968A6
:10B920008A44524605A9284600F08CFF0446401C74
:10B93000E6D113B0BDE8F08F282205F1200105A85B
:10B94000F6F79CFCB8F1000F0AD10898B04202D873
:10B950000998B04204D24C45E1D10898B042DED3F8
:10B96000069C4FF0010850340A9F13E0391B012058
:10B9700000EB510020F01F00204403906946284648
:10B9800002F0A8FD0198B04202D2039C203401E0ED
:10B99000039F203FBC42E9D903946946284602F040
:10B9A00099FD0198B042C4D3014611988142C0D894
:10B9B00068465A461C9990470028BAD1694605A89E
:10B9C00000F050FF0390401CE7D1A8E75B466C6194
:10B9D000736844425D5B74736C5D00005B25735D4E
:10B9E000200000004572726F723A2054534C202898
:10B9F0002573292069736E277420696E69746961E3
:10BA00006C697A65204F4B2E0A0000000269CA60FB
:10BA1000C2688A608068086108467047074808B5B0
:10BA2000426A0021322A02D9A2F13200C1B204488E
:10BA3000044B0090FFF748FF08BD000034000020D1
:10BA4000DC0B002059D8000808B5054800900648CE
:10BA5000044B4FF0FF32016A0148FFF735FF08BD84
:10BA60007C0B00202DD900083400002008B50548C3
:10BA700000900648044B4FF0FF32016A0148FFF77F
:10BA800023FF08BD7C0B002091D900083400002062
:10BA900038B5074C0020084B206406480090616AC6
:10BAA0004FF0FF32491CFFF70FFF206C38BD00003C
:10BAB00034000020DC0B0020E5D700082DE9F04120
:10BAC000074614460E460846F6F708FC804602462E
:10BAD00004F130033146384600F03CFE30B12146D7
:10BAE000384602F0E7F90120BDE8F08122463146F0
:10BAF000384600F025F8050005D042463146384664
:10BB0000236B04F055FF2846EEE770B504460D465A
:10BB100016460846F6F7E2FB0246A07890420AD1A4
:10BB2000607840B12078022805D1294604F1100040
:10BB3000F6F7E9FB08B1002070BD0120307070BD40
:10BB40001CB5144600228DF80420054A00920A46CE
:10BB500001AB214600F0D0FF9DF804001CBD0000A1
:10BB60000BBB00082DE9F0478146C0680C460D4626
:10BB7000401E8AB01646814308AA484600F088FE57
:10BB80004FF0FF3770B30898844231D02AE0202369
:10BB90006A4621464846FCF725FE00206B46DFF842
:10BBA00054A01BE0191813F800C091F801800CEBA9
:10BBB000082C91F80280C9784FEA084808EB016127
:10BBC0006144514507D1143AAA4204D320441438A1
:10BBD0000AB0BDE8F087401C1C2802D22218B242ED
:10BBE000E0D31C34B44203D204F12000B042CED3DF
:10BBF0003846EDE74B56303038B5064C4FF0FF3243
:10BC00000548A2630090054B216AFFF75DFEA06B1B
:10BC100038BD0000340000207C0B0020F5D900085E
:10BC200038B5064C0020074BE063054800904FF004
:10BC3000FF32616AFFF748FEE06B38BD3400002038
:10BC4000DC0B002059DA000838B5194C00252222F7
:10BC50006564A06AA0642946164802F07FFF164872
:10BC60000090164B6A1EA16AFFF72EFE606C032837
:10BC70001DD910492222124B0A707E224A702022BE
:10BC80008A706278CA70F0220A711A7881F82120CD
:10BC9000521C1A7001228B5C521C2B44DDB2222AEA
:10BCA000F9DBC5F1FF0281F82220A16CA16238BD49
:10BCB00034000020DC2600203C0C0020A5DA00081F
:10BCC000BD0200200349496911F8292F60F34102A0
:10BCD0000A707047E4040020014AC2E9000170477D
:10BCE000E40400207CB514491448FFF7F5FF8021D7
:10BCF000012002F059FC124C6061C8B106200A21F3
:10BD0000CDE90001C30100220E490FA003F04FF955
:10BD1000054600231A460EA1606903F069F8012068
:10BD2000FFF7D0FF15B1284603F052FA00207CBD82
:10BD30004FF0FF307CBD0000401F0108C01E01080D
:10BD4000E404002059BD0008747368656C6C000041
:10BD500073687278000000006B4E0027706910F85D
:10BD6000291F41F00101017002F082FD0500FBD4A2
:10BD70001B2D07D0746994F82800012807D00228E9
:10BD80000ED017E07169012081F82800ECE75B2DE7
:10BD900002D084F828700DE0022084F82800E3E740
:10BDA00084F82870412DDFD0422DDDD0442D2ED0D7
:10BDB000432D32D0002DD7D0FF2DD5D0092D36D030
:10BDC0007F2D4CD0082D4AD00D2D73D00A2D71D067
:10BDD000B4F87A00502801D3A4F87A70B4F87C0043
:10BDE000B4F87A1088427BD20A1A04F12A0101447D
:10BDF0002B34204402F098FE7069B0F87C102A3091
:10BE00000D547169B1F87C00B1F87A1065E0B4F8AE
:10BE10007C000028A8D0401E06E0B4F87C00B4F8EE
:10BE20007A108842A0D2401CA4F87C009CE7002035
:10BE3000B4F87C1000E0401C8142FCDC2A3401F0A4
:10BE40000DFA012802D1204601F080F970692A30EC
:10BE5000F6F744FA716921F87A0F488084E7B4F85C
:10BE60007C00002880D0B4F87A10401E491E89B2A8
:10BE700080B2A4F87A10A4F87C00814217D90A1A7B
:10BE800004F12B0101442A34204402F04DFE706974
:10BE9000B0F87A102A300F547169B1F87C00B1F80B
:10BEA0007A1000E0401C8142C0DBFBE702E02A344C
:10BEB0000F5559E701F0D2F9012805D17069B0F8A2
:10BEC0007A102A3001F092F9706950212A30F6F781
:10BED000EEF9706914E003E0401C8142FCDC01E0F3
:10BEE0002A340D557069B0F87A10491C89B2A0F84F
:10BEF0007A10B0F87C20521CA0F87C20502995D3F1
:10BF000020F87A7F47802FE7E404002010B502462E
:10BF10000846516800F08CF8002010BDF0B51746B7
:10BF2000C2680446B1FBF2F00E4602FB106089B015
:10BF3000002812D01DA0FCF7C7FB20A02168FCF749
:10BF4000C3FB40F2CA221FA125A0FCF7BDFB274A74
:10BF500027A12EA0FCF7B8FBFEE72046FCF738FC33
:10BF6000050020D1FF2224216846F6F799F9012225
:10BF700004216846FCF768FE0122042103A8FCF7AF
:10BF800063FE2A48CDE90607681E089024236A4606
:10BF900031462046FCF72DFC0546E0683146821903
:10BFA000204604F040FE09B02846F0BD5B466C61B7
:10BFB000736844425D5B6B765D0000005B25735DDA
:10BFC000200000002E2E5C666C61736864625C73F6
:10BFD00072635C6664625F6B7664622E630000006D
:10BFE0002825733A2564292000000000411001082B
:10BFF0006164647220252064625F7365635F7369A6
:10C000007A6528646229203D3D2030002825732967
:10C010002068617320617373657274206661696C56
:10C0200065642061742025732E0A00004644423066
:10C0300030B5C2680546B1FBF2F00C4602FB104079
:10C0400095B0002811D016A0FCF73EFB18A0296877
:10C05000FCF73AFBE62218A11EA0FCF735FB204AAC
:10C0600020A127A0FCF730FBFEE72846FCF7B0FB39
:10C07000002812D101200090042301AA214628465D
:10C08000FCF7F8FD002808D125480490042304AAF1
:10C0900004F10C012846FCF7ACFB15B030BD0000E4
:10C0A0005B466C61736844425D5B74736C5D000059
:10C0B0005B25735D200000002E2E5C666C6173684A
:10C0C00064625C7372635C6664625F747364622E44
:10C0D000630000002825733A256429200000000031
:10C0E0007F1001086164647220252064625F7365BB
:10C0F000635F73697A6528646229203D3D203000C2
:10C100002825732920686173206173736572742018
:10C110006661696C65642061742025732E0A0000D5
:10C1200054534C3010B504460A2802D10D2001F0BA
:10C130004FFBE0B201F04CFB204610BD10B50028CB
:10C1400021D0114B0022001F196803E0814203D85F
:10C150000A4649680029F9D152B11368841A9C42F1
:10C1600004D1006818441060104602E0506000E0FE
:10C17000186039B102680B1A934203D10B681A4454
:10C1800002604968416010BD900500202DE9F04132
:10C19000154CE07AF6F716FB0546E069F6F712FB58
:10C1A0002946F6F749F91149F6F714F90546606B87
:10C1B0000746F6F707FB0646206BF6F703FB31460A
:10C1C000F6F702F901462846F6F736F9A064384634
:10C1D000FDF730F9A062E0632062E0622064A063B2
:10C1E0000120E074BDE8F081280300200000204118
:10C1F000007810B10868401C0860002070470000FB
:10C2000030B58BB00446002516480995CDE900509D
:10C2100009AB012203A92046029503F0DBF912A025
:10C22000FCF752FA14A02168FCF74EFA40F21242D1
:10C2300013A11AA0FCF748FA01221BA00999FCF7E8
:10C2400043FA0998012809D824482346CDE900502B
:10C25000002203A91846029503F0BCF984F828507F
:10C260000BB030BDF1C100085B466C61736844429D
:10C270005D5B6B765D0000005B25735D2000000058
:10C280002E2E5C666C61736864625C7372635C66BC
:10C2900064625F6B7664622E630000002825733A47
:10C2A00025642920000000005468652072656D61D6
:10C2B000696E20656D70747920736563746F722088
:10C2C00069732025752C2047432074687265736854
:10C2D0006F6C642069732025642E0A00D5A20008C3
:10C2E0002DE9F05F964C4FF0FF31606802F0ADFD34
:10C2F0006B2004F063FA18BB9248007800B3012069
:10C30000E07028222021904802F028FC8F488E4BB4
:10C31000202107888A488E4D0A224FF0EB091830F9
:10C320008FB1C7261E7083F80190BD269E70C1266E
:10C33000DE70B0261E71E8265E719971D9711DE01C
:10C34000E078401CDCE7834E3678EEBB94F803C0FF
:10C35000DFF804B200264FF03E0E9A465FEACC7337
:10C3600004D1052E02DD0AF806E003E01BF8068082
:10C370000AF80680761C082EF0DB2FB380F80090B8
:10C38000C32343708170C170017141718171C171AA
:10C39000724BA978C1F3C3011B88C1EB0111C3EB38
:10C3A00081010223616103E0022B01DD91FBF2F1C7
:10C3B0004D000DD091FBF2F502FB1515002D00DAB2
:10C3C0006D423035C55400E004E05B1C082BEBDB0C
:10C3D0006161B0E0624B644E1F78624B77B194F8B4
:10C3E00001C0BCF1000F09D195F803C0BCF1FE0FEC
:10C3F00004D096F800C0BCF1010F0BD01B6863613C
:10C400000023C1545B1C082BFBDB302387B167780A
:10C4100047B10DE0DFF854C11B68BCF900C0A3EBC5
:10C420000C03ECE7EF78FE2F02D03778012F08D00D
:10C430006769002F19DA4FF02D0C80F806C0C17122
:10C4400017E06169002904DC2F783F0604D5002934
:10C4500006DB2978090603D5D9278771C92702E0A9
:10C46000E0278771B627C77101E08171C1716169E9
:10C4700011B10027616905E0037036E0002F01DD8E
:10C4800091FBF2F15FEA410C0FD091FBF2FC02FB51
:10C490001C1CBCF1000F01DACCF1000C0CF1300CCB
:10C4A00000F807C07F1C082FE8DB616130490A787B
:10C4B000DAB1042107E0475C202F03D000EB010C28
:10C4C0008CF80170491E9142F5DA2E2181548118B1
:10C4D0004F78202F00D14B70002104E0475C202FC3
:10C4E00000D14354491C9142F8DB317819BBA9783B
:10C4F000090620D51F49F822CB230978012906D047
:10C50000062904D0032902D0042905D013E081793B
:10C5100041718271C3710EE0BC210170CA2141706A
:10C52000AA218170BF21C170CF210171C821417141
:10C53000B7228271C1716068BDE8F05F02F06ABC29
:10C5400028020020BE02002038270020C40200205C
:10C55000EC0200206D02002004290020CE02002001
:10C56000B902002098020020BC020020C80200206E
:10C57000750200203B00002070B5394C012004F109
:10C58000340520712878374EC0F30111307881428C
:10C590000BD9A1EB0000C1B24FF00A0000F0AAFED7
:10C5A000B4F91010B1FBF0F009E00ED2A0EB0100DD
:10C5B000C1B24FF00A0000F09DFE218A484320825C
:10C5C0003178287861F305102870217826480129F0
:10C5D00014D048F6D0210180287800F00301C0F380
:10C5E0000110814214D9A1EB0000C1B24FF00A0042
:10C5F00000F080FE6978B1FBF0F011E02978008846
:10C600000906218A01D4084400E0401A2082E3E7A9
:10C610000CD2401AC1B20A2000F06CFE697848437F
:10C6200068702878010961F3010028706878218A10
:10C630000A1A084462820D49A082002008700C4941
:10C6400008700C4908700C480078C01E042806D2F7
:10C65000BDE870404FF40041084802F04BB870BD8F
:10C66000B802002075020020420000207D02002058
:10C6700078020020790200203B00002010270020D3
:10C680001EB52C4AF12907D1B2F924102A4B994240
:10C6900002DD1184938401E0518C11842749CB7809
:10C6A0009C089DF8083064F387038DF808304B88A8
:10C6B0009C09BDF8073064F38913ADF807308B7817
:10C6C0005C089DF8073064F345038DF80730B1F836
:10C6D00001301C09BDF8063064F30813ADF80630CC
:10C6E0000B889C09BDF8053064F38B13ADF8053059
:10C6F00009789DF8053061F3050311498DF805307F
:10C700000988ADF80310118CADF8011052799DF82D
:10C71000001062F3461121F08F0141F010018DF8F5
:10C72000001000990160019941609DF808100172A4
:10C730001EBD0000700200200080FFFFD802002014
:10C74000420000200249C86A401CC86270470000CD
:10C75000340000202DE9F047064688B098469246FE
:10C7600089460020FEF7ECFB070C002406EBC4050D
:10C77000296B481C0ED0A88DB8420BD120236A46E5
:10C7800030462831FCF72EF8524669464846F5F700
:10C79000BAFD30B1641C102CE8D3002008B0BDE80D
:10C7A000F08706EBC400016BC8F80010E88D4FF667
:10C7B000EF71884202D34FF6FF7000E01030E88539
:10C7C0000120EBE72DE9F0410646487814460D4676
:10C7D0004FF0FF3701281CD0216B481C686808D037
:10C7E000F26802448A4214D3607828B1A0680144F8
:10C7F00003E02430BDE8F081091D3046243AFFF7FC
:10C80000B1F96968F2681144814202D3A168002934
:10C81000F0D13846EEE74A68531C0BD0C9684B1C70
:10C820000AD0C36801FB03218068806B884206D967
:10C830000846704700207047C1681144F4E74FF084
:10C84000FF30704710B5C36880689C18826B9442B3
:10C8500005D848681844904200D3002010BD4FF01E
:10C86000FF3010BD024640784FF0FF33012804D05E
:10C87000C86851692030884200D9184670470000C6
:10C880000249086B401C0863704700003400002018
:10C8900010B5002300EBC304D4F8AC408C4207D1A0
:10C8A00022B100EBC300D0F8B0001060012010BD31
:10C8B0005B1C042BEED3002010BD00002DE9FC41D1
:10C8C0002F4C0020A076F6F745F9411C00D02066D9
:10C8D000A17E19B9401C01D0206E2063206BF6F7B1
:10C8E0001DF928492063DFF8A0804978274E284F9A
:10C8F000054608293BD2DFE801F03A0431281F3110
:10C900002831F5F764FF234B0022CDE9002300BF57
:10C91000F9F7F2F82063F6F7CFF820631E48008895
:10C92000322800D22563206BFCF784FDA062F7F764
:10C9300075FA606ABDE8FC81F5F749FF154B0022E6
:10C94000CDE90023154A164BE2E7F5F740FF114BFE
:10C950000022CDE9002342463B46D9E7F5F737FFF1
:10C960000C4B0022CDE9002342463346D0E7F5F7D1
:10C970002EFF084B0022CDE900234FF07F53C7E77D
:10C9800028030020082C00209A9999999999B93F79
:10C990009999A93F0000E03F8E0200207B14AE472A
:10C9A000E17A843F0249486B401C486370470000AD
:10C9B0003400002011490868086840001BD5C81ED3
:10C9C00002782AB102780278027802780278007838
:10C9D0000A48001F027822B10278027802780278B1
:10C9E00000780648801E02882AB1028802880288E0
:10C9F0000288028800880868704700002CED00E07B
:10CA0000002070470120704710B50D48FEF74CFF1D
:10CA10000B486038FEF748FF0948C038FEF744FF6E
:10CA200008480021C162016341636B2001F074FD7D
:10CA3000702001F071FDBDE81040772001F06CBD61
:10CA40003C0C00203400002010B5FAF7A7FA00F0E3
:10CA5000ABFC00F011F8064800780E2801D1F6F77B
:10CA6000CDF804480068BDE8104002F0D3B90000DA
:10CA70003800002020020020174810B50068C16867
:10CA800041F01001C160642214491348F8F74AFFCD
:10CA900013480068C16841F01001C1606422114967
:10CAA0000F48F8F73FFF10480068C16841F01001D7
:10CAB000C16064220D490C48F8F734FF0C48006847
:10CAC000C16841F01001C160BDE81040642209490D
:10CAD0000748F8F727BF0000A807002098050020A6
:10CAE000E8070020FC050020280800206006002040
:10CAF00028070020C40600202DE9F04186B00C462E
:10CB00000C9D1E4617468046002100236A4640467B
:10CB100001F0B8FAD8B9D5B19DF80100022801D0CA
:10CB2000032814D10198243020632146404601F0A7
:10CB3000C1F9324639462046A84700280ED1224680
:10CB400069464046FFF73EFE2063401CEDD1694632
:10CB50004046FFF760FE0146401CD6D106B0BDE856
:10CB6000F081000070B50748074D046805E0022217
:10CB700006A12068F5F7C7FB083428688442F6D37D
:10CB8000002070BDE4040020E80400205F5F000086
:10CB9000F0B591B00026082306AA042101A800F0F0
:10CBA0002CF81020401EFDD206AF01A9304600F03F
:10CBB00036F80646002518E057F82540143CF5F7EE
:10CBC000D3FA217C9DF80C2021F08001914202D003
:10CBD000F5F7CEFA08E0F5F7CBFAE16904F11C00AD
:10CBE000814201D003F080FB6D1C0598A842E3DC74
:10CBF000002EDAD111B00020F0BD2DE9F04104463D
:10CC00001E4617460D46084602F016F8001D206025
:10CC1000257200206760C4E90360BDE8F0812DE95A
:10CC2000F0410D4600212961E96891B1297A81B16D
:10CC30002E6888B10446F5F797FA0146A4F114006E
:10CC40002A7A007C20F08000904209D00846F5F74F
:10CC50008FFA0020BDE8F0813446F5F785FA0146E9
:10CC6000686800272468B44201D1002404E010C0A1
:10CC7000EA687F1CBA42F5D10846F5F779FA2046F2
:10CC80002F61E7E77047F0B591B00026082306AAA8
:10CC9000022101A8FFF7B1FF1020401EFDD206AF10
:10CCA00001A93046FFF7BBFF0646002518E057F8FC
:10CCB0002540143CF5F758FA217C9DF80C2021F012
:10CCC0008001914202D0F5F753FA08E0F5F750FAE7
:10CCD000E16904F11C00814201D003F005FB6D1CE9
:10CCE0000598A842E3DC002EDAD111B00020F0BD97
:10CCF000F0B5B5B0002608232DAA012101A8FFF741
:10CD00007CFF1021491EFDD201A93046FFF787FFA5
:10CD10000646002520E02DA850F82540143CF5F7E4
:10CD200023FA0746207C9DF80C1020F080008842F2
:10CD300003D03846F5F71CFA0DE09022214606A8EC
:10CD4000F5F79CFA3846F5F713FA206B00E0401C23
:10CD500001782329FBD06D1C0598A842DBDC002E4E
:10CD6000D2D135B00020F0BDF0B591B00025082338
:10CD700006AA0A2101A8FFF740FF1021491EFDD293
:10CD800006AF01A92846FFF74AFF0546002404E044
:10CD9000F5F7EAF9F5F7ECF9641C0598A042F7DC21
:10CDA000002DEED111B00020F0BD72B6704700002A
:10CDB000F7F7A8FFFBF74DF8F8F76CFFF8F714FF4B
:10CDC000F8F7FEFFF8F7C4FFF8F7DEFFF9F714F8FD
:10CDD000F9F72EF803F0DCFB03F0AEFB4A4D4FF001
:10CDE000FF394946286802F030F8484C4FF40047B4
:10CDF00039462046F7F76EFF4FF48048D0B14646DB
:10CE000041462046F7F766FFA0B1FA2002F094F9F8
:10CE100039462046F7F75EFF60B131462046F7F706
:10CE200059FF38B1FFF7F0FDFCF764FC494628686C
:10CE300002F00BF84FF48059494626462046F7F792
:10CE400049FF334C334F012530B1207804280BD3F0
:10CE5000062809D0072807D041463046F7F73AFFA1
:10CE6000A0B12078042811D1FA2002F065F94946D2
:10CE70003046F7F72FFF20B941463046F7F72AFF33
:10CE800020B12078062800D125703D7003F01AFBF0
:10CE9000FAF70CFE3878012819D0F5F73FFFFAF7BA
:10CEA0008FFF2078022819D003F024FAFCF79CFFAA
:10CEB00003F040FA03F064F803F080F803F0E6FAB8
:10CEC00002F0D4FCF6F7F4FD00F064FC0AE0FCF795
:10CED00011FCF8F7CBFF03F0BBFA03E0FCF70AFC08
:10CEE0000D4805700D4C4FF4FA754FF40056284666
:10CEF00002F022F931462046F7F7F1FE8021204664
:10CF0000F7F7EDFEF3E7000020020020000C0140DF
:10CF10003B000020000000204E02002000100140D5
:10CF200010B501F05DFBBDE81040FFF741BF000008
:10CF3000F0B50B30154D20F007010024144A0FE026
:10CF400003688B420BD38B4205D95E1A431847689E
:10CF5000C3E9006700E04368136002C004E0021DFB
:10CF600010680028ECD12046002802D1286808B1BA
:10CF70000020F0BD064A07481060074A121A22F046
:10CF80000702C0E9002401202860D7E794050020AB
:10CF90009005002004B3002000B500202DE9F04FDB
:10CFA00081460878A3B00C464FF0000A022805D14C
:10CFB00000230A4619464846FCF76AFE01A948467E
:10CFC000A268FCF7F5FA0546401C15D099F829101F
:10CFD00004F1100BA1B124210CA8F5F768F9A2788F
:10CFE00059460CA8F5F76EF915AA0CA94846FEF7A4
:10CFF000A7FD00286CD103E0072023B0BDE8F08F27
:10D00000A2680023164601A9484603F01FFD01202F
:10D010000090062307AA29464846FBF72BFEA6F1F7
:10D02000140700261CE000BF06F12000B84201D220
:10D03000202000E0B81B8046C01C20F00303216BB9
:10D0400006F1140001440CAA4846FBF7CBFBA919D2
:10D0500043460CAA48461431FBF7CBFB82464644B4
:10D06000BE42E1D302200090062307AA2946484683
:10D07000FBF700FEA078C01C20F003004119E06817
:10D08000C01C20F003000A18D9F80C002832401EFA
:10D0900025EA0001484603F0C6FDA2782B46594612
:10D0A000484603F085FC0EA0FBF70EFB10A0D9F854
:10D0B0000010FBF709FB40F2BD320FA115A0FBF7F2
:10D0C00003FB0095A1785A4615A0236BFBF7FCFAE9
:10D0D0000123224600214846FCF7DAFD50468CE742
:10D0E0005B466C61736844425D5B6B765D0000007B
:10D0F0005B25735D200000002E2E5C666C617368FA
:10D1000064625C7372635C6664625F6B7664622EF9
:10D11000630000002825733A2564292000000000E0
:10D120004D6F76656420746865204B562028252E47
:10D130002A73292066726F6D203078253038582088
:10D14000746F203078253038582E0A002DE9F047CA
:10D150008046002500782C4618B12048204F0668EC
:10D160002DE0BDE8F0470021084600F05FB8062238
:10D170001CA13068F5F7C7F800BB306800F106095C
:10D180004046F5F7ABF8024649464046F5F7BBF88E
:10D19000A0B925B94C464846F5F7A0F805464946DA
:10D1A000204601E0401C491C02781AB10B780BB1F3
:10D1B0009A42F7D0001BA84200DA054608363868C4
:10D1C0008642D4D3002C06D02A4621464046BDE8EC
:10D1D000F04701F072BEBDE8F0870000E4040020D3
:10D1E000E80400205F5F636D645F000038B50446AB
:10D1F00001E0491E641C20782028FAD00928F8D0C4
:10D2000029B16A462046FBF7C1FD10B104E00020B9
:10D2100038BD009838BD641C2078202801D0002833
:10D22000F9D100202070401E38BD000070B50748BD
:10D23000074D046805E0062206A12068F5F763F8AB
:10D24000083428688442F6D3002070BDE40400202E
:10D25000E80400205F5F636D645F00000120704799
:10D2600070B500231C461E4640E000BF00F8016B6D
:10D270005B1C0578202D01D0092D01D18B42F5D3FF
:10D28000082C05D3002000E0401CA042FCD32FE076
:10D290008B422DD2EDB2222D03D042F82400641C23
:10D2A0001BE0401C42F824005B1C641C08E05C2D61
:10D2B00004D14578222D01D1401C5B1C401C5B1C15
:10D2C0000578222D01D08B42F1D38B4210D200F889
:10D2D000016B5B1C0AE0401C5B1C0578202D03D011
:10D2E000092D01D08B42F6D38B4201D28B42C0D3A1
:10D2F000204670BD034609B1012203E001207047BA
:10D300005843521C8A42FBDB704700002DE9F04174
:10D31000174688460546002440F2CD363A46414637
:10D320002846FCF745F9411C1AD195F82810002928
:10D3300016D0002C14D10BA0FBF7C6F90DA029685C
:10D34000FBF7C2F932460DA113A0FBF7BDF9394630
:10D350001448FBF7B9F92846FEF752FF0124DDE730
:10D36000BDE8F0815B466C61736844425D5B6B763F
:10D370005D0000005B25735D200000002E2E5C66C2
:10D380006C61736864625C7372635C6664625F6B39
:10D390007664622E630000002825733A25642920F4
:10D3A00000000000181C01087FB5394802901620C3
:10D3B0000390384A02213848FDF7C0FE374A03215E
:10D3C0003548FDF7BBFE002402AB35A235A132483B
:10D3D0000094FDF733FF002859D12E4A022132482C
:10D3E000FEF748F82D4A03212F48FEF743F8302571
:10D3F000CDE900542D4B2EA22FA12B48FEF7C4F8E7
:10D40000002844D1224A0621203A2748FEF732F864
:10D410002548204A02216030FEF72CF822481F4A96
:10D4200003216030FEF726F81F48CDE90054234B56
:10D4300023A225A16030FEF7A7F8002827D1144ABF
:10D4400019481C3A06216030FEF714F81248114AB8
:10D4500002216038FEF70EF80F48104A03216038A9
:10D46000FEF708F80720CDE900040B48184B19A275
:10D470001BA16038FEF788F8002808D1044A064846
:10D48000183A06216038FDF7F5FF00F0ADFB7FBDCF
:10D4900080000020ABCD00089C0C0020AD090108E5
:10D4A0006B760000656E76007C0B002045C7000897
:10D4B00074735F6B657900006B65790081C8000843
:10D4C00074735F706C616E00706C616E00000000C0
:10D4D000A5C9000874735F77656967687400000008
:10D4E0007765696768740000034902480860002096
:10D4F000704700000020000808ED00E030B5134937
:10D5000043680A68134402F1080498420DD05D880C
:10D510005DB94D68AB4208D08D689D4200D18860EE
:10D520005D6845605B68851A1D51836813448342BA
:10D530000BD05D88002D08D18D68854200D18B60AD
:10D54000416859604068991A015130BD14050020A6
:10D55000874FDFF820A2DFF820B24FF0000900BFAC
:10D560004FF0FF315446DAF8180001F06EFC8349A1
:10D5700000204E4600EB4002401C8E540A441E28F8
:10D5800056709670F6DB2671702003F017F90028AC
:10D5900061D0FEF745FB7D784FF0FF31DBF80000EE
:10D5A00001F053FCF878122802D0152858D052E028
:10D5B0007048282220213F3001F0D0FA6C48282200
:10D5C0002021503001F0CAFA6D496A4BDFF8A08182
:10D5D00000200A783F33A5F10A0108F150080CE059
:10D5E00007EB000C012A9CF804C003F800C001D02E
:10D5F000062A01D108F800C0401C8842F0DD5D49D0
:10D600007A19393112F8040C087012F8050C4870B8
:10D6100002202A183A4412F8052C0A54401C062805
:10D62000F7DBA670702001F09BFF5248FD213430DB
:10D63000C17053480078C01E042804D24FF4007112
:10D64000504801F057F8DBF8000001F0E3FB4FF41D
:10D650007A7001F071FD4FF47A7001F06DFD92E780
:10D66000434828222021503001F078FA404A002017
:10D670005032A5F10B0103E03B181B791354401CF9
:10D680008842F9DD7919DFF8EC8011F8060D08F110
:10D69000340800024A7800B202432282E28100206C
:10D6A0002918394411F8041C08F80010401C0528FA
:10D6B000F6DB98F80000400601D55042208298F829
:10D6C0000300FD2801D2012000E000202E4A6070F6
:10D6D000E68201252D4915702D4A0E70E90311804F
:10D6E00027490978C91E042915D220B321483930A9
:10D6F0008078C00703D000BF4FF4006101E04FF411
:10D700008061204800F0F6FFFEF7C2F94FF4804137
:10D710001C4800F0EFFF174839308178CA070FD056
:10D7200098F8022021F0010122F0800288F80220FE
:10D730008170267005E00221124800F0DBFFDBE774
:10D74000257098F80200000604D598F80300E178E7
:10D75000884201D1FEF710FF98F80300FD2802D39C
:10D76000702000F0D9FEDBF8000001F053FBF7E673
:10D77000B4280020B80200202C0200205A280020E3
:10D780003B000020102700204E02002078020020DD
:10D79000940200201CB50520009001904FF44073C6
:10D7A0000022064906A001F002FC0849002808638F
:10D7B00003D0BDE81C4001F00BBD1CBD51D50008D5
:10D7C000706F7070726F647563740000B80200202F
:10D7D00001B501231A4669460148F8F7F1F808BD7A
:10D7E0006807002030B504460D46826885B02021C8
:10D7F000174801F0B3F916496846A268FDF78EFB99
:10D8000001462046FEF702F901462846FDF789FB4E
:10D810002078022802D0002005B030BD0D49606894
:10D8200008640B49C878152810D1487800220B38B5
:10D8300003E08B181B798B54521C8242F9DD2022A5
:10D8400001E00A54401CA3688342FAD20120E3E7B6
:10D85000DC28002034000020F0B5054685B00F46D6
:10D860008068FFF765FBAA680446282A01D92826A4
:10D8700000E0D6B22021284801F070F92146684620
:10D88000AA68FDF74BFB01462846FEF7BFF80146A4
:10D890003846FDF746FB324621461F4801F01EF987
:10D8A000E078122831D1287802282ED12822202190
:10D8B0001A4801F053F928222021194801F04EF9A5
:10D8C00018490020154AC979154D08E02318012987
:10D8D0001B79135401D0062900D12B54401C6378C6
:10D8E0000A3B8342F2DA6178201F085C0E49087017
:10D8F0006278601F105C4870022062781319421F22
:10D900009A5C0A54401C0628F7DB2046FEF716FCFA
:10D9100005B00020F0BD0000B4280020F702002070
:10D920000429002034000020F102002070B50446D4
:10D9300086B00E468068FFF7FBFA05460021A26814
:10D9400001F00CF929466846A268FDF7E7FA01469E
:10D950002046FEF75BF801463046FDF7E2FAE8782C
:10D96000F42801D0E42802D12078022805D02846E6
:10D97000FEF7E4FB002006B070BD044901204873A7
:10D980002846FEF7DBFB0120F5E70000340000200D
:10D9900070B5044686B00E468068FFF7C9FA0546A2
:10D9A0000021A26801F0DAF829466846A268FDF76E
:10D9B000B5FA01462046FEF729F801463046FDF744
:10D9C000B0FAE878F82801D0E82802D120780228B7
:10D9D00005D02846FEF7B2FB002006B070BD044912
:10D9E000012008732846FEF7A9FB0120F5E7000097
:10D9F0003400002030B504460D46826885B0002111
:10DA0000134801F0ABF812496846A268FDF786FAA0
:10DA100001462046FDF7FAFF01462846FDF781FA48
:10DA20000B49A06804E00A1812F8012C0A54401EA1
:10DA30000028F8DC207A08702078022802D0002024
:10DA400005B030BD03486168816301620120F7E7DA
:10DA5000DC2600203400002030B504460D468268E4
:10DA600085B000210D4801F079F80C496846A2689C
:10DA7000FDF754FA01462046FDF7C8FF0146284647
:10DA8000FDF74FFA2078022802D0002005B030BD03
:10DA900003496068C86348620120F7E7B4280020A2
:10DAA00034000020F0B58BB005460C46072203A9D0
:10DAB00005A8FDF733FA01462846FDF7A7FF014602
:10DAC0002046FDF72EFA0E4A0E4E0720516C03AC8D
:10DAD000C1EBC103C0F1070703EB000CB444E75DE1
:10DAE000401E8CF804700028F4DC491C6868032987
:10DAF000C2E9111002D901200BB0F0BD0020FBE7F4
:10DB000034000020DC260020C1888288891AC2885F
:10DB100083889A4202D20089491C014488B2704726
:10DB2000C1888288891AC28883889A4202D2008971
:10DB3000491C014488B2704700238380C380491E7A
:10DB400001810260704770B50446C088A2880D4606
:10DB5000431C4FF0FF31934203D02389984204D1F4
:10DB60001AB9204600F00EF80146E2882068855474
:10DB7000E0882289904201D1002000E0401CE08032
:10DB8000084670BD81880268525C0389994201D1C0
:10DB9000002100E0491C818010467047818802689E
:10DBA000525C0389994201D1002100E0491C818027
:10DBB0001046704730B500F100648307094802D071
:10DBC00003685B1C0360002305E000BF14F8015BE1
:10DBD00001F8015B5B1C9342F8D34168491C41602A
:10DBE000104630BD1400002000B585B001227B49ED
:10DBF0006846FDF793F9024679A17A48FDF7B2F934
:10DC000076490122C91C6846FDF788F9024676A1CB
:10DC10007448FDF7A7F971490122891D6846FDF78F
:10DC20007DF9024671A16F48FDF79CF96B4901220D
:10DC3000491C6846FDF772F902466DA16948FDF777
:10DC400091F966490122891C6846FDF767F9024689
:10DC500068A16448FDF786F960490122491D6846BC
:10DC6000FDF75CF9024664A15E48FDF77BF95B496C
:10DC70000122091D6846FDF751F902465FA1594886
:10DC8000FDF770F95548401E4179012901D901215C
:10DC9000017052490122C91D6846FDF73FF902464D
:10DCA00057A15048FDF75EF94C4904220F316846F0
:10DCB000FDF734F9024655A14A48FDF753F94749A3
:10DCC000012208316846FDF729F9024652A145486C
:10DCD000FDF748F94149012209316846FDF71EF96F
:10DCE00002464FA13F48FDF73DF93C4901220A3168
:10DCF0006846FDF713F902464CA13A48FDF732F9A0
:10DD00003649042213316846FDF708F902464AA154
:10DD10003448FDF727F93149042217316846FDF7E9
:10DD2000FDF8024647A12F48FDF71CF92B490422B4
:10DD30001B316846FDF7F2F8024644A12948FDF779
:10DD400011F9264904221F316846FDF7E7F802461B
:10DD500040A12448FDF706F92049042223316846F2
:10DD6000FDF7DCF802463EA11E48FDF7FBF81B4913
:10DD7000042227316846FDF7D1F802463BA1194835
:10DD8000FDF7F0F8154902220D316846FDF7C6F897
:10DD9000024639A11348FDF7E5F8042239496846DF
:10DDA000FDF7BCF8024638A10E48FDF7DBF801226A
:10DDB00038496846FDF7B2F8024637A10948FDF731
:10DDC000D1F804222F496846FDF7A8F8024636A18B
:10DDD0000448FDF7C7F805B000BD0000350000207D
:10DDE000434800009C0C002054510000504D00009E
:10DDF000574C00004150490043430000424C45004D
:10DE000061645F50657263656E74000061645F4DAC
:10DE1000617876616C00000061645F465300000029
:10DE200061645F506F696E740000000061645F4957
:10DE30006E746576616C000061645F5370616E7A28
:10DE40000000000061645F5A65726F0061645F5496
:10DE500061726500726561645F6B65790000000046
:10DE6000726561645F706C616E0000007265616470
:10DE70005F77656967687400626567696E77656971
:10DE800067687400D8020020626567696E74696D06
:10DE900065000000BB020020636F6D706C657465E7
:10DEA0006F7264657200000054696D65436F6E7334
:10DEB000740000002DE9F04F93B00C464FF00009BC
:10DEC0000746CA46096B282301AAFAF78BFC0621EC
:10DED00001A8FAF798FCC0B22070079DA560691CE4
:10DEE000CB4605D0B968896B8D4201D8202D23D24D
:10DEF0002821A160052819D0052525703CA0FAF736
:10DF0000E3FB3FA03968FAF7DFFB4FF4A3723EA1B1
:10DF100044A0FAF7D9FB46A0216BFAF7D5FB009590
:10DF2000062301AA3846216BFAF7A4FE84F801B053
:10DF3000022013B0BDE8F08FF8682438854214D968
:10DF40008D4212D22AA0FAF7BFFB2DA03968FAF74A
:10DF5000BBFB40F24D122CA132A0FAF7B5FB3F4AB1
:10DF60003FA140A0FAF7B0FBFEE70026203D17E0F6
:10DF700006F12000A84201D2202100E0A91B88461A
:10DF8000C91C21F00303216B0BAA01443846FAF7A0
:10DF900029FC42460BA94846FCF7D2FF814646447D
:10DFA000AE42E5D30899494504D084F801B04FF05A
:10DFB000020A1AE0012060709DF82400256BC01C45
:10DFC00020F00303283504F1100229463846FAF7F9
:10DFD00009FC9DF82400C01C20F003002844606365
:10DFE0000A98E0609DF82400A0705046A1E7000068
:10DFF0005B466C61736844425D5B6B765D0000005C
:10E000005B25735D200000002E2E5C666C617368DA
:10E0100064625C7372635C6664625F6B7664622EDA
:10E02000630000002825733A2564292000000000C1
:10E030004572726F723A20546865204B562040300A
:10E040007825303858206C656E6774682068617375
:10E0500020616E206572726F722E0A00281001080E
:10E0600030000000282573292068617320617373D4
:10E07000657274206661696C656420617420257323
:10E080002E0A00002DE9F0430546C0680F46B1FB9B
:10E09000F0F100FB1170002697B099461446002855
:10E0A00012D05AA0FAF710FB5CA02968FAF70CFB13
:10E0B0004FF4BA725BA162A0FAF706FB634A64A14F
:10E0C0006AA0FAF701FBFEE7B4B124230EAA394691
:10E0D0002846FAF787FB676014986C494FF00008F0
:10E0E000A06088421BD084F800804FF0FF30E060D1
:10E0F000082017B0BDE8F08344A0FAF7E5FA47A07E
:10E100002968FAF7E1FA40F2751246A14CA0FAF735
:10E11000DBFA4E4A5EA155A0FAF7D6FAFEE70120D7
:10E1200020701598E06004210EA8FAF76CFB60706F
:10E13000042111A8FAF767FBA070B9F1000F62D0B3
:10E14000C4F810806068243060616078012802D0D3
:10E15000022803D057E0E86824380BE004F11402E9
:10E1600039462846FEF794FB30B161686069401A71
:10E17000E968081A206146E0E86824382061606890
:10E1800024300C9069462846FFF794FE9DF8010064
:10E19000A0B99DF80000012810D005280ED01BA0C2
:10E1A000FAF792FA1DA02968FAF78EFA3AA00C99AC
:10E1B000FAF78AFA0226C4F810800FE06069029923
:10E1C0006A460844606120690299401A206121462C
:10E1D0002846FEF7F7FA0C90401CD3D16068E96836
:10E1E000421828466169FAF7C0FA6169814205D090
:10E1F00060616268E968801A081A206128466269CD
:10E20000616802F010FD304673E700005B466C6108
:10E21000736844425D5B6B765D0000005B25735D57
:10E22000200000002E2E5C666C61736864625C7373
:10E2300072635C6664625F6B7664622E63000000EA
:10E240002825733A256429200000000030100108B9
:10E250006164647220252064625F7365635F736923
:10E260007A6528646229203D3D20300028257329E5
:10E270002068617320617373657274206661696CD4
:10E2800065642061742025732E0A000046444230E4
:10E29000736563746F7200004572726F723A205436
:10E2A0006865204B56202840307825303858292082
:10E2B000435243333220636865636B206661696C47
:10E2C0006564210A000000002DE9F0419AB09846EB
:10E2D00014000F4605464FF000060FD050236A4643
:10E2E000FAF780FA676003984F490027A0608842D8
:10E2F00016D0277008201AB0BDE8F0814BA0FAF7BD
:10E30000E3F94EA02968FAF7DFF9A5224DA154A040
:10E31000FAF7DAF9554A56A157A0FAF7D5F9FEE708
:10E320000120207004216846FAF76DFA60700498A5
:10E33000E060062107A8FAF766FA207606210EA803
:10E34000FAF761FAC0B26076217E022904D0022871
:10E3500006D0012909D00AE005982061069802E05C
:10E360000C9820610D98606101E001280CD0616873
:10E3700001F150002062EA6811446162091AE1610A
:10E380006178022912D03DE028A0FAF79DF92BA070
:10E390002968FAF799F9BF222AA131A0FAF794F96E
:10E3A000324A3DA134A0FAF78FF9FEE7B8F1000F29
:10E3B00028D0179020E000BF9DF8500010B31598AA
:10E3C000206117986061206A203020621698616A87
:10E3D000C01C20F00300081A6062179820301790C4
:10E3E0001698E169C01C20F0030000F12002914260
:10E3F0000AD9081A2038E06114A9284600F06AF802
:10E400000028D9D0304676E708A0FAF75DF90BA0CE
:10E410002968FAF759F9DDE9162120A0FAF754F92D
:10E420000226E761EEE7000054534C305B466C6116
:10E43000736844425D5B74736C5D00005B25735DC3
:10E44000200000002E2E5C666C61736864625C7351
:10E4500072635C6664625F747364622E63000000C2
:10E460002825733A25642920000000006E10010859
:10E47000736563746F7200002825732920686173C7
:10E4800020617373657274206661696C65642061D4
:10E49000742025732E0A0000300000004572726F50
:10E4A000723A20746869732054534C2028307825C0
:10E4B000303858292073697A652028257529206904
:10E4C00073206F7574206F6620626F756E642E0AFC
:10E4D0000000000030B589B00C460546C96820230D
:10E4E0006A46FAF77FF906216846FAF78CF9C0B256
:10E4F0002070012808D00698A06007982061059830
:10E50000606009B0002030BD286DA0604FF0FF3082
:10E5100020610020F4E700000E496B280AD0702823
:10E5200010D0486B0422401C886228310AA000BF2A
:10E5300002F010BCC86A0422401C0862054909A008
:10E540002031F5E7086B0422401C4862014908A00D
:10E550002431EDE734000020726561645F776569FE
:10E5600067687400726561645F6B65790000000024
:10E57000726561645F706C616E0000001CB5022002
:10E580001421CDE9000143020022044904A000F057
:10E590000EFDBDE81C4000F01BBE000021CF0008AE
:10E5A0006D61696E0000000070B54843044600F0DC
:10E5B0001DFA050003D02246002100F0CFFA2846BC
:10E5C00070BD000070B5044C044D02E02068804727
:10E5D000241DAC42FAD370BDAC1E0108B41E010864
:10E5E00070B5044C044D02E020688047241DAC4205
:10E5F000FAD370BDB41E0108BC1E010810B5F3F7B4
:10E60000B3FD044A5188491C5180BDE81040F3F71E
:10E61000AFBD00006C05002070B514460A460546E3
:10E62000042100F01BFB6C7405F11C042C6200201B
:10E63000EC61686270BD2DE9FF470546DDF830806A
:10E6400017460E004FF0FF304DD000F09BFD044602
:10E650000020A063F3F788FD8146F80704D0686ABC
:10E6600036EA000005D011E0B8070FD5686A3042DD
:10E670000CD0B8F1000F03D0686A3040C8F8000031
:10E6800078072CD5686AB043686228E0039868B3BD
:10E69000666484F848706A7C214605F11C0000F02D
:10E6A0004DF90398002809DD04F1540003AA002164
:10E6B000054600F06FFE284600F0A8FE4846F3F736
:10E6C00057FD00F0FBFAA06B00280CD1F3F74CFDCE
:10E6D0008146B8F1000F02D0616CC8F800104846BE
:10E6E000F3F746FDA06B04B0BDE8F0876FF00100C2
:10E6F000A063F4E72DE9F04105460C004FF0FF3030
:10E700002BD00027F3F730FD8046686A05F11C0620
:10E7100020436862EC69B44216D12AE094F82C10C8
:10E72000A4F11C00CA071AD0416C6A6A91431ED139
:10E7300090F848102468490703D5696A426C9143F0
:10E74000696200F000FD0127B442E7D14046F3F7CB
:10E750000FFD0FB100F0B2FA0020BDE8F08189078B
:10E7600005D5416C6A6A114001D04164E0E7246834
:10E77000EAE74046F3F7FCFCEEE7000010B5F3F7DC
:10E78000F3FC0B4C6188491E09B2618000290ADC48
:10E7900000216180F3F7ECFC6068002807D0BDE839
:10E7A000104000F08BBABDE81040F3F7E1BC10BD9B
:10E7B0006C05002070B5002825D0134D29688842CB
:10E7C00021D3696888421ED2A0F10C044FF0FF31BA
:10E7D0000E4800F03AFB002060804FF4F550208096
:10E7E000A868844200D2AC6029686068611A401A47
:10E7F0002969081A28612046FEF780FEBDE87040AE
:10E80000024800F007BB70BD1405002098320020BC
:10E8100000487047003300200048704700B30020D4
:10E8200010B5F9F73DFB10484FF47A710068B0FB62
:10E83000F1F0401EB0F1807F09D24FF0E0210B4A89
:10E840004861FF2010700020886107200861FFF7F1
:10E85000B9FEFFF7E1FF0446FFF7DAFF2146BDE806
:10E86000104000F03DBB00000400002023ED00E05C
:10E8700038B50B484FF0FF3400680168C94389067A
:10E8800002D44068C4B209E00168C943090702D450
:10E890000168406800900A2000F04EFCE0B238BDEC
:10E8A0006807002010B504460748016819B12046E2
:10E8B0008847002807D02078400701D5FEF718FACE
:10E8C000FEF778F8FEE710BDFC04002070B50446A2
:10E8D000121D22F007000022094D403840F8225056
:10E8E000521C102AFAD301620021416281624FF06A
:10E8F000807200F13005C263C16285E81A0070BD04
:10E90000EFBEADDE10B5F3F72FFC044A1178491CB9
:10E910001170BDE81040F3F72BBC0000100500207B
:10E9200010B5F3F721FC044A1178491E1170BDE8B7
:10E930001040F3F71DBC0000100500202DE9F04148
:10E94000064614460D46084600F058FC05F11C0723
:10E95000B4B1012C18D134680EE000BF95F83D1019
:10E9600094F82120A4F11C00914204D239461C30B5
:10E9700000F022F802E02468B442EFD1B44203D19F
:10E980003946304600F018F80020BDE8F0810268F2
:10E99000516002680A600160486070470268516017
:10E9A00002680A600160486070470268516002684E
:10E9B0000A600160486070474268116042684A60BE
:10E9C000416008607047D0E900124A60D0E9001247
:10E9D0001160406000607047D0E900124A60D0E9E1
:10E9E0000012116040600060704700002DE9F047A0
:10E9F000002807D0374CC01C20F00306E068864290
:10EA000002D90020BDE8F0870C2E00D20C264FF072
:10EA1000FF31314800F019FAD4F808C02168E768DE
:10EA2000ACEB0100BA1B4FE00D186B88E3BB6B68C1
:10EA30001B1A0C3BB34246D36A6806F11803121A3C
:10EA40000C3A4FF001094FF4F55A9A422DD383192D
:10EA50000C33CA184FF00008A2F800A0A2F80280F8
:10EA6000D5F80480C2E901806B60A5F80290506877
:10EA70000C37B84202D001F10802835020693044BB
:10EA80000C3020616269824200D26061A5F800A06A
:10EA9000654512D1A06842887AB1626890420CD074
:10EAA00040680844A060F6E70DE0A5F802906868A9
:10EAB0006A1A801A22691044E3E7074800F0AAF9AD
:10EAC00005F10C009EE768688242ADD8024800F06C
:10EAD000A1F996E7140500209832002010B50346EE
:10EAE000102A1DD341EA0304A40719D110C9103A12
:10EAF00010C310C9102A10C351F8084B43F8084B33
:10EB000051F8044C43F8044CF0D202E010C9121F33
:10EB100010C3042AFAD203E011F8014B03F8014BA9
:10EB2000521EF9D210BD000010B50346994211D211
:10EB30008C189C420ED9811804E000BF14F8013DE6
:10EB400001F8013D521EF9D210BD00BF11F8014B72
:10EB500003F8014B521EF9D210BD000010B5034658
:10EB6000CCB2042A1AD3810718D1194644EA0423E7
:10EB700043EA034306E008C1103A08C141F8083BE4
:10EB800041F8043C102AF6D201E008C1121F042A01
:10EB9000FBD20B4602E000BF03F8014B521EFBD232
:10EBA00010BD2DE9F0410F46064600F045F8054638
:10EBB000C068FFF71BFF040019D00021EA68FFF7C7
:10EBC000CDFF26740020607410223946204600F0E4
:10EBD00074F9F3F7C9FA064604F11401281DFFF78A
:10EBE000D6FE3046F3F7C4FA2046BDE8F081002097
:10EBF000FBE770B5044600202074F3F7B5FA05462C
:10EC000004F11400FFF7DFFE2846F3F7B1FA2046BF
:10EC1000BDE87040FFF7CEBD70B5044600202074FB
:10EC2000F3F7A2FA054604F11400FFF7CCFE2846DC
:10EC3000BDE87040F3F79CBA074A002102EB0113CC
:10EC40001B78834202D102EB01107047491C042952
:10EC5000F4DB0020704700002C0500202DE9F04176
:10EC6000044616460D460846FFF7E6FF0746FFF73F
:10EC7000C5FC381D796800E009688142FCD1FFF7C6
:10EC80007DFD45F08000207410223146204600F0C2
:10EC900014F9F3F769FA054604F11401381DFFF77A
:10ECA00076FE2846BDE8F041F3F762BA007C000624
:10ECB00001D5012070470020704700002DE9F04188
:10ECC000F3F752FA194D0746688838BBA868F9F778
:10ECD0001BFD1749401E6E6851F830401C3CB44281
:10ECE0001CD028706C60206B0178232906D1616AE2
:10ECF000814203D9626B1044884205D2FDF7F8FFC8
:10ED0000F3F732FA0028FDD10A48007804F1240113
:10ED1000002806F1240006D0F3F72DFA3846BDE8A6
:10ED2000F041F3F725BAF3F726FAF7E76C05002070
:10ED3000C03200201005002010B50446F3F714FA85
:10ED4000024694F83C000E4920F00F00401C84F865
:10ED50003C0094F83D0001EBC00104F11C004B683D
:10ED600018604B68236248600648E161216C836843
:10ED700019438160BDE810401046F3F7F9B900006F
:10ED8000C03200206C05002010B50446F3F7ECF902
:10ED900004F11C01D1E900235360D1E900231A607A
:10EDA0002162E16194F83D20074951F8323001EBCE
:10EDB000C2018B4204D10549236C8A689A438A6058
:10EDC000BDE81040F3F7D4B9C03200206C05002034
:10EDD00070B50C46014615460220FFF7E2FE0028FA
:10EDE00005D000F11C010162C1618484457470BDCD
:10EDF0002DE9F04116460A461F4605460221FFF757
:10EE00002DFF05F11C042C62EC61AE846F740020B0
:10EE1000BDE8F08170B50446F3F7A6F90546E06950
:10EE200004F11C01884208D01C3800F08CF92846F7
:10EE3000F3F79EF9FFF742FF05E0A08C401CA08489
:10EE40002846F3F795F9002070BD73B50546F3F732
:10EE50008BF90646A88C28B1401EA8843046F3F7EB
:10EE600087F921E0019808B300F08CF904460020EE
:10EE7000A0636A7C214605F11C00FFF75FFD019845
:10EE8000002809DD04F1540001AA0021054600F024
:10EE900081FA284600F0BAFA3046F3F769F9FFF72D
:10EEA0000DFFA06B002800D100207CBD3046F3F799
:10EEB0005FF96FF001007CBD704710B5002A07D0E4
:10EEC000034611F8014B03F8014B2CB1521EF8D147
:10EED00010BD03F8011B00E00021521EF9D110BD46
:10EEE000C01C10B521F0030120F0030018291FD920
:10EEF000A1F1180282421BD30E4C091A1839E160A5
:10EF00004FF4F5522060028000230C31C0E9011358
:10EF1000438043681844606002800122428041605F
:10EF20008160002304A10648FFF762FF2068A0600B
:10EF300010BD00001405002068656170000000002D
:10EF40009832002010B50A4900230A4C4B8018461D
:10EF500004EBC002401C526012600828F8DB072056
:10EF6000087003484B600C308B604060006010BD3F
:10EF70006C050020C032002010B5074CA068F9F7DE
:10EF8000C3FB0649401E51F830001C386060BDE8E4
:10EF900010402430F3F71DB96C050020C03200206A
:10EFA00001484060006070478405002070472DE9EB
:10EFB000FF478946DDE90C76824601461D469046AC
:10EFC0000120FFF7EEFD041E0DD02846FFF70EFDD1
:10EFD00060B103968DE8A10043464A46514620465B
:10EFE000FAF752F9204604B0BDE8F0872046FFF753
:10EFF00000FE0020F7E7000070B513480468F3F73F
:10F00000B3F805462046FFF7BFFE042084F83C0015
:10F0100004F1540000F0D6F92046FFF747FE01281E
:10F0200002D1D4F8880058B104F11C010748FFF759
:10F03000B5FC2846F3F79CF8BDE87040FFF73EBEEC
:10F040002046FFF7E9FDF4E7700500207805002071
:10F0500000F002F8FCE7000070B528E0F3F784F850
:10F060000546F9F789FE60B318480168A1F11C0450
:10F07000D1E900024260D1E90002106049600960F4
:10F08000FFF7BCFAD4F8881009B12046884720461B
:10F09000FFF70CFE01280FD0FFF770FB2846F3F7AF
:10F0A00067F8206BFFF786FB2046FFF7A2FDF9F714
:10F0B00063FE0028D2D170BD2046FFF7ADFDFFF7FB
:10F0C0005DFB2846BDE87040F3F752B87805002094
:10F0D0001FB5202308480722D9008DE80F00002320
:10F0E000064A07A1903800F00FF804B00248BDE8C6
:10F0F0001040903800F06CB89831002051F00008B2
:10F100007469646C650000002DE9FF5F92460EAAE9
:10F110000C4692E8E0010A46994683460121FFF732
:10F120009DFD8DE8E0014B46524621465846FAF7D0
:10F13000ABF804B0BDE8F09F10B500F0C1F8BDE831
:10F14000104000F025B870B5044690F83C0000F07F
:10F150000F00022802D04FF0FF3070BDF3F704F823
:10F16000054604F11C00FFF737FC04F1540000F0E1
:10F1700093F92846F2F7FCFF2046FFF7DDFD00205B
:10F1800070BD000001480068704700007005002055
:10F19000F1B5F2F7E9FF05460C480468204600F097
:10F1A0002DF804F154006A460021064600F0F2F8FA
:10F1B000304600F02BF92846F2F7DAFFFFF77EFD24
:10F1C000A06B801C00D1A0630020F8BD700500205A
:10F1D00010B590F83E10012280F83D108A400221BF
:10F1E000026480F83C10FFF7AEFF0348006808B1E6
:10F1F000FFF764FD002010BD7005002070B50446C7
:10F2000090F83C0000F00F00012802D04FF0FF30D2
:10F2100070BDF2F7A9FF054694F83C0020F00F00FE
:10F22000801C84F83C002046FFF7AEFD04F154003A
:10F2300000F032F92846F2F79BFF002070BD10B5B0
:10F2400004466FF00100A06304F11C00FFF7C4FB4B
:10F250002046FFF771FDBDE81040FFF72FBD00000D
:10F2600070B5F2F781FF06461348046894F83C0035
:10F2700000F00F00012819D1D4E90701884215D008
:10F2800004F11C000546FFF7A7FB94F83D000B496D
:10F2900001EBC00041680D6041686960456028600D
:10F2A0003046F2F765FFFFF709FD02E03046F2F75E
:10F2B0005FFF002070BD000070050020C0320020FC
:10F2C000002802DA4FF0FF3070474FF47A7190FB5C
:10F2D000F1F290FBF1F301FB130000EB40034A4312
:10F2E000C3EBC0104B1E03EBC00090FBF1F01044C9
:10F2F0007047000001480068704700000C050020BE
:10F30000094810B50168491C0160FFF73BFF016D1A
:10F31000491E016503D1C16C0165FFF7A1FFBDE87E
:10F32000104000F003B800000C0500202DE9F0416A
:10F33000FFF7E0FF0646F2F717FF0746144D1EE001
:10F3400060696FF00041301A1C3C88421AD2204696
:10F35000F9F7E2FFD4E909108847FFF7CBFF06462B
:10F36000607C810708D5C10706D020F001006074D9
:10F37000204600F04BF802E020F0010060742C6899
:10F38000AC42DDD13846BDE8F041F2F7F1BE0000F5
:10F390008405002049B1012904D0022908D003299D
:10F3A0000ED109E0C06A10600AE01168C16207E08E
:10F3B000417C21F0020102E0417C41F002014174F4
:10F3C0000020704770B50546F2F7CEFE0446284689
:10F3D000F9F7A2FF2046F2F7CBFE2846FFF71CFC08
:10F3E000002070BD2DE9F8439046DDE908450A4646
:10F3F0001F4606460A21FFF731FC23463A4641469E
:10F4000030460095F9F77AFFBDE8F883F8B5044671
:10F41000F2F7AAFE05462046F9F77EFF607C20F051
:10F42000010060742846F2F7A3FEFFF763FFE16A6C
:10F4300008442063F2F798FE0546164A0020009221
:10F4400002EBC002694653686FF0004C5DF8202063
:10F450000BE01268A2EBC0067769266BB74202D0B8
:10F46000BE1B664503D341F820209A42F1D10948DA
:10F47000001F0168491C016004F11C010098FFF79E
:10F4800094FA607C40F0010060742846F2F770FE48
:10F490000020F8BD8405002070B50446407CC007FC
:10F4A0000ED0F2F761FE05462046F9F735FF2846F3
:10F4B000F2F75EFE607C20F001006074002070BDF9
:10F4C0004FF0FF3070BD00207047002070470020D3
:10F4D00070470020704710B5F2F746FEFFF7A0F91D
:10F4E000FFF7EAFCFFF75CFDFFF72CFDFFF746F89E
:10F4F000FFF75CFDFFF7ECFDFFF73EFD002010BDC0
:10F500002DE9F04741258246157054265670572044
:10F5100090705220D070144689460D27177105222D
:10F5200021464846F6F7A6FA4FF4FA684146504697
:10F53000FFF78BFC78B9257066704320A0704E20D1
:10F54000E0702771052221464846F6F793FA4146B6
:10F550005046FFF77AFC5046BDE8F047FFF75ABC2B
:10F5600010B5034601F02AF900281ED00F496B2B75
:10F570000BD0702B11D0886A0422401C886228317D
:10F580000BA0BDE8104001F0E5BB086A0422401C56
:10F590000862064909A02031F3E7486A0422401CAA
:10F5A0004862024908A02431EBE710BD3400002076
:10F5B000726561645F77656967687400726561642C
:10F5C0005F6B657900000000726561645F706C615B
:10F5D0006E0000002DE9F05F9946DDE90B56DDF87D
:10F5E00028A0144688468346002700234246394611
:10F5F0005846FEF747FD1CB198F80100A0420DD116
:10F600002EB10123424639465846FEF73BFD2DB147
:10F61000524649464046A847002806D1414658462A
:10F62000FDF7F9F80746401CDFD1BDE8F09F2DE952
:10F63000F05FD1F804A0DDE90B799B4616460C4635
:10F64000804600250023224651464046FEF73CFEF8
:10F6500016B16078B0420FD1B9F1000F05D0012387
:10F66000224651464046FEF72FFE2FB1594620460E
:10F670000A9AB84700280BD1D8F80C002146054457
:10F680002A464046FDF7DEF88246B0F1FF3FD9D169
:10F69000BDE8F09F037863B14078012802D00228CA
:10F6A00004D006E00868401C086002E01068401CB6
:10F6B00010600020704700005B4E5C4DDFF870B1B9
:10F6C000DFF870A15C4C4FF0A1084FF07E09B078D4
:10F6D00001286ED15948007820B92878012806D031
:10F6E000032804D0564829780078084361D11720B0
:10F6F000207084F801901521A1705249484609787C
:10F70000E1702A78012A05D0032A03D04E490978EE
:10F71000092902D984F8048001E0F1212171607186
:10F720004520A071404F0020484B1837211813F88E
:10F7300000C081F807C0C0F1070C401C17F80CC0CE
:10F7400081F80FC00828F1DB2178002060540120E7
:10F7500004E0635C275C401C3B4463542178814295
:10F76000F7DCC8B2012A205CC0F1FF00605405D06C
:10F77000032A03D00120364A21783CE04FF0FF31C4
:10F78000DAF80000FFF761FB28784FF0C10201288A
:10F790004FF001010BD0022000F03EFB26492D481E
:10F7A00001F048FB01212C4BCBF8000007E00120C1
:10F7B000F2E733E0425C5F18491C07F8012C02783D
:10F7C0008A42F7DA2978012905D003290BD1234988
:10F7D0000978012907D1D2B21F492148F6F74AF921
:10F7E0003220FFF7A9FCDAF8000015E0235C1718B7
:10F7F000401C07F8013C8142F8DA1A4F4FF0FF3104
:10F800003868FFF722FB227811491748F6F732F9DA
:10F810003220FFF791FC3868FFF7FCFA4FF41670BE
:10F82000FFF78AFC53E70000280200203700002081
:10F83000D80100209C010020EC0100201C020020C7
:10F840001D020020350000203A000020042900207D
:10F8500070240020842B00207023002094010020BD
:10F86000E8070020A0010020280800207CB57E20A9
:10F870008DF800001A4804228DF8012000788DF8D8
:10F880000200184CF8208DF80300607900218DF8F3
:10F890000400401C607108466B461D5C401C2944F6
:10F8A000C9B20528F9DBC1F1FF008DF80500194642
:10F8B0000D48921C00F04AFF702000F07FFF0028E6
:10F8C0000DD0FCF7ABF84FF400710848FEF712FFBB
:10F8D0004FF47A70FFF730FCA069FFF79BFA7CBD0C
:10F8E00035000020B80200207C0B002010270020EB
:10F8F000F0B58BB004460146002608A8FCF7C0FE10
:10F9000008AB93E8070005AB83E807007E208DF87D
:10F9100000000F208DF801002F4805AA4FEA0D01C5
:10F92000007800F00F008DF802008DF803400920E8
:10F93000C0F109030C18D35C401EE3700028F7DC0B
:10F94000264D0027A5F13404E8788DF80D008DF8D8
:10F950000E7060798DF80F00401C607138460A5CAB
:10F96000401C3244D6B21028F9DBC6F1FF008DF8F6
:10F9700010009DF80100801CC2B2194800F0E6FE9C
:10F98000E8781649E0700422143916A001F0E2F973
:10F990007020FFF7E5FDF9F7ADFEF9F7D3FDE87844
:10F9A000FE2808D0A8784FF0010510F0780F05D098
:10F9B000A5810BB0F0BD00F001FBFAE70C480D4942
:10F9C0000222008808800CA001F0C4F92570A0690B
:10F9D000FFF720FAA781ECE735000020EC020020B9
:10F9E0007C0B002054696D65436F6E7374000000DA
:10F9F0009202002042000020626567696E776569A7
:10FA0000676874002DE9F0418CB00446002502219E
:10FA100008A8FCF735FE08AB6E4693E8070005AB77
:10FA200083E807007E208DF800000F208DF801008C
:10FA30002848092100788DF802008DF8034005A8B8
:10FA4000C1F109027318825C491EDA700029F7DCE3
:10FA5000214F4FF00008F42C33D0787A8DF80D0048
:10FA600097F80A008DF80E0078798DF80F00401C89
:10FA700078710020315C401C2944CDB21028F9DB9C
:10FA8000C5F1FF008DF810009DF801006946801C4B
:10FA9000C2B2124800F05AFEF42C0FD1104811499E
:10FAA00087F800800088088002220FA001F052F938
:10FAB0000949042220310FA001F04CF90CB0BDE837
:10FAC000F081F9F717FEFD20787240468DF80D8021
:10FAD000C8E7000035000020B80200207C0B0020A1
:10FAE0009202002042000020626567696E776569B6
:10FAF0006768740054696D65436F6E73740000002D
:10FB000070B526480721284A01707E2141700521E1
:10FB1000817023490978C170B221017121490978A6
:10FB2000417111788171491C11700021C17101214D
:10FB30000278445C491C835C2344835402788A42E3
:10FB4000F6DCD1B2425CC2F1FF0242540121C12273
:10FB5000084600F061F91149144801F06BF9144CA2
:10FB60000121144A206004E0435C5518491C05F843
:10FB7000013C03788B42F7DA0F4D4FF0FF312868D4
:10FB8000FFF763F920680B4902780C48F5F772FF1C
:10FB90002868BDE87040FFF73DB90000EC01002087
:10FBA0008C01002037000020BD020020842B0020A3
:10FBB000D8010020702300209C010020E8070020CD
:10FBC0002DE9F05FDFF8DCB0412554279BF80300F6
:10FBD0004FF050084FF030094FF00D0A4FF4FA661D
:10FBE00008BB334C304A31492068FAF719FC3146DA
:10FBF0002068FFF72AF998B92B48062201460570BC
:10FC00004770857080F8038080F8049080F805A024
:10FC10002648F5F72FFF31462068FFF716F970B137
:10FC20002068FFF7F7F8254C224A23492068FAF7A5
:10FC3000F7FB31462068FFF708F930B11FE01A4A98
:10FC40001A492068FFF75CFCEDE71A480570477019
:10FC5000857080F803809BF8031011B13221017187
:10FC600001E080F8049080F805A0062211491248AE
:10FC7000F5F700FF31462068FFF7E7F830B120685C
:10FC8000FFF7C8F8BDE8F05FF9F734BD094A0A4943
:10FC90002068FFF735FCF9F72DFD4FF4FA70FFF7F8
:10FCA0004BFAEFE7340000207024002028080020E1
:10FCB000A001002070230020E80700209C01002004
:10FCC00031B50C480099C161C27AB1FBF2F202EB86
:10FCD0008203D0E90C20141AB4EB430F09D38242FB
:10FCE00007D9002905D0FCF751FABDE83840F2F7F2
:10FCF000B5BF38BD280300202DE9F05FDFF8FC9088
:10FD000044274FF0410A99F803004FF054084FF090
:10FD1000490B4FF4FA66462538BB3B4C384A394903
:10FD20002068FAF77DFB31462068FFF78EF8C8B9E6
:10FD300033483721092280F800A080F8018080F83C
:10FD400002B0C7700171457185714521C1710D21E6
:10FD5000017201462B48F5F78DFE31462068FFF70A
:10FD600074F870B12068FFF755F82A4C274A2849E3
:10FD70002068FAF755FB31462068FFF766F830B186
:10FD800028E01F4A1F492068FFF7BAFBEDE71F482C
:10FD9000372180F800A080F8018080F802B0C77099
:10FDA00001714571857199F8021031B1092901D9A4
:10FDB000373100E03031C17100E0C5710D210172B1
:10FDC000092212491248F5F755FE31462068FFF71F
:10FDD0003CF830B12068FFF71DF8BDE8F05FF9F797
:10FDE00089BC0A4A0A492068FFF78AFBF9F782FCB6
:10FDF0004FF4FA70FFF7A0F9EFE70000340000209D
:10FE00007024002028080020A0010020702300207A
:10FE1000E80700209C01002070B5164B7E241025B9
:10FE20001C7000245C601D7201255D7201280FD0DA
:10FE30000228204616D0104C1E18255C401CB572B6
:10FE40000828F9DB4FF6FE70586119765A7670BDB6
:10FE50009C72DC721C735C739C73DC73FF201874DF
:10FE60005874EFE7054C1E18255C401CB572082835
:10FE7000F9DBE7E7842B0020DC010020E40100200F
:10FE80004FF08056B5103D4C6F004FF47A78A07853
:10FE9000C0F344011D2908D16288C2F38312022AEB
:10FEA00003D1E27812F00C0F17D11E2908D1628815
:10FEB000C2F38312022A03D1E27812F00C0F0CD0A5
:10FEC0001F2914D16188C1F38311042905D00629A3
:10FED00003D0092901D00B2909D120F03E00801C54
:10FEE000A070608806EBB0204FEAB0506080608858
:10FEF000C0F383110D290AD120F470704030608066
:10FF0000E078012101EB900161F38700E070207837
:10FF100005EBB0104FEAB06000F03F0120703C29C3
:10FF200008D120F03F002070208805EB30304FEAE8
:10FF3000305020802088C0F385113C290AD120F45C
:10FF40007C602080B4F8010007EB70204FEAF0508D
:10FF5000A4F80100B4F80100C0F30411182909D174
:10FF600020F4F870A4F80100A07807EBB0104FEA75
:10FF7000B060A0704046FFF7DFF888E7D8020020A5
:10FF80001CB505210320CDE900014FF48073002248
:10FF9000064907A0FFF70BF807490028886203D03D
:10FFA000BDE81C40FFF714B91CBD000081FE00082D
:10FFB00054696D6572000000B80200202DE9F05F01
:10FFC000DFF8ECB04FF0FF31DBF80000FEF73DFF4B
:10FFD0000020384A20211154401C2828FBDBDFF880
:10FFE000D8A03448EB239AF800202830C824A12553
:10FFF000BC26C6274FF0C7084FF0BB0C4FF0AE0928
:020000040801F1
:10000000012A04D0062A02D0032A10D01AE02B4A73
:10001000127862B1D6220270D8224270C122827058
:10002000BF22C270017141718171C1710AE080F813
:10003000008043708470C5700671477180F806C0F7
:1000400080F80790282220211D48FEF787FD1C49D3
:100050000020891FFE24C87008718A78088022F069
:10006000F7028A70A1F13902491F10820B7823F040
:10007000BF030B7048708B78CC7023F0FC038B703F
:100080005070507290729AF80000C01E042808D276
:1000900002210C48FEF72EFB4FF400610948FEF7E1
:1000A00029FBDBF80000BDE8F05FFEF7B3BE0000FF
:1000B0002C020020DC2800203B0000206D020020E4
:1000C000F7020020102700202DE9F041484C4FF4A2
:1000D0000048B4F91400A16A00F57A72914205DC77
:1000E000A0F57A72914208DA414509D0E28A032AE2
:1000F00003D2521CA062E28273E011F5004F70DD62
:10010000A1820020E082411E206BFEF79EFEB4F922
:100110001010A06A814200DA2082B4F912108142E4
:1001200000DD6082E16A0844E062E078401CE07033
:10013000607A401C6072206BFEF76CFE2D4D2978B2
:1001400011F00C0F4DD02C480078012849D12B4ECE
:10015000A06A2B4BB6F90020904207DD294FB7F972
:100160000070B84202DA1F78012F06D890421CDDD9
:1001700008061AD41878012817D1234800780428D3
:1001800001D006280CD1214F387848B92048007892
:10019000012805D041461F48FEF7ACFA012038700F
:1001A000207A401C2072208DA084B6F90010A06A2D
:1001B000884202DD2A78120604D5884205DA2A78B8
:1001C000120602D5F9F7C6F90BE0884202DA2A785E
:1001D000120604D5884204DD2878000601D5F9F717
:1001E000B1F9BDE8F04180210B48F4F778BD00007B
:1001F00070020020EC020020BC020020CA02002095
:100200003A000020CC0200203B000020BA0200206F
:10021000880100201027002000100140F8F7ECB9F9
:10022000064810B5006B0649401E884205D200F012
:1002300061FEBDE81040F2F711BD10BD280300209B
:100240007FF0FA022DE9F8431D465FEA02080746EF
:10025000894623D0234C0846F2F740F8C01C20F012
:100260000301E81C20F003000A1821463846283212
:10027000FDF74CF8401C18D0A4F138024946384626
:10028000FBF71CFC060013D00023A4F138024946FA
:100290003846F9F7FDFC04000AD01BE001230022D8
:1002A0003846F9F7F5FC04461AE00720BDE8F88364
:1002B00043464A460B4938460095F9F789FB044600
:1002C00046B13CB9074A0123383A49463846F9F75E
:1002D000DFFC044697F8280010B13846FBF790FF82
:1002E0002046E3E7640B0020016800E009688142D2
:1002F000FCD170471CB50520009001904FF480732D
:100300000022064906A0FEF752FE09490028C860EF
:1003100003D0BDE81C40FEF75BBF1CBD8D3F00084D
:10032000446973706C617964656C617900000000E8
:10033000280200201CB50520009001904FF4407366
:100340000022064906A0FEF732FE07490028886011
:1003500003D0BDE81C40FEF73BBF1CBDA93F000811
:10036000446973706C61790028020020354D364E67
:10037000364C4FF0FF373946E068FEF766FD01E086
:10038000F7F72EFB206AFDF7BFFB0028F8D122E02B
:1003900028780028606A08D0FDF7F4FB0146206C3D
:1003A000FDF7D1FBF7F7A6F808E0FDF7EBFB0146F8
:1003B000E06BFDF7C8FB01E0F6F756FEE06BFDF7DA
:1003C000A3FB0028F8D101E0F7F756F9606CFDF7C0
:1003D0009BFB0028F8D1606AFDF796FB0028D7D177
:1003E00021E0287880B13078012805D0032803D097
:1003F000A06AFDF7C7FB16E0A06AFDF7C3FB014644
:10040000206AFDF7A0FB0EE0A06AFDF7BBFB0146EA
:10041000606CFDF798FB01E0F7F72EF9606CFDF7D3
:1004200073FB0028F8D1A06AFDF76EFB0028D8D135
:1004300002E0E06AFDF7A6FBE06AFDF765FB002835
:1004400099D0F6E737000020390000208C01002009
:100450001CB504200521CDE90001C3010022064995
:1004600006A0FEF7A4FD08490028886003D0BDE877
:100470001C40FEF7ADBE1CBDA95E00084D656E7543
:100480004469737000000000280200201CB505209C
:10049000009001904FF440730022064906A0FEF739
:1004A00086FD07490028086103D0BDE81C40FEF71F
:1004B0008FBE1CBDB9F6000852656D6F74654400AF
:1004C000280200201CB504200521CDE9000103020B
:1004D0000022064906A0FEF76AFD08490028C86107
:1004E00003D0BDE81C40FEF773BE1CBD6D030108C0
:1004F000456D707479427566000000008C01002023
:100500000B4D0C4C4FF0FF364FF4C87731466868FE
:10051000FEF79BFC012240212046F4F7E8FB384619
:10052000FEF70AFE002240212046F4F7E0FBEDE74B
:100530004C020020001001401CB5002211460CA006
:10054000FEF746FC0E4C05214FF4807360600320DB
:10055000CDE9000100220B490BA0FEF728FD206128
:10056000002803D0BDE81C40FEF732BE1CBD0000D1
:100570007468726561645F626565705F73656D0064
:100580004C02002001050108626565700000000052
:100590001CB50022114631A0FEF71AFC334C002294
:1005A0001146206032A0FEF713FC35490022086096
:1005B000114634A0FEF70CFC3649002208600121E8
:1005C00035A0FEF705FC374900220860012136A05E
:1005D000FEF7FEFB38490022086038A13B48FEF7D1
:1005E0001BF8002201213AA0FEF7F2FB3B49002252
:1005F000086001213AA0FEF7EBFB3C4900220860AD
:1006000001213BA0FEF7E4FB3C49002208600121E8
:100610003BA0FEF7DDFB3D490022086001213CA024
:10062000FEF7D6FB3D490022086011463CA0FEF7CC
:10063000CFFB41494FF44873002208600521032095
:10064000CDE900013D493EA0FEF7B1FC6060002805
:1006500003D0BDE81C40FEF7BBBD1CBD74687265CD
:1006600061645F696E69745F73656D0020020020CC
:10067000706F705F70726F647563745F73656D0027
:10068000D002002064656C61795F6B65795F73658A
:100690006D000000D40200207765696768745F6CA4
:1006A0006F636B00A0020020646973706C61795FF6
:1006B0006C6F636B000000002C0200206469737093
:1006C0006C61795F6576656E74000000102700200C
:1006D00075617274315F6C6F636B000014020020EF
:1006E00075617274325F6C6F636B00009C01002057
:1006F00075617274335F6C6F636B0000A001002042
:1007000075617274345F6C6F636B0000A40100202C
:1007100075617274355F6C6F636B000018020020A6
:100720007468726561645F456D7074794275666660
:1007300065725F73656D00009801002049CA00086A
:10074000696E69745F656E7472790000F0B5194C5A
:10075000064685B0002020730D466073174616A12B
:100760003068F1F7C2FD30B9E878F82801D0E82800
:1007700001D1FBF77BF910A13068F1F7B6FD30B974
:10078000E878F42801D0E42801D1FBF75DF9207B5B
:10079000617B08430CD13A4629466846FAF7BEFB0E
:1007A00001463046FBF73EF810B1002005B0F0BD21
:1007B0000120FBE7340000206B6579000A496B28B3
:1007C00004D0702809D08A6A486B08E00A6AC86AAF
:1007D00005E030B1801A401C70474A6A086B8242BB
:1007E000F7D9002070470000340000202DE9FC41BB
:1007F0000446C06C0E46804705467068216D8842ED
:1008000012D927A0F7F760FF29A02168F7F75CFF4E
:100810004FF4AE7228A12FA0F7F756FF304A31A14E
:1008200037A0F7F751FFFEE72B46324604F12001CF
:10083000204600F041F9002830D12A4631462046B2
:1008400000F098FA070029D1206CC4E90C50203040
:1008500020647068616CC01C20F00300081A60649A
:100860007068E16BC01C20F00300081A2038E063B8
:10087000A06CA84201D8A5640FE009A0F7F724FFF7
:100880000BA02168F7F720FF0021A06CCDE9000143
:100890002A460B462248F7F717FF3846BDE8FC8189
:1008A0005B466C61736844425D5B74736C5D000011
:1008B0005B25735D200000002E2E5C666C61736802
:1008C00064625C7372635C6664625F747364622EFC
:1008D000630000002825733A2564292000000000E9
:1008E0008D100108626C6F622D3E73697A65203C41
:1008F0003D2064622D3E6D61785F6C656E00000086
:1009000028257329206861732061737365727420D0
:100910006661696C65642061742025732E0A00008D
:10092000001D010830B58DB00546002410482B4647
:10093000CDE900400494224603A918460294FEF72C
:1009400076FE6C656C62002305F120022146284684
:10095000AC64FDF7B9FC07A0F7F7B6FE09A029685B
:10096000F7F7B2FE09A0F7F7AFFE0DB030BD0000FB
:100970000DBF00085B466C61736844425D5B747335
:100980006C5D00005B25735D20000000416C6C20F5
:10099000736563746F7220666F726D61742066692F
:1009A0006E69736865642E0A0000000062B67047C5
:1009B0002DE9F041064610241F4625460020FAF78F
:1009C000BFFA010C00204FF6FF7384467A1C06EB39
:1009D000C00221D0B2F82CE08E4504D106EBC00055
:1009E0000763BDE8F081D2F830E0BEF1FF3F0FD0E1
:1009F000B2F82EE0BEF1000F03D0AEF1010EA2F866
:100A00002EE01FFA8EF29A420FD2054613460CE0F2
:100A1000102C0AD1044608E0928D8A4205D106EBDB
:100A2000C0004FF0FF3101630DE0401C1028CDD312
:100A3000102C02D206EBC40003E0102DD1D206EB3D
:100A4000C50007638185A0F82EC0CAE72DE9FF41E4
:100A50000746487800261D460C46012802D0022889
:100A60000AD025E0022000904968042301AA3846F4
:100A7000F8F700F906461BE02069482802D3801ADF
:100A8000482812D203200090042301AA3846616846
:100A9000F8F7F0F806466168F8680A18384600F07A
:100AA000C2F82DB10120287002E00DB100201870AD
:100AB00004B03046BDE8F0812DE9FF430546487893
:100AC00000268BB00C464FF0020802287ED15068F9
:100AD000E169C01C20F003002030814277D295F8F4
:100AE0005800002874D0206A05F148072038099082
:100AF000217E6668012011B1617EC9B13FE006F137
:100B00001C010090062304AA89462846F8F7B2F88B
:100B100000286CD104233A4606F114012846F7F761
:100B200068FE002863D1042309AA06F1180117E022
:100B300006F138010090062304AA89462846F8F7F2
:100B400099F8002853D104233A4606F1300128468B
:100B5000F7F74FFE00284AD1042309AA06F1340111
:100B60002846F7F746FE002841D1062304AA494645
:100B70002846CDF80080F8F77DF8002837D103200B
:100B80000090042301AA31462846F8F773F80600BE
:100B90002DD16068E9684718A868806B874200D348
:100BA000002705F120020023914639462846FDF72B
:100BB0008BFB607801281DD0A968E868896B3844F0
:100BC000884200D300203946686502E00AE028E048
:100BD0000CE02846FBF72CFA00234A463946284603
:100BE000FDF772FB6078012804D01AE007200FB0EF
:100BF000BDE8F08384F801800E99E160CDF80080B3
:100C0000042301AA28466168F8F734F80028EED1D9
:100C1000616804230EAA28461031F7F7EAFD0600A2
:100C2000E5D13046E3E770B5042400238A4216D9A3
:100C3000C5680D44954212D900EBC306D6F8AC50F6
:100C40008D4206D100EBC300C0F8AC10C6F8B0204E
:100C500070BD6D1C10D1042C0ED11C460CE000EBB5
:100C6000C305D5F8AC508D4206D100EBC3004FF060
:100C7000FF31C0F8AC1070BD5B1C042BD6D3042C24
:100C8000F9D200EBC400C0E92B1270BD10B5FEF71D
:100C900013F9002010BD00001349097801290DD077
:100CA00007290ED0042910D0092911D0082912D003
:100CB0004FF416520A2911D0426070474FF4E131C7
:100CC00001E04FF41671416070474FF49641FAE726
:100CD0004FF49661F7E74FF41641F4E70021016104
:100CE000C0E90121C1607047380000202DE9F047BC
:100CF00000F10064DFF8589090460F46800704D05A
:100D0000D9F80010491CC9F80010F3F7D3FE0025EC
:100D100012E03E680023324621460220F3F78AFEA5
:100D20002068B04205D0F3F77BFE4FF0FF30BDE8FE
:100D3000F087241D2D1D3F1D4545EAD3F3F770FEB6
:100D4000D9F808104046491CC9F80810EFE7000020
:100D50001400002010B586B004466846FAF7DEF8A5
:100D6000024621460248FAF75FF906B010BD0000BE
:100D70009C0C002070B50646056C8AB048680C468D
:100D8000CDE90620C01C716C20F00300081A089001
:100D900001200090062301AA29463046F7F76AFF92
:100DA000002818D10C2306AA05F114013046F7F7E4
:100DB00020FD00280FD1D4E9002330460899F7F729
:100DC00018FD002807D102200090062301AA294619
:100DD0003046F7F74FFF0AB070BD000010B5144A57
:100DE0004178517002210B4614E0C45C7E2C05D082
:100DF0007D2C03D0112C01D0132C06D17D2454540A
:100E0000C45C491CC9B284F020045454491C5B1CC6
:100E1000C9B2DBB204789C42E7D24B1E13700023A8
:100E200003E0D45CC4545B1CDBB28B42F9D910BD27
:100E30002C290020F0B50C782D4B04F10E024260F5
:100E400002785A708288120A9A700279DA70057AEA
:100E50001D71467A5E7135440622EEB200254719AF
:100E60006D1CBF7A9F54521CD2B29F18EDB217F876
:100E7000017C082D3E44F6B2F1D3858A2D0A9D549B
:100E8000521CD5B25A1912F8012C3244067D5E5517
:100E90006D1CEDB25E1916F8016C3244067E5E558B
:100EA0006D1CEDB25E19407E16F8016C58556D1C34
:100EB000E8B21D18324415F8015C2A44D5B201226B
:100EC000641C0AE08E5C1E54401CC0B21E18521CEA
:100ED00016F8016CD2B23544EDB2A242F2D3C5F19C
:100EE000FF01195418700248FFF778FF0048F0BD61
:100EF000C22900200148016B41637047280300208C
:100F000000000000000000000102030406070809B9
:100F1000000000000102030473746D33325F6F6ED2
:100F2000636869700000000000000000000000001D
:100F300000000008000004000008000005CA0008C6
:100F4000B5DB0008ED0C01084BA4000820000000F0
:100F500066616C5F696E697400000000180F01081B
:100F600066616C5F666C6173685F696E6974006668
:100F7000616C5F666C6173685F6465766963655F09
:100F800066696E640066616C5F7061727469746931
:100F90006F6E5F696E69740066616C5F7061727418
:100FA0006974696F6E5F66696E640066616C5F6725
:100FB00065745F706172746974696F6E5F74616289
:100FC0006C650066616C5F7365745F7061727469F3
:100FD00074696F6E5F7461626C655F74656D7000DB
:100FE00066616C5F706172746974696F6E5F72655F
:100FF00061640066616C5F706172746974696F6EC0
:101000005F77726974650066616C5F7061727469A4
:1010100074696F6E5F6572617365005F6664625FBD
:10102000696E69745F657800726561645F6B7600F4
:10103000726561645F736563746F725F696E666F1A
:1010400000666F726D61745F736563746F720066C2
:1010500064625F6B7664625F636F6E74726F6C0064
:101060006664625F6B7664625F696E697400726564
:1010700061645F736563746F725F696E666F00664B
:101080006F726D61745F736563746F720074736CFB
:101090005F617070656E64006664625F7473646241
:1010A0005F636F6E74726F6C006664625F7473640A
:1010B000625F696E69740000000000009630077777
:1010C0002C610EEEBA51099919C46D078FF46A703C
:1010D00035A563E9A395649E3288DB0EA4B8DC795C
:1010E0001EE9D5E088D9D2972B4CB609BD7CB17EDC
:1010F000072DB8E7911DBF906410B71DF220B06AAC
:101100004871B9F3DE41BE847DD4DA1AEBE4DD6DBB
:1011100051B5D4F4C785D38356986C13C0A86B64BB
:101120007AF962FDECC9658A4F5C0114D96C0663DB
:10113000633D0FFAF50D088DC8206E3B5E10694CBB
:10114000E44160D5727167A2D1E4033C47D4044BFB
:10115000FD850DD26BB50AA5FAA8B5356C98B242DB
:10116000D6C9BBDB40F9BCACE36CD832755CDF455B
:10117000CF0DD6DC593DD1ABAC30D9263A00DE518B
:101180008051D7C81661D0BFB5F4B42123C4B3567B
:101190009995BACF0FA5BDB89EB802280888055FFB
:1011A000B2D90CC624E90BB1877C6F2F114C68585B
:1011B000AB1D61C13D2D66B69041DC760671DB0149
:1011C000BC20D2982A10D5EF8985B1711FB5B6061B
:1011D000A5E4BF9F33D4B8E8A2C9077834F9000F5B
:1011E0008EA8099618980EE1BB0D6A7F2D3D6D08FB
:1011F000976C6491015C63E6F4516B6B62616C1CEB
:10120000D83065854E0062F2ED95066C7BA5011B1A
:10121000C1F4088257C40FF5C6D9B06550E9B712BA
:10122000EAB8BE8B7C88B9FCDF1DDD62492DDA157A
:10123000F37CD38C654CD4FB5861B24DCE51B53A9A
:101240007400BCA3E230BBD441A5DF4AD795D83D9A
:101250006DC4D1A4FBF4D6D36AE96943FCD96E34DA
:10126000468867ADD0B860DA732D0444E51D0333BA
:101270005F4C0AAAC97C0DDD3C710550AA410227CA
:1012800010100BBE86200CC925B56857B3856F209A
:1012900009D466B99FE461CE0EF9DE5E98C9D929FA
:1012A0002298D0B0B4A8D7C7173DB359810DB42E3A
:1012B0003B5CBDB7AD6CBAC02083B8EDB6B3BF9A86
:1012C0000CE2B6039AD2B1743947D5EAAF77D29D12
:1012D0001526DB048316DC73120B63E3843B6494F2
:1012E0003E6A6D0DA85A6A7A0BCF0EE49DFF0993F2
:1012F00027AE000AB19E077D44930FF0D2A3088762
:1013000068F2011EFEC206695D5762F7CB67658011
:1013100071366C19E7066B6E761BD4FEE02BD38911
:101320005A7ADA10CC4ADD676FDFB9F9F9EFBE8E71
:1013300043BEB717D58EB060E8A3D6D67E93D1A1B1
:10134000C4C2D83852F2DF4FF167BBD16757BCA691
:10135000DD06B53F4B36B248DA2B0DD84C1B0AAF31
:10136000F64A0336607A0441C3EF60DF55DF67A8B1
:10137000EF8E6E3179BE69468CB361CB1A8366BC41
:10138000A0D26F2536E2685295770CCC03470BBB91
:10139000B91602222F260555BE3BBAC5280BBDB291
:1013A000925AB42B046AB35CA7FFD7C231CFD0B531
:1013B0008B9ED92C1DAEDE5BB0C2649B26F263EC23
:1013C0009CA36A750A936D02A906099C3F360EEB31
:1013D0008567077213570005824ABF95147AB8E2F1
:1013E000AE2BB17B381BB60C9B8ED2920DBED5E5D1
:1013F000B7EFDC7C21DFDB0BD4D2D38642E2D4F121
:10140000F8B3DD686E83DA1FCD16BE815B26B9F6B0
:10141000E177B06F7747B718E65A0888706A0FFF10
:10142000CA3B06665C0B0111FF9E658F69AE62F8D0
:10143000D3FF6B6145CF6C1678E20AA0EED20DD7D0
:101440005483044EC2B30339612667A7F71660D0F0
:101450004D476949DB776E3E4A6AD1AEDC5AD6D930
:10146000660BDF40F03BD83753AEBCA9C59EBBDE50
:101470007FCFB247E9FFB5301CF2BDBD8AC2BACA00
:101480003093B353A6A3B4240536D0BA9306D7CD70
:101490002957DE54BF67D9232E7A66B3B84A61C490
:1014A000021B685D942B6F2A37BE0BB4A18E0CC350
:1014B0001BDF055A8DEF022D5F6664625F777269EC
:1014C00074655F737461747573005F6664625F72E4
:1014D0006561645F73746174757300C9E8B1B8B510
:1014E000D8D6B7CCE1C8A1B7BDCABDCDF8C2E7B167
:1014F000E0BAC5C9E8B1B8C0E0D0CD544D52CAFD7C
:10150000C1BF204150492020202020D0A3D5FDD6A6
:10151000D8C1BFD7EEB4F3B3C6C1BFC2CBB2A8C95E
:10152000EEB6C8D0A1CAFDB5E32020B7D6B6C8D65E
:10153000B52020B8F4C0EBD6D8C1BF202020202091
:101540002020204E45574C6162656C5A4D33303334
:10155000202020584B333139302020544D52203236
:10156000202020544D522033202020455A3334303F
:10157000302020414432353020202050544D20204E
:10158000202020542D323030302020534C31303048
:10159000303020584B33313930433854444932309D
:1015A0003049204944353131202020D7D4B6AF20EE
:1015B0002020202020202020202020BFD8D6C6C6D2
:1015C000F72020D4B6B3CCCFD4CABEB4F3C6C12062
:1015D000202020B4F3C6C131202020005C4333001A
:1015E000D4D8D6D8A3BAC7EBB1B8A3BA202020204C
:1015F00020BFC6C5C8CCDA544D5257617463682009
:1016000020202020202020C8ABBBECBACFC8D5C1F9
:10161000B8BCE0B9DCCFB5CDB32020200000C1C0FC
:1016200081C1400101C3C003800241C201C6C0069E
:10163000800741C70005C1C581C4400401CCC00C6E
:10164000800D41CD000FC1CF81CE400E000AC1CA2E
:1016500081CB400B01C9C009800841C801D8C0181E
:10166000801941D9001BC1DB81DA401A001EC1DE9E
:1016700081DF401F01DDC01D801C41DC0014C1D48E
:1016800081D5401501D7C017801641D601D2C012AE
:10169000801341D30011C1D181D0401001F0C0307E
:1016A000803141F10033C1F381F240320036C1F69E
:1016B00081F7403701F5C035803441F4003CC1FC6E
:1016C00081FD403D01FFC03F803E41FE01FAC03A2E
:1016D000803B41FB0039C1F981F840380028C1E85E
:1016E00081E9402901EBC02B802A41EA01EEC02E9E
:1016F000802F41EF002DC1ED81EC402C01E4C0248E
:10170000802541E50027C1E781E640260022C1E2AD
:1017100081E3402301E1C021802041E001A0C060BD
:10172000806141A10063C1A381A240620066C1A69D
:1017300081A7406701A5C065806441A4006CC1AC6D
:1017400081AD406D01AFC06F806E41AE01AAC06A2D
:10175000806B41AB0069C1A981A840680078C1B81D
:1017600081B9407901BBC07B807A41BA01BEC07E9D
:10177000807F41BF007DC1BD81BC407C01B4C0748D
:10178000807541B50077C1B781B640760072C1B2AD
:1017900081B3407301B1C071807041B00050C190FD
:1017A000819140510193C053805241920196C0569D
:1017B000805741970055C19581944054019CC05C6D
:1017C000805D419D005FC19F819E405E005AC19A2D
:1017D000819B405B0199C059805841980188C0485D
:1017E00080494189004BC18B818A404A004EC18E9D
:1017F000818F404F018DC04D804C418C0044C1848D
:10180000818540450187C047804641860182C042AC
:10181000804341830041C1818180404068656C6C98
:101820006F0076657273696F6E005F5F636D645FF2
:1018300076657273696F6E006C6973745F74687239
:10184000656164005F5F636D645F6C6973745F748E
:101850006872656164006C6973745F73656D005FC5
:101860005F636D645F6C6973745F73656D006C6951
:1018700073745F6576656E74005F5F636D645F6C43
:101880006973745F6576656E74006C6973745F74F8
:10189000696D6572005F5F636D645F6C6973745F2F
:1018A00074696D6572006C697374005F5F636D6469
:1018B0005F68656C70005F5F636D645F7073005F8D
:1018C0005F636D645F667265650000000100020081
:1018D00001000300010002000100040001000200F9
:1018E00001000300010002000100050001000200E8
:1018F00001000300010002000100040001000200D9
:1019000001000300010002000100060001000200C6
:1019100001000300010002000100040001000200B8
:1019200001000300010002000100050001000200A7
:101930000100030001000200010004000100020098
:101940000100030001000200010007000100020085
:101950000100030001000200010004000100020078
:101960000100030001000200010005000100020067
:101970000100030001000200010004000100020058
:101980000100030001000200010006000100020046
:101990000100030001000200010004000100020038
:1019A0000100030001000200010005000100020027
:1019B0000100030001000200010004000100020018
:1019C00001000300010002000100303132333435E0
:1019D00036373839616263646566003031323334DA
:1019E0003536373839414243444546006C69737493
:1019F0005F6D656D00000000466C61736820646572
:101A000076696365207C20252A2E2A73207C20613C
:101A10006464723A2030782530386C78207C206CF1
:101A2000656E3A20307825303878207C20626C6BE7
:101A30005F73697A653A20307825303878207C6980
:101A40006E697469616C697A65642066696E697330
:101A5000682E0000496E697469616C697A65206658
:101A600061696C65642120506172746974696F6E7C
:101A700028257329206F666673657420616464721B
:101A800065737328256C6429206F7574206F662038
:101A9000666C61736820626F756E64283C256429EA
:101AA0002E000000506172746974696F6E20777245
:101AB000697465206572726F72212020446F6E27F1
:101AC0007420666F756E6420666C6173682064654F
:101AD0007669636528257329206F66207468652000
:101AE000706172746974696F6E282573292E000005
:101AF000506172746974696F6E20726561642065EB
:101B000072726F722120446F6E277420666F756E3B
:101B10006420666C61736820646576696365282556
:101B20007329206F6620746865207061727469740F
:101B3000696F6E282573292E0000000050617274B1
:101B40006974696F6E206572617365206572726F6A
:101B5000722120446F6E277420666F756E64206654
:101B60006C61736820646576696365282573292034
:101B70006F662074686520706172746974696F6E35
:101B8000282573292E000000536563746F72206846
:101B9000656164657220696E666F20697320696E85
:101BA000636F72726563742E204175746F20666F67
:101BB000726D6174207468697320736563746F72E9
:101BC0002028307825303858292E0A00466F756E47
:101BD0006420616E204B562028252E2A73292077F9
:101BE0006869636820686173206368616E67656413
:101BF0002076616C7565206661696C65642E204E87
:101C00006F772077696C6C207265636F7665727987
:101C10002069742E0A0000005761726E696E673A7F
:101C200020416C6C6F6320616E204B5620287369D5
:101C30007A6520257529206661696C65642077685E
:101C4000656E206E6577204B562E204E6F7720777D
:101C5000696C6C204743207468656E2072657472ED
:101C6000792E0A005761726E696E673A204D6F7661
:101C7000656420616E204B56202873697A652025A3
:101C80007529206661696C6564207768656E2072CD
:101C900065636F766572792E204E6F772077696C59
:101CA0006C204743207468656E2072657472792ECB
:101CB0000A000000284644425F47435F454D5054A8
:101CC000595F5345435F5448524553484F4C442055
:101CD0003E2030202626204644425F47435F454D44
:101CE0005054595F5345435F5448524553484F4CF5
:101CF00044203C20534543544F525F4E554D2900DC
:101D00005761726E696E673A2063757272656E74A0
:101D10002074696D657374616D702028256A64296B
:101D2000206973206C657373207468616E20746819
:101D300065206C61737420736176652074696D65CC
:101D40007374616D702028256A64290A0000000000
:101D5000545344422028257329206F6C64657374A2
:101D600020736563746F7273206973203078253037
:101D700038582C2063757272656E74207573696EA5
:101D80006720736563746F72206973203078253023
:101D900038582E0A000000005761726E696E673A6B
:101DA00020536563746F7220737461747573206956
:101DB000732077726F6E672C20746865726520617E
:101DC0007265206D756C7469706C652073656374E1
:101DD0006F727320696E207573652E0A0000000013
:101DE00043430000424C4500434800004150490035
:101DF000574C0000504D00005451000061645F4694
:101E000053000000626567696E74696D65000000CB
:101E100061645F546172650061645F496E746576E8
:101E2000616C000061645F4D617876616C00000058
:101E3000726561645F706C616E00000061645F5A7E
:101E400065726F00636F6D706C6574656F72646549
:101E500072000000726561645F776569676874008D
:101E6000626567696E7765696768740061645F5071
:101E7000657263656E74000061645F506F696E74B3
:101E80000000000054696D65436F6E7374000000BC
:101E9000726561645F6B65790000000061645F5387
:101EA00070616E7A00000000D3F40008CBF40008E3
:101EB000E9D40008C7F40008E5BC0008CFF4000826
:101EC0001C18010801CA0008221801088D0C01081D
:101ED0002A1801088D0C010838180108F1CC0008F7
:101EE00044180108F1CC00085618010887CC0008F6
:101EF0005F18010887CC00086E18010891CB000814
:101F00007918010891CB00088A18010869CD0008EA
:101F10009518010869CD0008A618010865CB0008CE
:101F2000AB1801082DD20008B6180108C79900089F
:101F3000BF180108BD990008EC19010885CC0008FC
:101F400030315045626C00000000000000000000CD
:101F500000000000000000000000000073746D33FA
:101F6000325F6F6E6368697000000000000000005F
:101F70000000000000000000000800000000000059
:101F8000303150456170700000000000000000001A
:101F900000000000000000000000000073746D33BA
:101FA000325F6F6E6368697000000000000000001F
:101FB0000000000000080000008001000000000098
:101FC000303150456B76000000000000000000003A
:101FD00000000000000000000000000073746D337A
:101FE000325F6F6E636869700000000000000000DF
:101FF000000000000088010000F000000000000068
:102000003031504574735F706C616E0000000000E9
:1020100000000000000000000000000073746D3339
:10202000325F6F6E6368697000000000000000009E
:1020300000000000007802000068000000000000BE
:102040003031504574735F6B65790000000000000B
:1020500000000000000000000000000073746D33F9
:10206000325F6F6E6368697000000000000000005E
:102070000000000000E00200006800000000000016
:102080003031504574735F7765696768740000008C
:1020900000000000000000000000000073746D33B9
:1020A000325F6F6E6368697000000000000000001E
:1020B000000000000048030000B000000000000025
:1020C000E02001080000002098050000582A0008C0
:1020D0004C2201089805002068B300005C870008C6
:1020E000511324F43201022810192D120513040192
:1020F00012044202233075456666663F3B20231F6B
:10210000790401201EE81D01083537292C1AF80C26
:102110005A380C1AF40C5A3B0C1AF00C5A360C1A9A
:10212000EC0C5A370C1AE00C5A3A0C1AE40C5A39D7
:102130000C5E6C1E01083C0C1A240C1A440C320470
:102140001AFC245A3D181A78185A3E0C1A180C1901
:10215000BD390C1A9C0C5A48301A3C0C5A4C0C1ABB
:10216000100C5A500C1A900C5A540C1A300C5A5825
:102170000C1A540C5A5C0C1A600C1A420C32021ADB
:10218000040C4BD802181A440C1ABB0C296C9A8404
:10219000182910290401527BFFFF08137E1504370C
:1021A000F17E450A13019F5A2001410B2508084A78
:1021B000912241041580FF7F6A80B801115A7E8BFD
:1021C000AAFD4A0113021B044809D2BBBAC5C5A324
:1021D000C9E1B901312A025F0B1B01107F012803FD
:1021E00024803F181A303132333435363738390DC0
:1021F0000A3A2A48463630314141533730318462F9
:1022000080146302371CA306021123012E140880D8
:102210000444B880103A0AB32A01AE0299130C554F
:102220005C43311E014932011330052A20043290EB
:1022300032021A400C2904322832041A500C2904A4
:0C2240002910320A1A600C2904022F3405
:04000005080021319D
:00000001FF
